:020000040800F2
:1000000000000110A9440808ED2400082574020826
:100010004945080849450808494508080000000006
:10002000000000000000000000000000AD450008D6
:10003000B145000800000000B545000891E6000841
:100040004945080849450808494508084945080838
:10005000494508084945080831B0000835B000088E
:100060004945080839B000083DB00008F1270008EC
:1000700005280008192800082D2800084128000834
:100080005528000869280008494508084945080816
:1000900049450808494508084945080841B000088D
:1000A0009D260008C5260008ED26000889260008C0
:1000B00015270008292700083D270008494508089A
:1000C00049450808494508084945080849450808B8
:1000D0004945080849450808F1240008FD2400089E
:1000E00045B0000849450808B945000879270008C7
:1000F000A1270008C9270008652700087D280008F7
:100100004945080849450808512700084945080895
:10011000092500081525000849450808494508082B
:1001200091280008A5280008B9280008CD28000853
:10013000E1280008494508084945080849450808D4
:100140004945080849450808494508080546000882
:10015000F5280008092900081D29000821250008A4
:100160004945080849450808494508084945080817
:100170004945080849450808494508084945080807
:0801800049450808494508083B
:1001C000D0E907239A423CBFC1685218D01A704741
:1001D000D0E9092300699A4238BF1218D31A0138AE
:1001E000C01A7047D0E90902101AB0FA80F040092D
:1001F000704700BF0246036A4069D168C05C0133A2
:100200008B4228BF00231362704700BF436A826994
:10021000D154436A0169426B01338B4228BF0023EA
:100220004362D36843F08003D3607047436B188800
:1002300010F0100002D01A889B880120704700BF80
:10024000436B99891A88890610B504460AD592B27B
:10025000900607D5E26A002A2AD09888216B80B2DE
:100260009047636B99891A88090692B210D51006D7
:100270000ED5D4E909128A4215D0A1692069895C9A
:100280000132C9B29980B2FBF0F100FB1122A262E7
:10029000998A1A88C90592B204D5D20744BF4FF68D
:1002A000F7721A8010BDDA6822F08002DA60EFE798
:1002B0009B88E2696169DBB28B54E269E168636B38
:1002C0000132B2FBF1F001FB1022E261CAE700BF8C
:1002D000036942681F2B10B40AD95468A3F1200C9B
:1002E000202101FA0CF1214207D15DF8044B70473F
:1002F0001468202199402142F7D081690024C86800
:100300000C7480684C68016821F00101016020686C
:1003100094F805C00C4C818934F81C4089B221EA5C
:1003200004011F2B818107D9A3F1200120238B40D9
:100330005DF8044BD3607047202101FA03F35DF8A8
:10034000044B9360704700BF7C4C080882B00922C0
:10035000274B8DF80720DA68D00319D4DA68D10664
:1003600040D4DA68D20541D4DA6812F0E00F3BD10C
:10037000DB6813F0020F0CBF092308238DF8073048
:100380009DF80730012B0AD09DF8070002B0704796
:1003900001238DF807309DF80730012BF4D1144A62
:1003A00012E0D368DB0519D4D36813F0E00F17D13E
:1003B000D36813F0020F0CBF092308238DF8073010
:1003C0009DF80730012BDFD1D168C8034FF001033E
:1003D000F4D4D368D906E4D50623EFE70223EDE78A
:1003E0000723EBE70623D4E70723D2E70223D0E76E
:1003F000003C0240704700BF704700BF704700BF1D
:1004000001207047034BD3E90003C01AC0F30A0070
:10041000704700BF30220020054AD2E900139942FC
:10042000FDD0D1180133C3F30A03087A5360704733
:1004300030220020064BD3F8080800B97047D3F8E3
:100440000808A0F10500B0FA80F04009704700BF2D
:1004500030220020012380F849307047044BD3E953
:100460000003C01AC0F30A00C0F50060704700BF67
:100470003022002010B5D0F8E83504461B699847B3
:10048000032384F81231002010BD00BF08B50422F8
:1004900090F81211D0F8E83580F8131180F8122185
:1004A000DB689847002008BD08B5D0F8E435DB6963
:1004B00003B19847002008BD08B5D0F8E4351B6AA1
:1004C0009847002008BD00BF08B5D0F8E4355B6A46
:1004D0009847002008BD00BF70B5037805460E465A
:1004E0001446DBB1013082F0CBFE431CDBB201339A
:1004F0005B00DAB223800323327073702C7864B10E
:100500002846022300215A1CD2B2F454B15410F8E8
:10051000014F0233DBB2002CF5D170BD022213462D
:10052000E8E700BF10B5074C2068FF2808D006494F
:10053000D1F80C2801F5016100F082F8FF23236057
:10054000002010BD0000002030220020432301487D
:100550000B80704704000020122301480B80704775
:1005600048000020042301480B8070475C000020F5
:1005700010B5044C04480A462146FFF7ADFF20465B
:1005800010BD00BF482A0020A40A090810B5044C79
:1005900004480A462146FFF79FFF204610BD00BFD2
:1005A000482A0020B00A090810B5044C04480A463D
:1005B0002146FFF791FF204610BD00BF482A0020CA
:1005C000B80A090810B5044C04480A462146FFF74A
:1005D00083FF204610BD00BF482A0020C40A090836
:1005E00010B5044C04480A462146FFF775FF204623
:1005F00010BD00BF482A0020D00A0908704700BF7C
:10060000704700BF704700BF704700BF704700BF12
:10061000704700BF704700BF044B00200522C3F89D
:100620000828C3F81809C3F81C09704730220020B5
:10063000024B0020C3F80808704700BF302200209A
:10064000212838B50C4625D0222816D0202812D1D2
:1006500089B1072A0FD1174DD5F81C3913B1096894
:10066000002098472168A288A379C5F82019A5F829
:10067000242985F82639002038BD0029FBD0022A1C
:10068000F9D10C4BD3F81839002BF4D0098800208D
:100690009847F0E70029EED0072AECD1054BD3F8B4
:1006A0002019B3F8242993F826392160A280A37178
:1006B000E1E700BF3022002010B4114CD4E9003231
:1006C0009A1AC2F30A020A44B2F5006F13D871B144
:1006D00001444A1E013810F801CFE118904203F19D
:1006E000010381F808C0C3F30A03F4D1236000209A
:1006F0005DF8044B704702205DF8044B704700BF63
:100700003022002010B58121044679F02BFC2046D0
:10071000012179F027FC2046822179F023FCFFF7A4
:1007200087FF002010BD00BF034610B4D9691A69C5
:10073000002040F20114A3F844410860D1699C6D87
:1007400021F002014FF0010CD161A3F89CC320609D
:10075000D369044923F4003381F827095DF8044B79
:10076000D361704730220020202301480B8070475E
:1007700060000020122301480B8070478000002099
:10078000042301480B807047940000200A4608B5F6
:10079000054920B90548FFF79FFE034808BD0448F6
:1007A000FFF79AFE004808BD582B0020E00A090810
:1007B000F80A090810B5044C04480A462146FFF718
:1007C0008BFE204610BD00BF582B0020100B0908DF
:1007D0001C48D0F8E837D0F8EC2710B59B184FF03C
:1007E0001A040C8001D1184810BD174AD0F8EA0746
:1007F00002F1100411464FF0000E4FEA137CB3F1E2
:10080000204F34BF0CF1300C0CF1370C81F802C0D2
:1008100081F803E002318C424FEA0313EDD102F17B
:1008200008040021030FB0F1204F34BF30333733B9
:100830009374D174023294424FEA0010F2D102480C
:1008400010BD00BF00F0FF1F9800002010B5044C41
:1008500004480A462146FFF73FFE204610BD00BF70
:10086000582B0020240B090810B5044C04480A46F4
:100870002146FFF731FE204610BD00BF582B002057
:10088000300B0908034BD3F8B42BB3F8B83B1383F0
:1008900000207047302200204FF40070034B10609E
:1008A000D3F8F03D0B600020704700BF30220020DD
:1008B00000207047012070470120704700207047DA
:1008C00010B41C6994420CD394460A4661448C428D
:1008D000996938BFA4EB0C0261445DF8044B7EF0CB
:1008E000FFBF5DF8044B7047704700BF704700BF03
:1008F000D0ED007AD0ED036A30EE677AE6EE877AC3
:10090000B0EE670AC0ED007A704700BF90ED017A43
:10091000B5EE407AF1EE10FAF0EE407A09D19FED93
:100920000D7A60EE870AF7EE006A86EEA07A80ED17
:10093000017A31EE077A90ED000A80ED021AC1EEDD
:10094000076A77EEC07AC0ED036AA6EEA70A80EDCB
:10095000000A7047DB0FC940D0ED056AD0ED017A7F
:1009600090ED066AD0ED025A90ED035AC0ED066A8A
:10097000B0EE407A26EEA70AD0ED007A80ED057A37
:10098000A7EE870AD0ED077AA5EE860A90ED086AF1
:10099000D0ED045AC0ED087AA5EE670AA5EEC60AA6
:1009A00080ED070A704700BFF0EE406AD0ED007A94
:1009B00090ED050A90ED037A90ED016AD0ED025AB0
:1009C000A7EEA60AD0ED047A27EE407A67EEC07A49
:1009D000A6EE267AE5EEA67A90ED066AC0ED067AD6
:1009E00036EE076A80ED056A704700BF03685A1C3F
:1009F00002601970704700BF2DE9F04FD0E9003157
:100A0000856889B04A1C00EB81045918F1EE407AE0
:100A10000591002D92FBF3F103FB1122426000F1DE
:100A2000800A84ED200AC4ED407A00F5807240F31C
:100A30008780691C012603F1FF3B06914FF00209F4
:100A40000795B6460599A1EB090090FBF3F103FB6E
:100A50001100411C91FBF3F403FB14110AEB800815
:100A600002EB800CF14501EB0E00D8ED006A90FB23
:100A7000F3F49CED006AA3EB090603FB140055DDBB
:100A8000CDE90198CDE903C637460D46044641E05D
:100A9000AB420AEB840902EB840804F1010441DD56
:100AA0000AEB850C02EB85060135DCED007AD8ED0A
:100AB000005A96ED007AF4EEE67AF1EE10FA0FDDC8
:100AC00099ED005AF4EEC57AF1EE10FA08DDB4EEB5
:100AD000E65AF1EE10FA58BFF0EE456ACCED006A26
:100AE000B4EEC67AF1EE10FA0DDDB4EEE57AF1EE71
:100AF00010FA08DDF4EEC65AF1EE10FA58BFB0EE67
:100B0000656A86ED006A01375F4530DAB0EE476A04
:100B1000F0EE676AA342BBDCAB429046D1464FF091
:100B20000104BDDC1646D4460125BEE706990EF148
:100B3000010E714509F102090BF1FF3B82D1079DBE
:100B40000599491B91FBF3F003FB10130AEB83019A
:100B500002EB830391ED000A93ED007A30EE470A31
:100B6000F6EE007A20EE270A09B0BDE8F08FDDE945
:100B70000198DDE903C698ED006ADCED006A41E00A
:100B80008B420AEB800C02EB800700F1010041DD93
:100B90000AEB810502EB81040131D5ED007AD7ED36
:100BA000005A94ED007AF4EEC67AF1EE10FA0FD501
:100BB0009CED005AF4EEC57AF1EE10FA08D5B4EEC9
:100BC000C65AF1EE10FAD8BFB0EE456A85ED006A5C
:100BD000B4EEE67AF1EE10FA0DD5B4EEE57AF1EE68
:100BE00010FA08D5F4EEE65AF1EE10FAD8BFF0EE9E
:100BF000656AC4ED006A01365E4597DAF0EE476A31
:100C0000B0EE676A8342BBDC8B421746D4464FF096
:100C10000100BDDC144655460121BEE703685A1C9D
:100C200002601970704700BF024BD3F8200E0368B2
:100C30001B68184730220020007970470079C0F304
:100C40004010704700794009704700BF90F83C2081
:100C5000034602F0FF0012B1002283F83C207047E7
:100C60002DE9F84345697DB90768C7F30D080446C7
:100C70000E46B8F1000F0AD0D6F80080FFF766FBE9
:100C800009283BD06FF001052846BDE8F883514B99
:100C90009F422AD303F580439F4224D303F5804328
:100CA0009F427FD34C4B9F427FD903F580339F42B5
:100CB0007ED903F500339F427DD903F500339F426F
:100CC0007CD903F500339F4269D903F500339F4275
:100CD00077D903F580239F4276D9B7F1016F76D398
:100CE00005200DF079FD4FF00808FFF72FFB0928CC
:100CF00021D04FF0FF352846BDE8F883374E3369E1
:100D000023F440733361336943F40073336133690F
:100D100043F001033361C7F80080FFF717FB336925
:100D2000092823F001033361ACD123680433236025
:100D30002846BDE8F883DFF8A490D9F8103023F4F2
:100D40004073C9F81030D9F8103043F40073C9F873
:100D50001030D9F8103023F0F803C9F81030D9F862
:100D6000103043EA080343F00203C9F81030D9F801
:100D7000103043F48033C9F81030FFF7E7FAD9F8A0
:100D8000103023F00203C9F81030D9F810300928C8
:100D900023F0F803C9F810303FF46EAFA9E74FF025
:100DA0003808A2E74FF010089FE74FF018089CE7BB
:100DB0004FF0200899E74FF0280896E74FF03008E9
:100DC00093E74FF0400890E74FF048088DE74FF069
:100DD00058088AE700400008FFFF0008003C024076
:100DE0002DE9F0410446D0E90030134483421DD878
:100DF0000D4601EB0208B2B104F10C07002601E038
:100E0000A84510D023695A1C2261234415F8011B00
:100E10001973042AF4D139462046FFF721FFA8456B
:100E2000C4E90460EED16069BDE8F0814FF0FF30A5
:100E3000FAE700BF2DE9F0411F4E80460B4696F8B9
:100E4000242E002AFBD19BB343445F1E08F1FF38D8
:100E5000D6F8283ED6F82C2E0133C3F30A039A4263
:100E600016D10DF05DFC04460D460DF059FC001B3B
:100E700061EB0501B0F57A7F71F10001F5D3D6F889
:100E8000283ED6F82C2E0133C3F30A039342E8D050
:100E9000D6F8282ED6F8283E18F8011F3244013320
:100EA000C3F30A03B84582F8301EC6F8283ECFD1F6
:100EB0000020BDE8F08100BF302200200A4B10B5B1
:100EC000D3F8084804B910BDD3F80838052BFAD177
:100ED000064C002A0846D4F838351146F3DDFFF7F2
:100EE000A9FFD4F8383510BD302200202833002067
:100EF00090F84820531C0244DBB280F8483082F856
:100F0000341090F849204AB1132B06D9002280F8FA
:100F100048200C4AD2F8081829B9704780F84820B0
:100F2000002BF6D17047D2F80828052AF5D110B564
:100F3000054C19463430D4F83835FFF77BFFD4F828
:100F4000383510BD302200202833002090F848109A
:100F50000023A0F8483001B97047094BD3F808289E
:100F6000002AF9D0D3F80838052BF5D110B5054C77
:100F70003430D4F83835FFF75DFFD4F8383510BD7C
:100F800030220020283300202DE9F047564E1F461E
:100F900006EB80039C68002C00F0A28004F13E0365
:100FA000A36104F59F73E3614FF48073C4E90433D4
:100FB0002836236866600546E16094F83D00A36327
:100FC00091460AF00BF9804694F8440294F83CA04C
:100FD000261D002853D194F8450250BBD4F8403266
:100FE0006BBB3B0731D419F0020F5FD119F0010F31
:100FF00048D1D4F8483294F9471294F847221B019B
:101000000029DBB20DDB3949881880F8003350091C
:10101000012302F01F02934041F820303046BDE822
:10102000F087334902F00F02114430460B76BDE8D9
:10103000F08772F001F9D4F84032002BD1D02D4A5C
:10104000116B0B4313633B07CDD50135EDB207F0B0
:101050001003B8F1000FCCD040F2067288F80850A7
:10106000A8F8062094F84622002B34D117F0200F60
:101070000CBF3221122140460AF0A0FAB9E772F003
:10108000DBF8A8E750460AF0A9F86A1CD2B200289B
:10109000AFD0027240F20662012DC28094F846225F
:1010A0000CBF322102210AF089FAA2E76B1CDBB2E5
:1010B000B8F1000F9AD088F8083040F20653A8F82B
:1010C000063094F84622404602210AF077FA19F0D9
:1010D000010F8ED0D6E7022140460AF06FFA88E76A
:1010E00026463046BDE8F0877C4C080800E100E069
:1010F000FCEC00E0003802402DE9F047038A8489C7
:10110000A4B21C4082B047D0814688464FF00045CB
:1011100001F14C0701F13406B4FA84F325FA03F225
:10112000D24391B2A9F8101014401B3BB8F1000F44
:101130005FD0042B2ED8DFE803F052483D32030085
:10114000D8F80C30D9F82CA033B19B6823B11FFA22
:101150008AF108F104009847D8F8243033B19B682D
:1011600023B11FFA8AF108F11C009847D8F83C30E7
:1011700033B19B6823B11FFA8AF108F13400984714
:10118000D8F8543033B19B6823B11FFA8AF108F1C3
:101190004C009847002CBFD102B0BDE8F087D8F8CA
:1011A0000C30D9F834105B6808F104009847002C23
:1011B000B2D1F1E7D8F82430D9F838105B6808F1DB
:1011C0001C009847002CA7D1E6E7D8F83C30D9F8A6
:1011D0003C105B6830469847002C9DD1DCE7D8F87E
:1011E0005430D9F840105B6838469847002C93D1AA
:1011F000D2E7042B07D8DFE803F01903140F0A0025
:10120000D9F83C300193019B002C85D1C4E7D9F873
:101210002C300193019BF7E7D9F834300193019BFF
:10122000F2E7D9F838300193019BEDE7D9F8403067
:101230000193019BE8E700BFF8B5264C94F8242EF3
:10124000012A034603D0022A09D00020F8BD224E0D
:10125000D6F83C558DB984F8245E0020F8BD0025F1
:1012600040F20112C0E95455C0E95655A0F8442196
:1012700000F5A27178F072FFEDE7402D20D94027EC
:10128000D4F82C1E154AC3F858710A44C3E95422F5
:1012900040F20112A3F844210022C3F85C2103F5B7
:1012A000A271184678F05AFFD4F82C3E3B44ED1B4F
:1012B000C3F30A03C4F82C3EC6F83C550020F8BD21
:1012C000AAB2402A01D02F46DAE7022284F8242E5F
:1012D000D5E700BF302200202833002060300020F6
:1012E00001EB810138B500EBC1010F4DB1F88C1352
:1012F00004462846FFF7E0F9E378C4F8A853012034
:1013000083424FF000024FF04001C4E9EC12A4F810
:101310009C0304F56771204608BFC4F8AC5378F00D
:101320001DFF002038BD00BF68380020F8B52A4CEA
:10133000D4F880350F2B04D05A1CC4F88025002027
:10134000F8BD264D95F8243E0022C4F88025002BD8
:10135000F5D1D5F82C2ED5F8283E9A42EFD0D5F805
:101360002C2ED5F8283E9A422DD8D5F8286ED5F8DF
:101370002C3EF61A402E2BD8B3B2402B13BF374663
:10138000402702230123D5F82C2E85F8243E144B48
:10139000C0F858711344C0E9543340F20113A0F867
:1013A00044310023C0F85C3100F5A27178F0D6FE1C
:1013B000D5F82C3E3B44F61BC3F30A03C5F82C3E7C
:1013C000C4F83C65BBE7D5F82C6EC6F50066D1E7DE
:1013D00001234027D7E700BF283300203022002018
:1013E0006030002010B5324B93F8902593F8A4C5D7
:1013F000D3F88C35044613B152EA0C0231D00123E4
:10140000E06984F8463140F20112A4F844210268F0
:101410002849002AA8BFC2F380739B0301EA124146
:1014200043F020030B4363F31F42BCF1020F026041
:1014300000D010BDE278204BC4F8A8331F20002153
:10144000C4E9EC01012A4FF00101A4F89C1308BF84
:10145000C4F8AC3304F567712046BDE8104078F05D
:101460007DBE012178F044FD0122E06984F8462127
:1014700040F20113A4F84431016800290A460CDB4C
:10148000C1F380730B4C9B0343F0200304EA11412A
:101490000B4363F31F42026010BD064B03EA114386
:1014A00043F4804343F0200363F31F42026010BD06
:1014B00028330020DFBFFFFFAC3800202DE9F041CA
:1014C000B0F8CC15D0F8CE35B0F8D255B0F8D085FC
:1014D000C0F84051012284B080F8112101F01F02B0
:1014E000012A044600F2CC56ADF80810C1F3072ECD
:1014F000CDF80A30ADF80E504FEA134C51D0022A05
:101500007746C9B29BB210D0002A55D1BEF1090F5F
:101510004BD8DFE81EF08900AD004A00C8004A0041
:101520005C01DF004A001301330101F06001202952
:101530005FFA8CF272D0012F00F0B881032F00F017
:10154000A181AFBB90F81231022B00F0E381032B95
:101550002BD11CF0800F40F0E98102EB820200EBFE
:10156000C20393F87623003A18BF0122C24D02232A
:101570004FF48071C4E94E3384F81131C4F830312E
:10158000A4F81C1105F2B4530021C4F83411C4E9C5
:101590004A3304F58E712046C5F8B42578F07CFDF9
:1015A00006E090F81231032B0ED0204678F068FC4C
:1015B000002004B0BDE8F08101F0800178F098FCD3
:1015C000002004B0BDE8F0815FFA8CFCBCF1010F93
:1015D000EBD8D0F8E43502A99B689847BDF80E30E7
:1015E000002BE5D1C4E94A33C4E94C3304214FF45C
:1015F000807284F81111A4F81C2104F58E71204624
:1016000078F04AFD636D9D4A1A61E278012ACFD1D4
:101610005E614FF0802219681A60C9E7D0F8E4359E
:1016200002A99B689847C3E790F81231023B012B4F
:10163000BBD8914BD0F818210021C3F8AC1512B1DA
:101640000222C3F8AC258E4A02234FF48070002199
:10165000C4E94C31A4F81C01C4E94E33C4E94A2260
:1016600084F8113104F58E71204678F015FD9FE75E
:1016700090F81221023A012A97D8012B98D1D0F87C
:10168000E43500259B68C0F8185102A99847042248
:101690004FF48073C4E94A55C4E94C5584F81121CC
:1016A000A4F81C31A9E7012B00F03B81022B7FF449
:1016B0007FAF5FFA8CF3002B7FF47AAF03694FEAB8
:1016C0001C22023A5B68032A00F2BD81DFE802F0C7
:1016D000B6CED2D01E0A022EADF8065000F08A8196
:1016E000032E00F04E81012E7FF45FAFD0F8EC3571
:1016F00080781B680DF106019847BDF80630002B75
:101700003FF456AFBDF80E20002A3FF451AF93428C
:1017100028BF13464FF480720221A4F81C21002236
:10172000C4E94A0084F81111C4E94E33C4E94C32CB
:1017300004F58E71204678F0AFFC39E7012D7FF477
:1017400034AF90F81231022B00F00881032B7FF4A4
:101750002CAF4FF4807200F588730221A0F81C2191
:10176000002280F81111C0E94E55C0E94A33C0E9A2
:101770004C5200F58E7178F08FFC19E7DDB23E4FC8
:10178000012D87F8A5553FF610AF90F81231022BC6
:1017900000F0D880032B7FF408AF002D00F03581D6
:1017A00090F81011012910D0D0F8E4355B68984703
:1017B00097F8A515D4F8E43584F810111B68204675
:1017C0009847D4F8E8359B68984700230AE758EA19
:1017D00005027FF4EAAE90F8121103293FF4E5AE5A
:1017E00003F07F0580F814510069114663F30A1174
:1017F000036819430423016084F811314FF48073A6
:10180000C4E94A22C4E94C22A4F81C3104F58E71C3
:10181000204678F041FC636D184A1A61E278012A8B
:1018200006D0002D00F0FC80022384F81231BFE6C0
:101830005E614FF0802219681A60F2E702210E48BB
:1018400061F306130022C0F8B0350423C4E94A222C
:10185000C4E94C2284F8113101224FF4807304F55D
:101860008E7184F81621A4F81C31C8E60321E6E73E
:101870000521E4E70421E2E728330020180008608E
:10188000D438002090F81211022943D003297FF4A4
:101890008CAE23B9510602D0114678F029FBD4F85A
:1018A000E4359B6802A9204698478EE790F812110C
:1018B00002292FD003297FF478AE002B7FF478AE75
:1018C00012F07F0181D01CF0800F40F0AD8002EB60
:1018D000820100EBC10181F8763381F8753328234A
:1018E00081F8742303FB020300EB820193F8772352
:1018F000496D0B68023A012A23F400138CBFC3F32D
:101900000072012262F31C73D4F8E4250B60936823
:1019100002A9C8E753063FF44BAE114678F0E8FA47
:1019200046E6D0F8E425C0F81831F0E702F07F026F
:1019300002EB820200EBC20393F81E21003A18BFAB
:10194000012213E6002D3FF4A2AE01210322D0F8BC
:10195000E43580F8101180F812212FE73B4A80F817
:1019600011314FF480710023A0F81C11C0E94E55CD
:10197000C0E94A22C0E94C5300F58E7178F08CFB27
:1019800016E6DBB2052B3FF610AEDFE803F02B23A3
:101990001B130B03D0F8EC3580789B690DF1060121
:1019A0009847AAE6D0F8EC3580785B690DF106011E
:1019B0009847A2E6D0F8EC3580781B690DF1060156
:1019C00098479AE6D0F8EC358078DB680DF106018F
:1019D000984792E6D0F8EC3580789B680DF10601C7
:1019E00098478AE6D0F8EC3580785B680DF10601FF
:1019F000984782E6D0F8E43580789B6A0DF10601BD
:101A000098474670C4F8F00577E60222D0F8E4352E
:101A100080F8122180F810515B682946984736E615
:101A2000012384F81231C3E5282202FB010080F86B
:101A30001C1104EB810180F81E3180F81DE190F843
:101A40001F21896955E70121F9E600BFD038002040
:101A500010B5044629B990F81121032A0DD00020B1
:101A600010BDD0F8E4359B69002BF8D090F8122116
:101A7000032AF4D19847002010BDD0F890230B46DC
:101A8000D0F87C138A4219D9521AC0F8902394F8DE
:101A900003C0D0F880038A4228BF0A46BCF1010F78
:101AA00092B234D0C4E9E22304F55D71C4F8800336
:101AB000A4F87433204678F0EFFAD0E7D0F8E43594
:101AC0001B691BB190F81221032A1ED000234FF48A
:101AD00080720421C4E94A33C4E94C3384F81111FB
:101AE000A4F81C2104F58E71204678F0D5FA636DB8
:101AF0000D4A1A61E278012AB1D104F2CC545C613A
:101B00004FF0802219681A60A9E79847DEE7084479
:101B1000C4E9E22304F55D71C4F88003A4F87433CA
:101B2000C4F88403C6E700BF1800086038B504464F
:101B300049B990F81131022B11D094F81631012BCC
:101B400039D0002038BDD0F8E4355B69002BF8D0DF
:101B500090F81221032AF4D19847002038BDD0F81C
:101B60003831D0F8242193422FD990F803C09B1A22
:101B7000BCF1010F0D46C0F83831D0F828116ED0F5
:101B80009BB2C0F830314FF48073C0E94A11C0F8FD
:101B9000345100F58E71A0F81C3178F07DFAC4E95B
:101BA000E255C4F8805304F55D71A4F874532046DF
:101BB00078F072FAC1E73F4B2269D3F8B015516053
:101BC000002384F81631002038BDD0F83C31B3FB37
:101BD000F2F502FB15350DBB9A421FD8D0F8402113
:101BE00093421BD24FF48073A0F81C3100F58E7124
:101BF000C0E94A55C0E94C5578F04EFAE378C4F88C
:101C00004051012BC4E9E255C4F88053A4F8745341
:101C100008BFC4F8845304F55D71C8E7D4F8E4350F
:101C2000DB681BB194F81221032A15D0E278002357
:101C30000521012A84F81111C4E9E233C4F8803384
:101C4000A4F8743304F55D7124D0204678F024FAAA
:101C5000636D194A1A6170E720469847E6E79BB220
:101C60001144C0F830314FF48073C0E94A11C0F814
:101C7000345100F58E71A0F81C3178F00DFAC4E9EA
:101C8000E255C4F8805304F55D71A4F87453C4F8A8
:101C900084538CE7C4F88433204678F0FDF9636DF3
:101CA0000548186104F2CC525A614FF080211A683D
:101CB000196042E7283300201800086070B50B78DF
:101CC00013F060020D46044624D0202A04D020469A
:101CD00078F0D6F8022070BDCA8848781AB31B067F
:101CE00040D5324E3146FEF7ABFCEB884FF48072A4
:101CF0000221A4F81C21002284F81111C4E94E33FA
:101D0000C4E94A66C4E94C3204F58E71204678F085
:101D1000C3F906E04B780A2B10D00B2B08D0062B0A
:101D2000D5D0002070BD02221144FEF789FCF8E7EF
:101D30008B78C3BB1E4AC2F8B835F2E7022180F89F
:101D400011114FF48071A0F81C111A490123C0E948
:101D50004A11C0E94E33C0E94C3200F58E7178F07B
:101D60009BF9DEE71449154B0860E078C3F80C28AE
:101D7000002103F5016301284FF00305C4F88C131B
:101D8000A4F87413C4E9E42284F81151C4F8882338
:101D9000C4F8803304F55D7108BFC4F8843320466D
:101DA00078F07AF9BDE778F06BF8BAE7402A0020BE
:101DB00028330020E03800200000002030220020DE
:101DC000002310B519460446402278F0FBF8802124
:101DD00020460023402278F0F5F8D4F8E835A078C2
:101DE000012284F812215B689847002010BD00BFD3
:101DF00010B5022304464022812178F0E3F8204602
:101E000002234022012178F0DDF820460323082236
:101E1000822178F0D7F8104B0222A3F84C20FEF76D
:101E2000FBFBE2780D4BC4F8A8334021C4F8B01393
:101E3000012A4FF000004FF00101C4F8B403A4F8E8
:101E40009C13204604F5677108BFC4F8AC3378F0E2
:101E500085F9002010BD00BF000000206838002078
:101E600030B5812183B0044678F07CF8012120460A
:101E700078F078F82A4900250223402281F8275972
:101E80002046812178F09EF801210223402220463D
:101E900078F098F8234BD3F8BC2583F8A455126842
:101EA000284690470095009AE1681F4B42F01002C7
:101EB0000092009A0A610A690092013B02D0009ADE
:101EC000D006F8D400230193019B43F02003019333
:101ED000019A154B012060F38A120192019A0A615E
:101EE0000A690192013B02D0019A9206F8D4E27885
:101EF0000E4BC4F8A8331F200021C4E9EC01012ACD
:101F00004FF00101A4F89C13204604F5677108BF47
:101F1000C4F8AC3378F022F9002003B030BD00BF24
:101F20003022002028330020410D0300AC3800206F
:101F30002DE9F843DDF820800F46154600212022C8
:101F400004461E467FF0E4F8B8F1000F0CD0D8F834
:101F50000030E3811B0C2382D8F80430B8F80A2043
:101F6000E3821B0C62822383384681F089F9EB06F9
:101F700019D4431EB8B107EB000C01E0013B12D3AA
:101F80001CF801EDBEF12E0FF8D1C01A421E032A33
:101F9000A8BF0322082B03F10109A8BF082390461C
:101FA000B9441A4606E008280246B946A8BF0822E6
:101FB0004FF000084FF0203339462360636020461D
:101FC0007DF08EFC04F10800154B23814246494602
:101FD00083707DF085FC611EE21D11F801CFACF12C
:101FE0006103192B9CBFACF1200C81F800C0914219
:101FF000F3D104F10A0011F8013FA3F16102192A9B
:102000009CBF203B0B708142F5D118232373330C06
:10201000A382E572099B6683E361BDE8F88300BF94
:10202000202020002DE9F04FDFF858B4DBF8B40B86
:102030000C46BBF8B81B418385B0002B63D013441A
:10204000174604F5FE7A99461FE0002F69D0DBF8A9
:10205000FC3DBB4200F0CB80DBF8F83DBB4200F01A
:10206000FD80DBF8003EDBF8041EBB4250D8B942CD
:1020700000F27581791A204670F04EFB01374F450A
:1020800004F500740AF5007A39D0DBF8083EBB424B
:10209000DBD8DBF8185EFB1A296BDA0802328A42B9
:1020A00003F0070602D3AB6B9A420BD929461046C0
:1020B000029270F001FB029A0546002800F06F8141
:1020C000CBF8180E2B79002B40F02381D5F828800F
:1020D000B8F1000F00F05C812B6BD21AEB6806EBB5
:1020E000C20203EB422220462B464FF40071013717
:1020F000C0474F4504F500740AF5007AC5D1DBF8F6
:10210000B40BBBF8B81B0183002005B0BDE8F08F0D
:10211000B942AFD94FF40072002120467EF0F8FF9B
:10212000ACE74FF40072394620467EF0F1FF802381
:1021300084F8BE310C2384F8C231DBF8F81DC54A9F
:10214000DBF8F03DC4F8C6119142C4F8CA3100F37F
:102150000B81C14AC14D82FB010285FB01050A4486
:10216000C817C0EB6212C0EB2530BD4D84F8C10129
:1021700085FB0265C2EB82168010891B013120F0BD
:102180003F0015440843D117C1EBE5110A4484F818
:10219000BF21B04A84F8C001013B934200F3F080B4
:1021A000AD4AAE4882FB031280FB03101A44D917D4
:1021B000C1EB6212C1EB2031A94884F8C51180FB44
:1021C0000250C2EB821589105B1B013321F03F01E5
:1021D00010441943D317C3EBE0131A4484F8C41115
:1021E00084F8C3214AF65523A4F8FE3146E74FF0A0
:1021F000FF3384F8EC3184F8ED3184F8EE3184F863
:10220000EF315223237063706123A37084F8E731A8
:102210004123E37084F8E6317223002584F8E43129
:1022200084F8E531DBF8103EC4F8E8314FF4F07281
:102230002946201D7EF06CFF552384F8FE316FF097
:102240005503C4F8F051C4F8F451C4F8F85184F8B7
:10225000FC5184F8FD5184F8FF310FE74FF4007210
:10226000002120467EF054FF7E4B03CB45F6EB0366
:1022700023809023C4F80710A37002220821F823BA
:10228000C4F80300617322746375DBF8F03D2273B8
:10229000A27384F82C20DBF8F82D9B1A2362DBF85C
:1022A000002EDBF8043E9B1A63620023E372E373A3
:1022B0006377A377E37784F82D3084F82E3084F8A1
:1022C0002F3084F83130684BA361684BC4F842303A
:1022D0003E232377012384F83030654A802384F835
:1022E000403084F846104AF65521A4F8FE1103CA7E
:1022F000604BC4F84700C4F84B1003CB1388A4F814
:102300004F309378C4F85200C4F8561084F8513016
:10231000B4E64FF40072002120467EF0F9FE002E54
:1023200044D12B6C04F12008002B7BD02B6B52493D
:102330001122CDE900662046FFF7FAFD2B6C1A6CDE
:10234000002A7ED01B6B4D49CDE900664046112224
:10235000FFF7EEFD04F140084FF4E0736DE0F91A69
:10236000204670F0D9F989E6FF2284F8C1214FF6A2
:10237000FF72A4F8BF21374A013B93427FF710AFA9
:10238000FF2384F8C5314FF6FF73A4F8C33129E762
:1023900041464FF4007220467EF0BAFE6EE6384A9F
:1023A000231F43F8042F9A45FBD167E6D5E9102592
:1023B0003301002A43D0023B002D3FF45FAE013BC6
:1023C000AD6CF9D1A0464FF40073002D3FF456AE2A
:1023D000CDE9027A08EB0306A24608E00024CDE925
:1023E00000C4FFF7A5FDAD6CBDB1B04515D02C798B
:1023F00029682B6B404605F11C0C112208F12008BE
:10240000002CEBD16A792C6942F02102CDE900C49D
:10241000FFF78EFDAD6C002DE7D15446029FDDF82D
:102420000CA02BE6CDE900663346DBF8F41D08224C
:102430002046FFF77DFD4FF4F0736D6CC5E7013B5F
:10244000BAE7CDE900660D49334640461122FFF751
:102450006FFD7FE7FF03FB0083200882975545410E
:1024600081808080400B09083F00FF0029940E0DF9
:102470004C0B0908580B090840120908A413090855
:10248000DEADBEEF302200208C4613460146624688
:10249000184649F059BB00BF1049114BD1F88820AC
:1024A00042F4700210B4C1F888201A680D4C002064
:1024B00042F001021A6098601A6822F0847222F4D5
:1024C00080321A605C601A68074C22F480221A601D
:1024D000D8608C605DF8044B704700BF00ED00E0F1
:1024E000003802401030002400000008704700BF90
:1024F0000148FDF7A5BE00BFB80000200148FDF768
:102500009FBE00BF040300200148FDF799BE00BF35
:10251000500500200148FDF793BE00BF9C07002036
:102520000148FDF78DBE00BFE8090020704700BFDD
:10253000B0B130B443688D685A791C680223934067
:102540004A689BB26AB1A2899DB192B2134381607D
:10255000A381A3899BB243F00103A38130BC7047E0
:102560007047A28992B222EA0303A38165B1816018
:10257000EFE722F001021204120CA281A28981600D
:1025800092B21343A381E9E7A38923F001031B045B
:102590001B0CA3818160E1E738B5D0E9004007EE6C
:1025A000902A0068324A334B2468D3F8303C2468C0
:1025B000013990428DB210D002F5806290420CD069
:1025C00002F57052904208D002F58062904204D029
:1025D00002F58062904218BF5B0807EE103AF8EEF1
:1025E000677AB8EE477ADFED246A87EE270A30EE85
:1025F000260A79F0F5F91E492388421E8C4292B2D0
:102600009BB21AD01D498C4217D0B4F1804F1FD015
:10261000A1F580318C421BD001F580618C4217D02E
:1026200001F580618C4213D015498C4219D1238069
:102630000123E5622285A38238BD23F45C739BB23B
:1026400023800023E562228523860123A38238BDEF
:1026500023F45C739BB223800123E5622285A3826D
:1026600038BD08498C42E2D023F440739BB2DEE7C8
:1026700000000140000000200AD7233C0004014074
:102680000010004000140040024B0348D3F8C0156E
:10269000FEF732BD283300200000014010B5064C83
:1026A0000648D4F8C015FEF727FDD4F8E015044815
:1026B000BDE81040FEF720BD283300200000014097
:1026C0000040014010B5064C0648D4F8C015FEF78E
:1026D00013FDD4F8E4150448BDE81040FEF70CBD26
:1026E00028330020000001400044014010B5064C92
:1026F0000648D4F8C015FEF7FFFCD4F8E8150448E6
:10270000BDE81040FEF7F8BC28330020000001406F
:1027100000480140034B4FF08040D3F8C415FEF74A
:10272000EBBC00BF28330020024B0348D3F8C81588
:10273000FEF7E2BC2833002000040040024B0348AF
:10274000D3F8CC15FEF7D8BC283300200008004091
:10275000024B0348D3F8D015FEF7CEBC2833002037
:10276000000C0040024B0348D3F8DC15FEF7C4BC54
:10277000283300200004014010B5064C0648D4F868
:10278000DC15FEF7B9FCD4F8EC150448BDE81040A0
:10279000FEF7B2BC283300200004014000180040BE
:1027A00010B5064C0648D4F8DC15FEF7A5FCD4F8A5
:1027B000F0150448BDE81040FEF79EBC2833002009
:1027C00000040140001C004010B5064C0648D4F837
:1027D000DC15FEF791FCD4F8F4150448BDE8104070
:1027E000FEF78ABC2833002000040140002000408E
:1027F0000348D0F8403C13B100F634401847704706
:10280000000000200348D0F8603C13B100F65440AB
:1028100018477047000000200348D0F8803C13B1EF
:1028200000F6744018477047000000200348D0F8B5
:10283000A03C13B100F694401847704700000020F8
:102840000348D0F8C03C13B100F6B44018477047B5
:10285000000000200348D0F8E03C13B100F6D4405B
:1028600018477047000000200348D0F8003D13B11E
:1028700000F6F44018477047000000200348D0F8E5
:10288000203D13B100F61450184770470000002097
:102890000348D0F8403D13B100F634501847704754
:1028A000000000200348D0F8603D13B100F65450FA
:1028B00018477047000000200348D0F8803D13B14E
:1028C00000F6745018477047000000200348D0F805
:1028D000A03D13B100F69450184770470000002047
:1028E0000348D0F8C03D13B100F6B4501847704704
:1028F000000000200348D0F8E03D13B100F6D450AA
:1029000018477047000000200348D0F8003E13B17C
:1029100000F6F45018477047000000200348D0F834
:10292000203E13B100F614601847704700000020E5
:1029300002683649002310B422F0010221248842A3
:102940000260036043608360C3600361446138D008
:102950002F4B98422ED02F4B98423CD02E4B984272
:1029600040D02E4B984232D02D4B984241D02D4B27
:10297000984246D02C4B984217D02C4B98423CD0D2
:102980002B4B984216D02B4B984224D02A4B98427E
:1029900028D02A4B98421AD0294B984229D0294B4B
:1029A00098422ED0284B984208D14FF03D5243F820
:1029B000AC2C03E04FF4746243F8202C5DF8044B18
:1029C0007047224B5DF8044B3D229A607047204AC5
:1029D00043F8642CF2E74FF474125DF8044B43F8AB
:1029E000382C70474FF074625DF8044B43F8502C5C
:1029F0007047184A43F87C2CE0E73D2243F8082C46
:102A0000DCE7154A43F8942CD8E700BF1060024079
:102A100028600240406002405860024070600240FE
:102A200088600240A0600240B8600240106402402A
:102A300028640240406402405864024070640240CE
:102A400088640240A0640240B86402400060024012
:102A50003D000020400F002000003D20214A9368E7
:102A600003F00C03042B10B43AD0082B1FD01E4BDC
:102A70001C4C0360A1681D4AC1F30311114491F875
:102A80005C10CB404360A168C1F38221114491F8EE
:102A90005C1023FA01F18160A1685DF8044BC1F379
:102AA00042310A4492F85C20D340C36070475368B7
:102AB000516813F4800F536814BF0D4A0A4AC3F3D8
:102AC000881301F03F01B2FBF1F202FB03F3054A68
:102AD0005268C2F3014201325200B3FBF2F3C7E77E
:102AE000034BC5E7003802400024F4007C4C080882
:102AF00000127A0070B5446B8668A38923F40053F2
:102B00001B041B0CA381857990F805C02B0303F4EB
:102B10000051C5F380000CF001032A029B001CF059
:102B2000020F4FEA003002F4806218BF43F008033E
:102B300002431A43238A9BB223F440530B4323825C
:102B4000A38923F4B05323F00C031B041B0C134381
:102B5000A381A38A23F440731B041B0C84B0A382BB
:102B60006846FFF77BFF234B9C4205D003F580634B
:102B70009C4201D0029B00E0039BA2891E491204E3
:102B800003EB83034CBF7600B60003EB8303B3FB78
:102B9000F6F3A1FB0302A08952096426000406FB98
:102BA00012334FEA02121CD41B013233A1FB031370
:102BB000C3F3431313439BB223812A07A38A0AD585
:102BC0009BB243F00803A382A3899BB243F4005352
:102BD000A38104B070BD23F008031B041B0CA38267
:102BE000F2E7DB003233A1FB0313C3F342131343B9
:102BF000E1E700BF001001401F85EB512DE9F843CC
:102C00001D46344B9DF820609DF8249098428846DC
:102C1000174646D0304B98424BD0304B984250D05C
:102C20002F4B984235D02F4B98422ED14B463246EF
:102C300029460520FEF7A8F904460023C4E90B87BE
:102C4000C4E90733C4E909336671A56084F80690C6
:102C50002046FFF74FFFF107626B0ED4B30707D48E
:102C600093899BB243F4005393812046BDE8F883D7
:102C7000D36843F08003D360F2E74FF6DF7313802D
:102C8000D36843F02003D360E8E700242046BDE882
:102C9000F8834B46324629460420FEF775F9044670
:102CA000CBE74B46324629460120FEF76DF9044634
:102CB000C3E74B46324629460220FEF765F9044633
:102CC000BBE74B46324629460320FEF75DF9044632
:102CD000B3E700BF0044004000480040004C004003
:102CE0000050004000140140816003E7417101E79A
:102CF0008171FFE62DE9F043794F07EBC00985B0FC
:102D000005464FEAC00899F8380E08F067FA0446FD
:102D100099F8390E08F062FA064699F83A0E70F002
:102D20008BFA6B1CDBB2002C00F0AB8040F60C126F
:102D30002372E280002E00F0B680337240F60C233E
:102D40002046F38004223A2108F038FC0422304661
:102D50003A2108F033FC07EB0803624AD3F8344EFB
:102D6000944200F09680604B9C4200F0A2805F4B42
:102D70009C4200F0A980474497F83B3E022B32D09A
:102D8000032B7CD05A495B4F012B08BF0F46A68806
:102D90006846FFF763FE26F03F06029B564AB3FBE8
:102DA000F7F13604A2FB0323360C46EA9346A680CD
:102DB000228822F001021204120C22808AB2C1F38E
:102DC0000B019B0C09B942F001024FF4967101FB13
:102DD00003F34A49A1FB03139B0901339BB242F45D
:102DE000004223841FE0A6886846FFF737FE26F0DE
:102DF0003F06029A404B3604A3FB0213360C46EA08
:102E00009346A680218821F001010904090C218044
:102E10003B499209A1FB021292099B0C0133042A3F
:102E2000238438BF0422A2832388364A9BB243F00E
:102E300001032380238823F4816323F002031B040E
:102E40001B0C4FF4804143F480632380218123884D
:102E500023F080031B041B0C238023889BB202EB0E
:102E6000451243F0010323800121002382F8F85525
:102E700082F8F91582F8FA3505B0BDE8F083224FE3
:102E800085E7002E3FF467AF337240F60C23F380E2
:102E90005CE71E4B1A6A42F400121A621A6A22F4A4
:102EA00000121A6267E7042220463A2108F086FBE6
:102EB00051E703F5F0331A6A42F480021A621A6A83
:102EC00022F480021A6256E703F5EE331A6A42F4DE
:102ED00000021A621A6A22F400021A624BE700BF6B
:102EE000000000200054004000580040005C0040FA
:102EF000009F2400804F120083DE1B43D34D6210DD
:102F0000632D3E0528330020C02709000038024009
:102F10002DE9F047924E90F900108046807806EB3C
:102F2000C1050138CC0090B0D5F8341E14282DD836
:102F3000DFE810F04C012001150055005F009E00F5
:102F4000A600C301B6017A0084003C020402D70146
:102F5000C000D0002F003700A30195015401888ADA
:102F60000C8B81B27F4841EA0441884300F0208104
:102F7000D8E90201101A42F2107263EB010190428B
:102F800071F1000102D3152388F8023010B0BDE8BA
:102F9000F08798F813000882C8E90223122088F805
:102FA0000200888A0C8B80B240EA04406E4C844355
:102FB00000F0B28000200E900F9001200F910E9033
:102FC0000E99002900F017820F9914310F910F9973
:102FD00009684905CCD5142388F80230D6E798F85B
:102FE000110000F0FE000882C8E90223052088F8DD
:102FF0000200888A0C8B80B240EA04405B4C844318
:1030000000F0A1800020009001900120019100902B
:103010000099002900F0FB81019914310191019977
:1030200009684F05D7D4A3E798F8110040F00100D4
:103030000882C8E902230B2088F80200888A0C8BDA
:1030400080B240EA04404A4C84436DD00020049092
:1030500005900120059104900499002900F0D18188
:10306000059914310591059909684D05B3D47FE799
:1030700098F813000882C8E90223072088F80200A4
:10308000888A0C8B80B240EA0440374C84435ED07F
:1030900000200290039001200391029002990029E0
:1030A00000F0C181039914310391039909684E0519
:1030B00091D45DE7088820F480600004000C08804B
:1030C00098F8110000F0FE000882C8E902231020E1
:1030D00088F80200888A0C8B80B240EA0440234CB6
:1030E000844312D000200C900D9001200D910C9083
:1030F0000C99002900F091810D9914310D910D99D1
:10310000096848053FF567AF32E798F81330FF2BA1
:1031100006D198F810301BB1132388F8023035E738
:10312000112388F8023031E7D8F81400012800F0A4
:103130008F81022800F04382098B0E21C8E9022307
:1031400088F8021022E7062388F802301EE7D8F834
:103150001400002800F06D81082388F8023015E77C
:103160000000002001000300840007008200070027
:1031700002000300088820F400600004000C0880AE
:10318000088880B240F480600880088880B240F4EB
:1031900080700880032088F80200888A0C8B81B236
:1031A000A94841EA04418843C8E902237FF4EEAE0E
:1031B00098F81230002B40F0CE8198F81330FF2B96
:1031C00000F03F82042388F80230DFE60988890591
:1031D0003FF5CEAE002388F80230D7E6344494F8A9
:1031E000380E07F0FBFF064694F8390E07F0F6FF9D
:1031F000964AB2F8583601339BB28246A2F8583646
:1032000016B13368B2881A83BAF1000F04D0DAF825
:103210000030BAF804201A831121304605F03EFC34
:103220001121504605F03AFC4FF0090965272EB1EF
:103230003368B28819690A4240F02381013F00F0E7
:103240001D810BF06DFA04460D460BF069FA001B68
:1032500061EB0501052871F10001F6D3E7E7088865
:1032600080B240F4007008804FF6FF308882012160
:10327000C8E9022388F8021088E6D8F8140000286C
:1032800000F06D81D8F8184014F8016B0E820138F7
:103290001225C8E90504C8E9022388F8025075E63A
:1032A000888A0C8B81B2684841EA044188437FF4E4
:1032B0005FAE0A2388F8023068E6088880B240F4DE
:1032C00080700880092088F80200888A0C8B81B2FF
:1032D0005D4841EA04418843C8E902237FF456AEC1
:1032E000E7E7002401250A940B940B910A950A98AC
:1032F000002800F047810B9814300B900B98006861
:1033000046077FF535AED8F81400032800F06D812C
:10331000022800F24381088820F480600004000C39
:103320000880088880B240F400700880098A88F814
:103330001C40C8E9022388F8025027E60020012437
:1033400008900990099108940898002800F01481C9
:103350000998143009900998006847077FF508AE6E
:10336000EFF31185102080F31288088880B240F4B2
:1033700000700880D8F818000E8A471CC8F818702A
:10338000EDB2067085F311880D8AD8F818106FF029
:1033900001004E1CC8F818600D70C8E90223C8F877
:1033A000140088F81C4088F80240EFE500200690E1
:1033B0000790012007910690069C002C00F0E88001
:1033C000079C14340794079C246864067FF5D0ADED
:1033D0000C8AD8F818104D1CC8F818500C70D8F882
:1033E000141088F81C000139C8E90223C8F8141029
:1033F00088F80200CAE50F9918310F910F990968F2
:10340000B6E505991831059105990968B0E5019966
:103410001831019101990968AAE50D9918310D91AA
:103420000D990968A4E50399183103910399096876
:103430009EE5088880B240F4007008800121C8E948
:10344000022388F80210A1E50100030028330020C0
:10345000088820F480600004000C0880EFF31184D9
:10346000102080F31288088B088880B240F4007026
:10347000E4B2088084F311880C215FE616B133684A
:10348000B2885A830BF04CF904460D460BF048F90C
:10349000001B61EB0501052871F10001F6D316B19F
:1034A0003368B2881A830BF03BF904460D460BF0E3
:1034B00037F9001B61EB0501052871F10001F6D316
:1034C000B9F101097FF4B2AE16B13368B2885A83FC
:1034D0000BF026F904460D460BF022F9001B61EBB8
:1034E0000501052871F10001F6D3BAF1000F04D0EF
:1034F000DAF80030BAF804205A830BF011F90446C8
:103500000D460BF00DF9001B61EB0501052871F16B
:103510000001F6D316B13368B2881A830BF000F9B4
:1035200004460D460BF0FCF8001B61EB0501052875
:1035300071F10001F6D3BAF1000F04D0DAF80030CF
:10354000BAF804201A8398F90000441C3FF442AEF4
:10355000FFF7D0FB3EE60F2388F8023016E5088817
:1035600080B240F4007008800121C8E9022388F885
:103570001C1088F8021009E5099918310991099978
:103580000968F5E40B9918310B910B990968EFE480
:1035900007991831079107990968E9E4D8F81800E4
:1035A000098A441CC8F818400170D8F81410C8F8EB
:1035B00008200139C8F81410C8F80C30E6E408886F
:1035C00080B240F400600880EFF31184102080F393
:1035D0001288088B088820F480600004000CE4B294
:1035E000088084F311880D21A8E5088820F4806004
:1035F0000004000C0880EFF31184102080F312887F
:10360000D8F818000D8A461CC8F81860057008889C
:1036100080B240F40070E4B2088084F31188D8F8D6
:103620001800098A441CC8F818400170D8F8141012
:103630000C200239C8E90223C8F8141088F80200E7
:10364000A4E498F81030002B3FF4BCAD31E600BF85
:1036500038B5184D9DF814E005EB40144FEA401CB6
:1036600094F8F90500B938BD84F80B26C4F80C3677
:1036700001220023490005F5BF6584F80A2684F875
:103680001436049A84F808E6022384F80916C4F86C
:10369000102684F8FA3565440BF042F802460B46D2
:1036A0002846FFF735FC94F8FA35002BF4D194F84E
:1036B000140638BD2833002000680379012B0BD095
:1036C000022B01D0002070478368DB074FF0F00227
:1036D00019D5FF2105F07EBA00B5826890F910C0B7
:1036E000417C85B002F0010201920DF10F020092BF
:1036F0006046FF224FF0F00C8DF80FC0FFF7A8FFD7
:1037000005B05DF804FB7F2105F064BA70B505686B
:103710002B79012B84B004460E4617D0022B02D021
:10372000002004B070BDAB68E122DB074CBF11463E
:103730006121284605F04EFA0028F1D02068324673
:10374000FF2104B0BDE8704006F022BBAA68697C86
:1037500095F9100002F001020DF10F05019200959C
:10376000E1228DF80F20FFF773FFE5E770B50568DC
:103770002B79012B84B004460E4618D0022B02D0C0
:10378000002004B070BDAB68DB074FF0C3024CBF34
:10379000E1216121284605F01DFA0028F0D02068BB
:1037A0003246FF2104B0BDE8704006F0F1BAAA68C5
:1037B00095F91000697C02F0010201920DF10F02EF
:1037C0000092C3228DF80F20E122FFF741FFE4E7CA
:1037D00000680379CA4341EA0211012BCAB209D039
:1037E000022B01D0002070478368DB0717D5D22158
:1037F00005F0F0B900B585B090F910C08DF80F2034
:103800008268417C02F001020DF10F00CDE9000257
:10381000D2226046FFF71CFF05B05DF804FB522181
:1038200005F0D8B970B505682B79012B84B0044632
:103830000E461CD0022B02D0002004B070BDAB6835
:10384000DB074FF0F0024CBFE1216121284605F073
:10385000C1F90028F0D02246FF2152F8040B06F0EF
:1038600097FA0028E8D02379337004B070BDAA68B5
:1038700095F91000697C02F0010201920DF10F022E
:103880000092F0228DF80F20E122FFF7E1FEE0E741
:1038900000680379012B0BD0022B01D00020704768
:1038A0008368DB074FF0B40219D5FF2105F092B908
:1038B00000B5826890F910C0417C85B002F0010229
:1038C00001920DF10F0200926046FF224FF0B40CFE
:1038D0008DF80FC0FFF7BCFE05B05DF804FB7F213B
:1038E00005F078B900680379012B0AD0022B01D0CA
:1038F000002070478368DB070A4617D5A52105F02D
:1039000069B900B5826890F910C085B002F0010273
:103910008DF80F10417C0DF10F00CDE90002A522BA
:103920006046FFF795FE05B05DF804FB252105F024
:1039300051B900BF00680379012B0BD0022B01D0D5
:10394000002070478368DB074FF0960219D5FF21EE
:1039500005F040B900B5826890F910C0417C85B08F
:1039600002F0010201920DF10F0200926046FF2267
:103970004FF0960C8DF80FC0FFF76AFE05B05DF8AA
:1039800004FB7F2105F026B900680379012B0AD0DA
:10399000022B01D0002070478368DB070A4617D549
:1039A000872105F017B900B5826890F910C085B07D
:1039B00002F001028DF80F10417C0DF10F00CDE9EE
:1039C000000287226046FFF743FE05B05DF804FB66
:1039D000072105F0FFB800BF00680379C901012B7A
:1039E000CAB206D0022B01D000207047782105F022
:1039F000F1B800B585B090F910C08DF80F2082683D
:103A0000417C02F001020DF10F00CDE900027822A5
:103A10006046FFF71DFE05B05DF804FB0068037902
:103A2000012B0BD0022B01D0002070478368DB07ED
:103A30004FF0550219D5A52105F0CCB800B5826824
:103A400090F910C0417C85B002F0010201920DF1A5
:103A50000F0200926046A5224FF0550C8DF80FC062
:103A6000FFF7F6FD05B05DF804FB252105F0B2B8BF
:103A700038B5184D9DF814E005EB40144FEA401C92
:103A800094F8F90500B938BD490084F80B26C4F84C
:103A90000C3684F809160023049984F808E60222FB
:103AA00005F5BF6584F80A36C4F8101684F8143694
:103AB00084F8FA2565440AF033FE02460B46284690
:103AC000FFF726FA94F8FA35002BF4D194F814068F
:103AD00038BD00BF28330020F0B5044683B00D4642
:103AE0001746061D20680379012B1AD0022B02D03D
:103AF000002003B0F0BD8368DB0732464FF0FF01C2
:103B00005CBF3246FF2106F0F1F80028F0D015B175
:103B10002379DB07E6D4002FEBD023793B7003B089
:103B2000F0BD8268417C90F9100002F00102CDE9FD
:103B30000062FF22FFF79CFFE7E700BF30B50446B5
:103B4000051D20680379012B83B017D0022B02D00A
:103B5000002003B030BD8368DB072A464FF0FF0129
:103B60005CBF2A46FF2106F0C1F80028F0D0237977
:103B7000DB07EED520680379012BE7D18268417C11
:103B800090F9100002F00102CDE90052FF22FFF788
:103B90006FFFEAE730B50246044652F8040B03799A
:103BA000012B83B00ED0022B01D0002008E0FF21B2
:103BB00006F09CF80028F8D02079C04300F00100FE
:103BC00003B030BD8568417C90F91000009205F08B
:103BD00001050195FF22FFF74BFFEBE730B5B4225B
:103BE00083B00446FF21006805F04AF810B90020B0
:103BF00003B030BD20680379012B04F1040514D013
:103C0000022BF4D18368DB072A464FF0FF015CBF2B
:103C10002A46FF2106F06AF80028E8D02379DB075E
:103C2000E6D520680379012BEAD18268417C90F9BE
:103C3000100002F00102CDE90052FF22FFF718FF49
:103C4000EAE700BF30B50A4683B00446A521006804
:103C500005F016F810B9002003B030BD20680379D4
:103C6000012B04F1040514D0022BF4D18368DB0787
:103C70002A464FF0FF015CBF2A46FF2106F036F8C6
:103C80000028E8D02379DB07E6D520680379012BEB
:103C9000EAD18268417C90F9100002F00102CDE97E
:103CA0000052FF22FFF7E4FEEAE700BF70B582B0E2
:103CB000CDE900230446FFF791FF10B9002002B0C0
:103CC00070BD20685522A52104F0DAFF0028F5D048
:103CD000251D20682A46FF2106F05AF80028EDD05D
:103CE0002379DB07F5D40DF1FF350DF1070615F843
:103CF000011F2046FFF7A6FF0028DFD0B542F6D10E
:103D0000DDE700BF002A35D0F0B5044683B00E468B
:103D10008F18051D16F8012B2068A52104F0B0FFAF
:103D200090B9002003B0F0BD8268417C90F910008A
:103D300002F00102CDE90052FF22FFF799FE0028B0
:103D4000EFD02379DB0710D520680379012BEBD066
:103D5000022BE6D18368DB072A464FF0FF015CBFE8
:103D60002A46FF2105F0C2FFE9E7B742D2D1012080
:103D700003B0F0BD0120704770B5962282B00446B2
:103D80000E460068FF2104F07BFF10B9002002B04E
:103D900070BD251D20680379012B1FD0022BF5D1A2
:103DA0008368DB072A464FF0FF015CBF2A46FF21EC
:103DB00005F09CFF0028E9D02379DB07EAD4E12253
:103DC0002068114604F05CFF0028DFD020683246EE
:103DD000FF2102B0BDE8704005F0DABF8268417C87
:103DE00090F9100002F00102CDE90052FF22FFF726
:103DF0003FFEDFE7002A43D0F0B5044683B00E460D
:103E00008F18051D20689622FF2104F039FF90B914
:103E1000002003B0F0BD8268417C90F9100002F0F0
:103E20000102CDE90052FF22FFF722FE0028EFD069
:103E30002379DB0710D520680379012BEBD0022B07
:103E4000E6D18368DB072A464FF0FF015CBF2A46B4
:103E5000FF2105F04BFFE9E7E1222068114604F05D
:103E60000FFF0028D4D020683246FF2105F090FFD4
:103E70000028CDD00136B742C4D1012003B0F0BD37
:103E80000120704770B505460B460446164655F8A6
:103E9000040B82B087211A4604F0F2FE20680379F1
:103EA000012B1AD0022B02D0002002B070BD836813
:103EB000DB072A464FF0FF015CBF2A46FF2105F0D1
:103EC00015FF0028F0D02379DA07E7D4002EECD0D4
:103ED000C3F34013337002B070BD8268417C90F927
:103EE000100002F00102CDE90052FF22FFF7C0FDF1
:103EF000E7E700BF70B5782182B004461646006837
:103F0000002204F0BDFE10B9002002B070BD251DD6
:103F100020680379012B14D0022BF5D18368DB07CD
:103F20002A464FF0FF015CBF2A46FF2105F0DEFE66
:103F30000028E9D02379DA07EAD45B09337002B0AC
:103F400070BD8268417C90F9100002F00102CDE959
:103F50000052FF22FFF78CFDEAE700BF30B5CC220C
:103F600083B00446A521006804F08AFE10B9002041
:103F700003B030BD20680379012B04F1040514D08F
:103F8000022BF4D18368DB072A464FF0FF015CBFA8
:103F90002A46FF2105F0AAFE0028E8D02379DB0796
:103FA000E6D520680379012BEAD18268417C90F93B
:103FB000100002F00102CDE90052FF22FFF758FD88
:103FC000EAE700BF30B5B42283B00446FF210068A1
:103FD00004F056FE10B9002003B030BD251D206846
:103FE0000379012B22D0022BF5D18368DB072A4607
:103FF0004FF0FF015CBF2A46FF2105F077FE002845
:10400000E9D02379DA07EAD4CC212046FFF71AFE5B
:104010000028E0D002E02379DB07DDD520682A46BE
:10402000FF2105F0B5FE0028F5D1D4E78268417C78
:1040300090F9100002F00102CDE90052FF22FFF7D3
:1040400017FDDCE72DE9F04F8BB0CDE907230446DF
:10405000002004908A460390251D049B079A204661
:10406000DE0002EBC30BFFF7B9FD20B935E0237981
:1040700013F0010207D020682A46FF2105F088FED0
:104080000028F4D129E005929A07099040F1D880E0
:10409000F0212046FFF7D6FDF8B1079BDDF814802C
:1040A000083E3344012606933746BAF1000F54D038
:1040B000082F52D807F1FF394AFA09F909F0010926
:1040C00020684FEAC912782104F0DAFD28B120688F
:1040D0000379012B50D0022B06D00020089B049AB4
:1040E0001A700BB0BDE8F08F8368DB072A464FF0EB
:1040F000FF015CBF2A46FF2105F0F8FD0028ECD047
:10410000237913F00102E2D1C3F3801CD9099B0685
:1041100046D5BCF1000F60D1BAF1000F5AD0082F7C
:1041200058D8894540F08880B9F1000F48D01BF875
:10413000083033430BF808307600013716F0FF06DD
:10414000FFB2B2D108F101085FFA88F8B8F1080FA0
:1041500043D00126BAF1000FAAD1049BC3B1039B3F
:10416000BB4215D9069B13F808301E4214BF4FF00E
:1041700001094FF00009A3E78268417C90F9100023
:1041800002F00102CDE90052FF22FFF771FCB5E712
:10419000039BA3EB0709B9FA89F94FEA59198FE78D
:1041A000BAF1000F13D0082F11D8894596D1B9F173
:1041B000000FBCD1059BBCF1000F08BF3B46059327
:1041C0001BF8083023EA06030BF80830B4E700298F
:1041D000ADD1EFE70029AAD1F2E7402F06D8089B1E
:1041E000049A1B7893423FF638AF77E79BF8077045
:1041F0000BF1FF360BF1060B16F801CF082182EA0E
:104200000C0343F30003013923F0730383EA5202E2
:1042100011F0FF01D2B24FEA5C0CF0D1B345EBD103
:104220009742DCD1049B0133DBB20493059B002B46
:104230003FF454AF0393D2E7DDF8248040464DE7C6
:10424000804640464AE700BF10B500680379012B5D
:1042500084B00C461AD0022B02D0002004B010BD4E
:10426000836813F0010F03AA4FF0030314BF222148
:10427000A22105F009F90028EFD0BDF90D3003EBBC
:1042800083031B12E633238004B010BD8368417C96
:1042900090F9100003F00103019303AB0093222275
:1042A0000323FFF7E5FBE6E7F0B589B00023904A6A
:1042B00002930393136843F48033136003E0029B7B
:1042C000B3F5A04F09D0136803F400330393029BA6
:1042D00001330293039B002BF1D0854B1B6813F431
:1042E000003318BF01230393039B012B01D000BFB0
:1042F000FDE77F4B7F491A6C7F4842F080521A6479
:104300000A6842F440420A609A689A609A6842F4E5
:1043100000429A609A6842F4A0529A6058601A6803
:1043200042F080721A601A689001FCD5734A40F21C
:1043300005711160996821F003019960996841F055
:104340000201A2F580629960936803F00C03082BC8
:10435000FAD1936803F00C03042B00F0C680082BFD
:1043600000F0AB80664A624B66499868664D674EBE
:10437000674FC0F303100144002491F86C10CA4049
:104380006449E9606449586FA960596BC6F8302CDC
:1043900021F080015963596F604A614841F0807192
:1043A0005967196B0A431A635A6B5A639A6B9A637B
:1043B0001A6C5C490A431A64596C5B4A0A435A6492
:1043C00048F2FF7123462246CDE9004475F07AFF9A
:1043D0005648234622464FF6FF71CDE9004475F05A
:1043E00071FF5348234622464FF6FF71CDE9004442
:1043F00075F068FF4F48234622464FF6FF71CDE91E
:10440000004475F05FFF4C48234622464FF6FF718B
:10441000CDE9004475F056FF4848234622464FF642
:10442000FF71CDE9004475F04DFF45482346224613
:104430004FF6FF71CDE9004475F044FF4148234633
:1044400022464FF6FF71CDE9004475F03BFF23464D
:1044500022464FF6FF713C48CDE9004475F032FF2B
:1044600004A8FEF7FBFAD5F8FC200499D6F8303CF6
:10447000364842F08072C5F8FC20354AC2F8B00FC9
:104480005460106840F0010010604FF47A72B3FB82
:10449000F2F3013BB3F1807F2E4AB1FBF2F2C7F891
:1044A0005C2608D24FF0E022F0215361072385F803
:1044B00023109461136109B0F0BD516853685268CC
:1044C0004902C2F388124CBF23490D4903F03F0350
:1044D000B1FBF3F303FB02F2054B5B68C3F301434B
:1044E00001335B00B2FBF3F23DE71B4A3BE700BF41
:1044F000003802400070004008544007003C024071
:104500000024F4007C4C080800ED00E000000020CE
:10451000283300200003FA0500000008FF9167001F
:1045200000000240FFC9FE1033570700000402409C
:1045300000080240000C024000100240001402403B
:1045400000180240001C02400020024055CEACC5BD
:10455000001000E040420F0000127A0082B0064BCB
:10456000002201920193019B03EB80030193019BC5
:10457000196002B0704700BF5028004010B51C20E1
:1045800006F02CFE1121044604F088FA4CB1236891
:10459000A2885A83C8200AF0F1F82368A2881A83F7
:1045A00010BDBDE81040C8200AF0E8B8704700BF51
:1045B000704700BF704700BF10B5104C94F86A36C2
:1045C00023B90F4B4FF480225A6110BD4FF0E02207
:1045D000D2F8103D23F00603C2F8103DFDF75CFF52
:1045E000D4F870369B68DB07EBD5D4F86C271368DA
:1045F00023F0030161F307031360E2E7283300208F
:10460000003C01402DE9F04FA34CD4F86C365A69B8
:10461000D5078BB002D50BB0BDE8F08F5A699B6906
:1046200012EA0301F7D0C1F307430803019300F135
:10463000E180019B5D073FD48807CEB203D5D4F853
:104640006C3602225A610029C0F24A820A05C1F37F
:10465000072500F19981370708D5904B9048D3F88A
:10466000583E9847D4F86C3608225A61F60600F195
:104670000F82E80600F1BE81A80600F11781019BB8
:10468000DA0609D5854B8648D3F8683E9847D4F8B2
:104690006C364FF480125A61019B9B06BBD57F4B51
:1046A0007F48D3F86C3E9847D4F86C364FF400122C
:1046B0005A610BB0BDE8F08FD4F870369E69DB69A3
:1046C0001E40B6B2002EB7D0754D4FF0000B05F16D
:1046D00018080F46F00740F18280D4F87016D8F819
:1046E000002008694B6B23FA0BF3DB01DBB20343B9
:1046F0009068034013F00109D8B200F00F824B6BB1
:10470000012000FA0BF023EA00034B6301239360BE
:10471000624B6348D3F8503E5FFA8BF1984794F8A8
:104720006336012B00F07E8219F0800F57D0D5E957
:104730004CC1D5F82431D8F800E0ACEB010293422B
:10474000DEF8180028BF134680B20333B0EB930F96
:1047500045D9D4F8703694F86396CDE9026BBA4621
:1047600067469C46B94237D2D5F82431781A984228
:1047700028BF184600F1030BD5F828314FEA9B0BF0
:10478000B9F1000F10D182B203329210D8F8B8609C
:104790000AD04946013153F8047B37608A42F9D187
:1047A000D5E94C71D5F82831014403448F42C5F84E
:1047B0002831C5F83411DEF818300AD195F81C01FB
:1047C000012202FA00F0DCF8342022EA0002CCF8E0
:1047D00034209BB29B45C5D3DDE9026B5746760872
:1047E0000BF1010B05F1280508F104087FF472AF05
:1047F000394621E7D4F870369D69DB691D402D0CE0
:104800003FF417AF04F5CC68DFF890B0029104F2E2
:10481000B46600274FF00109C24608E06D0807F1B1
:10482000010706F1040608F1280800F09181EA0763
:10483000F4D53068D4F87016836849690B40D9B252
:10484000DB0740F1708194F86336C0F80890012BC3
:1048500007D10169D8F87C33C1F312015B1AC8F89B
:104860008C33DBF84C3EF9B25046984794F86336E7
:10487000012BD3D1002FD1D194F87137052BCDD195
:10488000D4F8B436074919610749596119684FF0DE
:1048900080211960C2E700BF2833002000000020FB
:1048A0008839002018000860543F0020D4F8705662
:1048B000D4F87826AB68C3F34103022B136814BF06
:1048C0000021032161F30A0313606B6843F48073D2
:1048D00006A86B60FEF7C2F8D4F86C26079ED36872
:1048E00023F47053D360A86810F0060FC0F34101A1
:1048F00000F03C819F49A0483144814240F2AE81A2
:104900009E48A6F57401A1F51051814240F2AA819A
:104910009B499C4831448142C0F0A8819A48A6F145
:104920008C71A1F54341814240F2A4819749984896
:1049300031448142C0F0A281964997483144814276
:10494000C0F0A0819548A6F1B771A1F558518142F8
:10495000C0F0A0819249934831448142C0F09681D1
:10496000914892493044884234BF062005204025B2
:10497000012160F38D23D3604FF4005384F8621655
:10498000A4F8645653617AE600238DF8133094F846
:1049900072378DF81330864B8648D3F8603E9847BF
:1049A000D4F87036D4F86C26986894F86A364FF4C8
:1049B00000615161002B3FF44EAEC3077FF54BAE53
:1049C00094F87537012B7FF446AE9DF81330032B16
:1049D0007FF441AED4F86C3777491A6842F001028F
:1049E0001A601A6842F003021A600B6943F006036A
:1049F0000B6130E6D4F87066D4F86C167368002743
:104A000023F0010373600597059B43F02003059392
:104A1000059B67F38A130593059B0B61674BBC46A7
:104A20000A690592013B02D0059A9206F8D494F8DF
:104A3000612652B1624B03EB820EFF2253F8040F42
:104A40008260D86B73458260F8D10B2363F307074C
:104A500063F3070C4FF0FF33B3614FF00113F361C1
:104A60007761C6F810C03368564823F4FE6333609C
:104A700094F86326D4F8B436012A18616FD04FF445
:104A800080534B614A4B4B48D3F85C3E9847F3E563
:104A9000D4F86C369A6922F010029A611A6AC2F34D
:104AA0004340022802F00F0100F09080062812D146
:104AB00001EB810104EBC101D4F83067D1F8EC09B6
:104AC000C2F30A1210443268C4F82C2C3268C4F8BD
:104AD000302CC1F8EC099A6942F010029A61C8E5DD
:104AE00094F86A363BB1D4F86C27136823F00300BE
:104AF00060F307031360D4F870262D4B2D48D3F8CC
:104B0000645E5368029123F001035360A847D4F810
:104B10006C3602994FF000425A6197E5010707D5BC
:104B2000082393605BE68A0707D50223836075E656
:104B3000C3060FD51023936051E60B077FF56EAEC9
:104B4000DBF8543E5046984733680821996065E683
:104B500002996EE5410679D5402393603FE61A4AF3
:104B60005A611A684FF080221A6088E74FF4007586
:104B70000920FEE6401E1BFF3F420F00DFC8100069
:104B80002013FBFE20D61300FF69180000D3CEFED1
:104B900040771B00C05BB3FEC091210040AC2700F2
:104BA000C01D6AFE40E13300803C36FEE09C4100BF
:104BB000000000208839002000ED00E0410D0300D6
:104BC0009C39002018000860543F002047F6F07020
:104BD000104280D0C2F30A1201EB810004EBC00046
:104BE00002F1030C5FEAAC0CD0F8E069D4F830E7CE
:104BF0004FEA810818BF002006D00130DEF80070AF
:104C000046F8047B8445F8D1414404EBC101D1F856
:104C1000E0091044C1F8E009D1F8EC091044C1F8EA
:104C2000EC0958E7BBF1000F7FF47EAD94F87137C3
:104C3000042B7FF479ADD4F8B436184A1A61184AB7
:104C40005A611A684FF080221A606DE5830758BFD9
:104C500081467FF569AD02239360C0E501214025BF
:104C60000E2086E6012140250D2082E60121402507
:104C70000C207EE6012140250B207AE6012140250B
:104C80000A2076E601214025092072E6012140250F
:104C900007206EE60121402508206AE6180008601A
:104CA000543F002070B5194D194BC5F8543C194BB1
:104CB00085F8601C002683F8276905F65443C0E98F
:104CC00054330D23C0F8583140F201130446C0F8A4
:104CD0005C6100F5A271A0F8443175F03FFA1F2322
:104CE000C4E9EC36E378012205F284559342C4F816
:104CF000A853A4F89C2308BFC4F8AC5304F567710B
:104D00002046BDE8704075F029BA00BF2833002066
:104D10005553425330220020F0B50B7813F0600257
:104D200083B004462BD0202A30D14A78FE2A39D0CD
:104D3000FF2A2DD14A88002A3BD1CA88002A38D1BF
:104D40001F0636D46148624B80F82729C4F8B42383
:104D5000E278012183F8A415A4F89C1303F284538C
:104D60001F21012AC4F8B013C4F8A83304F56771F1
:104D700008BFC4F8AC33204675F0F0F906E04B7874
:104D80000A2B1AD00B2B08D0012B2AD0002002E0CE
:104D900075F076F8022003B0F0BD4D4B4A8883F8D9
:104DA000652CF3E74F8827B9CD88012D01D11B066B
:104DB00042D4204675F064F8ECE7022180F8111126
:104DC0004FF48071A0F81C1142490123C0E94A1137
:104DD000C0E94E33C0E94C3200F58E7175F05CF9D4
:104DE000D4E78B88C0681E06DDB244D40192019AD4
:104DF000394B42F010020192019A0261026901925C
:104E0000013B02D0019AD206F8D4314E2946204601
:104E100075F0A8F8294696F8A455022340222046AA
:104E200075F0D0F8022DB1D18121204675F060F8DF
:104E3000002386F8A435A9E7254ED6F8BC359B6932
:104E40009847C0B286F8640C0028B2D0022306F658
:104E5000644684F811314FF48073C4E94E55C4E9B7
:104E60004A66C4E94C57A4F81C3104F58E712046FB
:104E700075F012F98AE70092009A174B42F020026F
:104E80000092009A65F38A120092009A0261026908
:104E90000092013B02D0009A9106F8D40C4E2946AC
:104EA000204675F05FF8294696F8A4550223402263
:104EB000204675F087F8022DB6D0012D3FF466AF7D
:104EC00001212046FFF7EEFE60E700BF3022002000
:104ED000283300208D3F0020410D030010B50D4BFD
:104EE00093F82739022B07D0033B012B02D800216E
:104EF000FFF7D8FE002010BD074B93F8911504462C
:104F00006DF058FC0028F5DA01212046FFF7CAFEB3
:104F1000F0E700BF3022002028330020F8B53F4CD6
:104F200094F8276905467EB1012E01D00020F8BD16
:104F30003B4B93F891156DF03DFC0028F6DA3146B5
:104F40002846FFF7AFFEF1E7354FB0F8B433D7F896
:104F50008C25C7F85C2C1F2BD7F88825C7F8582C50
:104F600008D1304BD7F884259A4203D197F8911590
:104F7000012919D997F8663C5A1CD2B207EBC30332
:104F8000042A18BF1646052283F8682C4FF40052F5
:104F90002846C3F86C2C022387F8666C87F8A43582
:104FA000FCF720FA0020F8BD97F89235013B0F2B53
:104FB000E0D86DF0FFFB002827DB94F82739013B90
:104FC000022BB3D9B7F8883C1BB3042284F82729F5
:104FD000154AC5F85C61C5E95422D7F88C2587F8D5
:104FE000606C934228BF1346D7F85C2CC5F8583143
:104FF00040F20111A5F84411D21A05F5A271284614
:10500000C7F85C2C75F0AAF890E72846FCF7EAF997
:105010008CE719462846FFF745FE87E73022002037
:105020002833002055534243406E002010B54FEA0C
:10503000511E024400EB8E0C624529D901F01F037A
:105040004FF0FF3450F82E1004FA03F30B4093FA9C
:10505000A3F3B3FA83F3DBB2202B16D10CF10401D6
:105060008A4202D817E08A4212D98C460431DCF811
:10507000003093FAA3F3B3FA83F3DBB2202BF2D020
:10508000ACEB000C03EBCC0010BD03EB4E1010BDDD
:105090004FF0FF3010BD204610BD00BF03694168CE
:1050A00090ED067AF0B4C56A3B4E876853EA010278
:1050B00004BFD6F8381541606A1C30EE077A013318
:1050C000012A80ED067A0361C26241D090ED075A51
:1050D000D0ED096AD6F8384507EE902A70EE455AA9
:1050E000B8EEE76A611AC5EE867AB94277EE857A3C
:1050F00030EE670AC0ED087AE5EE806AC0ED077A07
:10510000C0ED0A6AC0ED096A01D8F0BC7047012AF7
:105110002ADD07EE905AF8EEE77A86EEA76AB5EE3A
:10512000C06AF1EE10FA1FDBF1EEC67AF4EE677A90
:10513000F1EE10FA18D6D0ED056AF4EEE76AF1EE5A
:1051400010FA14D5037BF3B10323F0BC037070474E
:10515000D6F8382580ED080A521ABA424FF00001FD
:1051600080ED070A4162D0D9DFED0C7AE3E707EE64
:10517000903AF8EE677A0223C7EE276AF0BC037014
:10518000C0ED066A7047D6F8381541600022036109
:105190008261C362B9E700BF28330020000000002D
:1051A000DFED504A10B5844600F1480E0346B1ECDD
:1051B000017AD3ED067ADA6A77EE877A0132012A2C
:1051C000C3ED067ADA6255D093ED075A93ED096A7A
:1051D00007EE902A77EE455AF8EEE77AC5EEA76A11
:1051E00076EE857AF0EE466A37EE677AC3ED087A96
:1051F000E5EE876AC3ED0A6AC3ED077AC3ED096A73
:1052000018337345D3D1384C4168D4F83825036935
:10521000521A816801338A4203612AD990ED056AE6
:1052200000F1300EDCF82C20DCED0A6A012A02F1D4
:10523000FF3126DD07EE901AF8EEE77A86EEA77AC0
:10524000B5EEC07AF1EE10FA1BDBF1EEC77AF4EEA0
:10525000677AF1EE10FA14D6E645B4EEE76A0CF17F
:10526000180C16D0F1EE10FADCD5037B6BB30323D8
:10527000037010BDF0EE477AF0EE646A83ED087AB1
:10528000BAE7DFED187AE645B4EEE76A0CF1180CE0
:10529000E8D1F1EE10FAE8D407EE903AD0ED066AC4
:1052A00090ED0C7AD0ED125AF8EE677A022386EE72
:1052B000A76A0370C7EE276A85EEA77A80ED066AB3
:1052C000C0ED0C6A80ED127A10BD0022D4F83815BA
:1052D000416003618261C362026343648264C365A7
:1052E00010BD00BF0000000028330020B0EEC06AEF
:1052F000F0EEE05AF4EEC65AF1EE10FAF0EE407A13
:105300000EDCB5EE400AF1EE10FA4BD0F4EEC65AC0
:10531000F1EE10FAF0EE466A50D5B0EE655A03E0B1
:10532000F0EE656AB0EE465A85EE267A9FED252AA4
:105330009FED253A9FED254ADFED254ADFED252A31
:10534000DFED253ADFED256AA7EE023AE7EE223AD5
:10535000A7EE034AB7EE005AE7EE044AA7EE235A37
:10536000E7EE246AF4EEC65AB1EE667A87EE050AD5
:10537000F1EE10FA48BF9FED1A7AF5EEC00A48BF69
:1053800037EE400AF1EE10FA48BF9FED167AF5EEBF
:10539000C07A48BF37EE400AF1EE10FA48BFB1EECE
:1053A000400A7047DFED107A9FED100AF5EEC00A53
:1053B000F1EE10FA58BFB0EE670A7047B0EE465AE9
:1053C000B2E700BF39094E3DE3B59EBE88FA16BE6E
:1053D00045FE7FBF99FB243F69A2163EA7DFA8B414
:1053E000DB0FC93FDB0F4940A7DFA834DA0F494084
:1053F00091ED007AD0ED047A90ED054AD0ED064AA1
:1054000090ED075AD0ED085A90ED096AD0ED0A6A7E
:10541000E7EE077AF7EE003AC0ED047A91ED007AF4
:10542000D1ED017AA7EE274A90ED0B7A80ED054A7F
:1054300091ED024A91ED003AD0ED0C7AE3EE044A88
:10544000C0ED064AD1ED004A35EE245A80ED075AE8
:10545000D1ED014A91ED005AE4EE855AC0ED085AAB
:10546000D1ED015AA5EEA56A80ED096AD1ED015A88
:1054700091ED026AE5EE866AC0ED0A6AD1ED016A35
:1054800037EE267A80ED0B7AD1ED026A91ED007A43
:10549000E6EE877AC0ED0C7A91ED026AD1ED016AF1
:1054A000D0ED0D7A90ED0E7A90ED0F4AD0ED104AC6
:1054B00090ED115AD0ED135AE6EE267A75EEA35A06
:1054C000C0ED0D7AD1ED026AD0ED127A90ED006A4E
:1054D000A6EEA67AD0ED016A80ED0E7A91ED027A01
:1054E00034EE074A90ED027A80ED0F4A91ED004AC2
:1054F00074EE844AC0ED104AD1ED014A35EE245ACB
:1055000080ED115A91ED025AC0ED135A77EE857A6B
:10551000C0ED127AD1ED017AD1ED005A91ED025A27
:1055200067EEA77AE5EEA57AE5EE057AA5EEA76A1D
:1055300080ED006A91ED016AE6EE276AC0ED016A2E
:10554000D1ED026AA6EEA77A80ED027A90ED037A99
:1055500077EE277AC0ED037A704700BF2DE9F04F50
:105560004FF0000989B0864600F110050646034653
:1055700000F13008074648462C46CDF80CE08B4633
:105580009C46B24600283CD10CF1040CA445FBD14A
:10559000032800F1010151D09C46AA46029398B11C
:1055A000DCED047A0192AAEB0903B6467246F3ECED
:1055B000016A92ED007AE6EEC77A53450EF1100EBD
:1055C000CCED047AF2D1019ADCED046A15ED047A8F
:1055D000C6EE877A0CF1100CC4450AF1100ACCED26
:1055E000007ADCD1029B04361433084608F1040823
:1055F00014351034103709F104099C46B2460028CE
:10560000C2D0DCED007A0192D64639467246F1EC02
:10561000016A92ED007AE6EEC77A99420EF1100E19
:10562000CCED007AF2D10CF1040CA445019A0AF1F8
:10563000040AE6D1032800F10101ADD1DDF80CE048
:1056400000235946049305930693079376467746BD
:1056500004AD0020F2EC017AE5EC017AB0B104ACC3
:105660003B46B4EC017AF3EC016AE6EEC77AB3424A
:1056700045ED017AF5D1013004280BD0F2EC017A26
:1056800010371436E5EC017A0028E8D110371436CB
:105690000120DFE708AD75ED017A10310EF1400E03
:1056A00004287446A1F1040241ED017A1ED073462C
:1056B000F3EC016AB1EC017AE6EEC77AA342C2EDDF
:1056C000007AF5D15EED016A87EEA67A013882EDA7
:1056D000007A17D0AEF1140E103C114675ED017A28
:1056E0000428A1F1040241ED017AE0D15EED016AE6
:1056F00087EEA67A103CAEF1140E032001ED017A7C
:105700001146EBE709B0BDE8F08F00BFDFED297A65
:10571000B4EEE70AF1EE10FA28DD9FED277A30EEBD
:10572000470AB4EEE70AF1EE10FAF8DCDFED237A6F
:10573000B4EEE70AF1EE10FA2FDD30EE670A37EE2D
:10574000C00A60EE007A9FED1E7A9FED1E6ADFEDC3
:105750001E6AA7EE876A9FED1D7AE7EE866A60EE05
:10576000275AA7EEA67AA5EE870A7047DFED187ACA
:10577000B4EEE70AF1EE10FAD8D59FED0F7A30EECD
:10578000070AB4EEE70AF1EE10FAF8D4DFED0B7A6F
:10579000B4EEE70AF1EE10FACFDC9FED0E7AB4EE2C
:1057A000C70AF1EE10FA44BF30EE270A37EE400A7E
:1057B000C7E700BFDB0F4940DB0FC940DB0FC93F24
:1057C0009A7C2E36FAAF4FB93587083CA4AA2ABE78
:1057D000DB0F49C0DB0FC9BF10B5404CB4FBF2F47E
:1057E000A14219D3DFED3E7AF7EE005AB0EE677AA8
:1057F000B0EE676AF0EE676A0023C0ED005AC0EDB4
:10580000017A80ED027A80ED036AC0ED046A83615B
:1058100043610362C36110BD07EE902AB8EE677A58
:10582000DFED307A27EE277AB7EE006AC6EE076A18
:1058300007EE901A9FED2C7AF8EE677AB0EE405A98
:1058400067EE877AC7EEA64AFDEEE47A17EE902A55
:105850002032402A3FD8B0EE640AFFF757FFB0EE7F
:10586000404ADFED227A34EEA70AFDEEC07A17EE49
:10587000902A2032402A29D8FFF748FFF8EE006A24
:1058800060EE266A012B1CD0B7EE006A36EE406A45
:10589000F6EE004A66EE244A35EE055AF7EE007A37
:1058A00084EE057A77EE275A37EEC75A84EEA57A4A
:1058B000C6EE257A86EEA56AC5EE256AF0EE475A51
:1058C0009AE7B0EE666AF7EE004AE5E7DFED086AB0
:1058D0009FED030AD6E79FED024AC2E720A1070029
:1058E00000000000BD378635DB0FC940DB0FC93F24
:1058F00000000080DFED077A30EE270AFDEEC07A67
:1059000017EE903A2033402B00D8FFE69FED020AB5
:10591000704700BFDB0FC93F000000002DE9F84FC2
:10592000DDF82CB09DF828408946002C1BF8011B9F
:105930000CBF4FF020084FF030081C1E05461746DC
:1059400008463ADB00295CD0002C55D04FF0000A05
:105950005B4600E064B313F8016B013C002EF9D103
:10596000BAF1000F2FD1264644B14D454146284695
:1059700000D2B847013CF8D10B9B18780146A0B182
:105980004FF0FF344FF0000A00E09B464D4528469B
:1059900000D2B8475B4613F8011B0029F5D10B9BD9
:1059A000F61A5E44BAF1000F10D13046BDE8F88F08
:1059B000BAF1000F1BD15646E0E7634229B31C46FB
:1059C0004FF0010AC4E70028E0D10646002C04F19C
:1059D000FF3AEADD54464D454146284600D2B847D5
:1059E000013CF8D2013656443046BDE8F88F0646F1
:1059F0000028DAD02646C9E72646A2464FF0FF34F3
:105A0000C4E72646002CB0D1CFE76FEA040A0E4661
:105A1000E0E700BF0FB430B583B006AB0C4853F8D5
:105A2000042BD0F8241ED0F8200E01936FF068FCF0
:105A3000084C0546D4F8200E03685B699847002897
:105A4000F8D0284603B0BDE8304004B0704700BF2E
:105A500028330020302200200EB410B583B005ABEF
:105A6000044653F8042B0749009301A801946FF0F2
:105A700047FC019B00221A7003B0BDE8104003B040
:105A8000704700BF1D0C00080CB470B5334CD4F83F
:105A9000283EA4B0002B5BD094F8303E99420AD93E
:105AA000D4F8342E01238340134204D124B0BDE83E
:105AB000704002B07047D4F83835294AA2FB03027F
:105AC00092094FF47A7101FB123304A82549FFF7BC
:105AD000C3FF04AA29AB0244CDE902322249289A25
:105AE000064603A86FF00CFC039B0A22591C039185
:105AF0001A70039B0022591C03911A70D4F8285E77
:105B0000ADB12B685B6A1BB128469847D4F8285E74
:105B10009DF810100029C9D00DF111042B682846FA
:105B20001B68984714F8011B0029F7D1BEE7D4F889
:105B30002C3E002BBAD030440222009204A98218D5
:105B4000FD2039F0BBFA24B0BDE8704002B07047C8
:105B5000D4F82C3E002B9FD1A8E700BF28330020AB
:105B6000D34D6210640B0908ED090008194A10B5FD
:105B7000D2F8384E033004EB9003B3F5007F19D808
:105B8000C2F8383E02F63C6202EB8404124A02EB91
:105B9000810120F00300D1F84425C3F500731044BF
:105BA000C1F844050D4A9B0004210020FFF76CFF5B
:105BB000204610BD00210846094AFFF765FF094A43
:105BC000D2F8A830002443F00073C2F8A830204671
:105BD00010BD00BF2833002020440020700B0908AE
:105BE000940B0908000000102DE9F0410268214DD6
:105BF0000746002455F834309A4209D001340E2C5F
:105C0000F8D11D4A00210520FFF73EFF002013E0D8
:105C10001A4B03EB8408D8F8C0657EB1797901EBA3
:105C2000410306EBC30300221820C3E9032200FB53
:105C300001609F601A750430BDE8F081072164207F
:105C4000FFF794FF0146C8F8C00568B131466422E9
:105C50007BF05EFAD8F8C06505EBC405C6E90056CE
:105C6000F6617663F664D9E7054A0520FFF70CFF75
:105C7000CCE700BF084D0808A40B09082833002012
:105C8000CC0B090870B50668F46982B00546002C93
:105C90003FD03379012B04F103022DD0022B26D102
:105CA000B36813F0010F30464FF00D0314BF0C2101
:105CB0008C2103F0E9FBA070D8B1B4F90A3007EEEB
:105CC000903AF8EEE77AC5ED077AB4F90C3007EEB2
:105CD000903AF8EEE77AC5ED087AB4F90E3007EE9F
:105CE000903AF8EEE77AC5ED097A02B070BD00236C
:105CF000A370002002B070BDB368717C96F91000EB
:105D0000009203F0010301930C220D23FDF7B0FE76
:105D1000D1E709211420FFF729FFF06104462E681E
:105D2000B7E700BF38B50568EB690446E3B198787A
:105D300000B938BDB3F9042007EE902AF8EEE77AEF
:105D40000120C4ED047AB3F9062007EE902AF8EE9C
:105D5000E77AC4ED057AB3F9083007EE903AF8EE29
:105D6000E77AC4ED067A38BD09211420FFF7FEFE5C
:105D70000346E861DBE700BF03685A1C026018783D
:105D8000704700BF03681A46591C016012F8021BD5
:105D90000260587841EA0020704700BF10B40268E2
:105DA0001346511C016013F8021B0360D31C547886
:105DB000036093781B0443EA0423141D0460D07825
:105DC0005DF8044B0B4343EA0060704712B370B5B3
:105DD0000446864604E0981B17D114EB0C0C15D032
:105DE0001EF8013BA3F14100192811F8010BA0F1A5
:105DF000410598BF2033192DA2EB0E0C00F12006AF
:105E0000E9D91B1A04D10028E7D170BD604670BDE6
:105E1000184670BD1046704710B402888378184C3D
:105E200002F0030101EB4101013B03EB810304EBB1
:105E30004303C178B3F8FC30A2F5FA62920840F24D
:105E4000B55404FB02334A1E134401794279847924
:105E5000008903EB430301EBC301C1EB0111094BC3
:105E600002EB8102C2EB0212234403EB8203002106
:105E70004FF47A72C3FB02015DF8044B704700BF18
:105E80007C4C080880436D38F8B516461F4604461A
:105E9000394630464FF47A7200237EF029F93C4DA2
:105EA0003C4B054483FB05602844E917C1EB6011B6
:105EB00083FB01030B44384EC817C0EB631086FB0D
:105EC000003CC317354EC3EBAC0386FB03764FEAA9
:105ED000E37ECEEBE61EC1EB0116A5EB860CC0EB14
:105EE0000015A1EB8501617103EB4301A0EBC1003B
:105EF00040F2B55101FB1E33B3F5896F84F806C03B
:105F000020714FEA8E0637DA40F2DA218B4239DC13
:105F1000B3F5B77FB4BF4FF0000E4FF0010E20492C
:105F20000EEB4E0001EBC0017546B1F812014FEACD
:105F30004E071C4907EB0E0C01EBCC0C0CF1160CB8
:105F40000B2101E03CF8020D984212DD0139F9D134
:105F50001349774401EBC701B1F8FC00012101337B
:105F600006F5FA6E1B1A7544A170E3702281258034
:105F7000F8BD0131C9B2F2E7032540F29650AE46B2
:105F80000627D6E7022540F22940AE460427D0E78F
:105F900080BC92C789888888ABAAAA2A73B06D167C
:105FA0007C4C0808784D080830B52F4C86460D46C5
:105FB0000FCC8DB0EC46ACE80F000FCCACE80F0076
:105FC00094E80F001EF0030F8CE80F000FD1274B51
:105FD000274A03FB0EF3B2EBB30F43D3254AB2EBD0
:105FE000331F34BF01220022C2F11D0200E01C2237
:105FF0000EF1FF33002B019240F26D12194602FBA5
:106000000EF2B8BF0EF1020102EBA1021A491B4CBD
:1060100081FB0301DB17A3EB61100244C3EBE11327
:106020001A44253284FB02311144D317C3EBA10378
:10603000C3EBC303D31AADF10402EE4602EB8501B4
:106040005EF8040FC21884FB023C9444D317C3EBE0
:10605000AC03C3EBC3037145A2EB0303F0D1C01A39
:106060000DB030BD1D22C3E7D84D0808295C8FC292
:10607000285C8F020AD7A3001F85EB519324499215
:106080000E4B10B5D3F8D045D3F8D43554EA0302FB
:1060900009D1014640F201130020C1F80230887195
:1060A0000880088110BD064AD2F83825121943F13C
:1060B0000003FFF7E9FE012010BD00BF20440020CF
:1060C0002833002088422DE9F0414FF001043DD3F0
:1060D00001FB04F4B0FBF4FC8C45F9D23CB3002680
:1060E00016E0BCF1090F274698462C4623DD002A0E
:1060F0000CBF4FF0570E4FF0370EF444B94288F8FA
:1061000000C003F1010306F1010610D8B0FBF5FC55
:10611000B4FBF1F504FB1C00002EE2D1BCF1000F32
:10612000DFDCA1420AD90CF1300C03F801CB0022CC
:106130001A70BDE8F0814FF0300EDEE7B0FBF5FCE1
:106140002C4605FB1C00B5FBF1F5E7E78446C6E7E6
:106150002DE9F041044694421546084609D2B4FBA5
:10616000F2F6154B05FB16441B5D00F8013BBDE83C
:10617000F081B4FBF2F69642B6FBF2F70CD20E4B6E
:1061800005FB176705FB1644DA5D00F8012B1B5D64
:1061900000F8013BBDE8F081BA42B7FBF2F807D93D
:1061A000054B05FB187813F8082000F8012BE7E7EA
:1061B0004046FFF7CDFFF3E7E80B0908B5EEC00A4C
:1061C000DFED347AF1EE10FACCBF30EE270A30EE74
:1061D000670ADFED317A20EE270A30B5FDEEC07A8E
:1061E00087B017EE904A054684EAE470002303A9BD
:1061F000A0EBE470CDE9003302936DF07DF8002C44
:10620000B4BF2D23202303A88DF800307DF038F88B
:10621000012829D0022833D003281DD003A96846BD
:106220007CF06EFF68467DF02BF8C41EE4B2224677
:106230006946284679F054FB00232B5528467DF00B
:106240001FF82E232B5401300DEB040128447CF061
:1062500077FF284607B030BD302303A968468DF884
:1062600001307CF04DFFDDE743F23002302303A91B
:106270006846ADF801208DF803307CF041FFD1E78E
:1062800043F2300303A96846ADF801307CF038FFD3
:10629000C8E700BF6F12033A00007A440278202A50
:1062A000034600F10100F9D0092AF7D02D2A29D0A0
:1062B0002B2A03BF5A78B7EE000A0346B7EE000A4E
:1062C000A2F13001C8B20928DFED4C7A10D8F2EE05
:1062D000046A07EE101AB8EEC77A13F8012FA7EE7A
:1062E000A67AA2F13001C8B20928F0EE477AF0D9B7
:1062F0002E2A49D0197801F0DF01452907D020EE78
:10630000270A70475A78BFEE000A0346D8E710B450
:1063100059782D2962D02B2954D0A1F13002092AB5
:1063200003F1010355D80024002202EB820201EBA5
:10633000420213F8011FA1F130000928A2F1300236
:10634000F3D9B2F59A7F134628BF4FF49A73072A00
:1063500050D9DFED2B6A1A46B7EE007A083A072AC1
:1063600027EE267AFAD803F007032BB1F2EE046A7F
:10637000013B27EE267AFBD16CB3C7EE877A5DF836
:10638000044B20EE270A70475978A1F13002D0B2B1
:10639000092803F10103AED8F2EE046AF0EE665A62
:1063A00007EE102AB8EEC77A13F8011F87EE266AA7
:1063B000A1F13002D0B2092866EEA56A77EE867A9E
:1063C000EED998E79978A1F13002092A03F1020386
:1063D000A9D9B7EE007A67EE877AD0E79978A1F16C
:1063E0003002092A03F1020388BFB7EE007AC4D84D
:1063F000012499E7B7EE007AB7E700BF000000007C
:1064000020BCBE4C0378202B024600F10100F9D0DD
:10641000092BF7D02D2B08BF5378A3F13001CBB255
:1064200006BF02464FF0FF3C4FF0010C092B4FF026
:10643000000000D9704712F8013F00EB800001EB2B
:106440004000A3F13001CBB2092BF4D90CFB00F0D2
:10645000704700BF2DE9F04F91B045F027FC45F0A3
:10646000E9FBB0F1000A40F33C810024DFF80C9313
:10647000B54D27462646A04604E006F50066B2451F
:1064800040F3958020220DEB0201304645F05CFB85
:10649000AE49122208A879F05DFD83460028ECD1B0
:1064A000BE4222D0AA4BAB4908EB480203EB820361
:1064B00008F10108424601931846F31B0293FFF7C7
:1064C000CBFA4A46019B42F84C3B029BC9F80C7040
:1064D000C9E90433D9F81C30C9E908339E4BC9F81F
:1064E00028300123C9F8083091469C4BD3F8F03589
:1064F000C9F81C303746122202F140030DEB0301AC
:106500002B5D11F8201C994202F101020BD00024EE
:10651000202AF1D12037BA4508A938463EDB45F09C
:1065200013FB0022E8E70134152CF1D1D019202209
:106530000DEB020145F008FB894907AA08A879F08C
:1065400057F958B30023CDE90133CDF814B00393C4
:1065500004931F469B467B1E042B00F2BA81DFE8A2
:1065600003F082728A860300CDF814B0FFF74AFF69
:10657000059B8346049989B1DDE9012042EA401276
:1065800003985B0143EAC023A1F2BC7143EA6B03A9
:1065900042EA412243EA0243C9F81C30B8F1640FD1
:1065A0006DD0374606F50066B2453FF76BAFB8F1E0
:1065B000640FC34663D0BE421BD0654C65490C23B3
:1065C00003FB084408F1010B5A462046FFF744FA42
:1065D000614BC9F82830F61BD9F81C30C9F80040C7
:1065E000C9E90376C9E908330123C9F81460C9F879
:1065F0000830BBF1000F0BF1040143DC594C574A42
:106600004FEA4A03B3F1805FD2F8F0556EDB56498A
:1066100054484FF4987279F063F9544BA3F11C027B
:1066200003F598719D60C3E900554C338B42F9D155
:10663000A06828B923791BB12368002B40F0A28001
:1066400011B0BDE8F08FFFF7DDFE01904449002056
:1066500007AA013779F0CCF800287FF47CAF5B46BD
:10666000DDF814B086E7FFF7CDFE0290EEE7FFF706
:10667000C9FE8346EAE7FFF7C5FE0390E6E74FF061
:10668000640B6821374C354AD4F84C61C2F8F06588
:106690004C2707FB01F563193A46002118467AF0AA
:1066A00037FD3A4600217AF033FD314A625105F157
:1066B0001002DFF8CC80284FC0F820804FF001098D
:1066C000C0F80890876244F802A022441835C2F846
:1066D00004A0221D0BF10501565115446E6046625F
:1066E0008DE71E4B1F4CD3F8F05504214FF04C089A
:1066F00008FB01F6A7194246002138467AF008FD4A
:106700004246002138467AF003FD1A4BA3514FF060
:10671000010906F11002DFF86880C7F80890CAF195
:10672000006303FA09F34FF0020BC7E9078887F803
:1067300005B01148A35006F118012244536045509A
:1067400001444D607D6262E7340C0908100C0908B1
:10675000F8490020240C090889240008F8100020BA
:106760004C0C0908C84E0020084E0808E44E0020D2
:10677000540C0908640C0908CC4E0020F84F002086
:106780000068994F002600275449A064C4E91067A7
:10679000E063064607469646CD6C01F14C036DB3A7
:1067A0009D689F6406F1FF3C6545C1E92377DF637F
:1067B0000ED006F1010C65451DD113F8486C002E72
:1067C0003FF43EAF196443F8083C2E461946E3E710
:1067D000002E3FF435AF53F80C1C2E46002E3FF42C
:1067E0002FAF0D6CEA6B02F1010CC5F83CC01D64C3
:1067F0008B641946D0E7B542F0D021E772460227F4
:106800002E46A64615E0D36B17635B0118BF03F64F
:10681000FF73C2E9046614BF01EB13333B465363B5
:106820001946916352F84C4FCB1A1D444F1C01304E
:10683000CCB11379791E002BE5D1136917635BB1D5
:1068400003F6FF73546901EB133353634CB104F641
:10685000FF7C01EB1C31E4E754693B465363002C99
:10686000F5D13946DDE71E4A1E4BC2F81C0E013930
:1068700002F55F60C2F8F43D3E2640233F27C2F890
:10688000105EC2F8003EC0E902677446C2F80C1EF2
:106890008D0F8B00D9B140F2FF169B1945F1000511
:1068A0005B0A43EAC553C0E9094403F140042344A9
:1068B00003EBC101C2F8083EC2F8F01DCB0D49023E
:1068C00040F8043CC2F8044E40F8081CB8E6012326
:1068D000E9E7FFF797FD0490B8E600BFC84E002037
:1068E00030220020740C090870B5344D2B787E2BB3
:1068F00001D0002070BD08224FF4FC4341F221007A
:1069000019B200294FEA4303B6BF80EA41019BB2A6
:106910008BB2013AF4D1B5F8011069B32848294C7B
:10692000A042E6D206384618A642E2D241F2210C35
:106930000529DED9864214D0013806F1FF3E10F851
:10694000012F082183EA02231AB2002A4FEA4303E7
:10695000B6BF8CEA42029BB293B20139F4D17045C2
:10696000EDD1318849B1B21DA242C2D27218A24201
:106970003046BED21646DBE7134E741E41F22100AC
:10698000A44614F8012F082183EA02231AB2002A30
:106990004FEA4303B6BF80EA42029BB293B2013989
:1069A000F4D16645ECD17288D01A084A331D5B1BBE
:1069B000B0FA80F04009A2F8883A70BD00000E08D5
:1069C00007000E080000100801000E0820440020F7
:1069D0002DE9F04F914B924A8BB00020D21ACDE9AD
:1069E0000600CDE90800D11805928E4A0393049160
:1069F00010690028C0F281818A4AF320D06000200B
:106A000008908948012288428DF8242000F2718183
:106A10007E2007928DF818004FF4FC42082041F2C6
:106A2000210514B2002C4FEA4202B6BF85EA4404A5
:106A300092B2A2B20138F4D17C48ADF802207C4A6F
:106A400090427CD2804641F22105B8F80200B8F8A5
:106A50000020C0F30B07C2F30B04120BBE1D4FF056
:106A600000098DF808200204ADF80460ADF8064076
:106A70008DF8099000F1C38006338B4200F2398112
:106A800001AE0DF10A0B344601E0A34513D0079B7C
:106A900014F8011B03F128026A440133042B079305
:106AA00002F8101CF1D106A903A8FAF7D9F8A345FA
:106AB000CDE90790EBD1089B002BC0F21A81BDF8FD
:106AC000024016F8013B082284EA032423B2002B7B
:106AD0004FEA4404B6BF85EA4303A4B29CB2013A2C
:106AE000F4D1B345EDD1D8F804603A46314603A855
:106AF000FAF776F90028C0F2FC80F019864213D02C
:106B0000711E013811F8013F082284EA032423B2E0
:106B1000002B4FEA4404B6BF85EA4303A4B29CB2FB
:106B2000013AF4D18142EDD1DDE90302ADF8024032
:106B300011463F4A08F114089045034685D30233B5
:106B40004FF000089942ADF80480C0F0D28001AD4A
:106B50002E460DF106042F4601E0BC4213D0079BE0
:106B600017F8011B03F128026A440133042B02F8D1
:106B7000101C0793F1D106A903A8FAF771F8BC42DB
:106B8000CDE90780EBD1089B002BC0F2B280BDF8A5
:106B9000023041F2210016F8012B83EA0223082279
:106BA00019B200294FEA4303B6BF80EA41019BB204
:106BB0008BB2013AF4D1B442EDD10399ADF8023071
:106BC000049B0231994200F294800DF102061446B2
:106BD00002E0B54200F08A80079B16F8011B03F122
:106BE00028026A440133042B02F8101C0793F0D1E9
:106BF00006A903A8FAF734F8CDE90740E9E7CB4640
:106C00000BF1010B06335FFA8BFB99428DF809B04B
:106C10006FD301AE0DF10A0A34460DE000000E08F4
:106C200000001008003C024001000E08EC81090839
:106C300050870908A24515D0079914F801CB01F136
:106C400028030DEB030001310429079100F810CC53
:106C5000F0D106A903A8FAF703F80023A24508908B
:106C60000793E9D1089A002A43DBBDF8024016F8E1
:106C7000012B082184EA022422B2002A4FEA4404AC
:106C8000B6BF85EA4202A4B294B20139F4D1B2454A
:106C9000EDD1D8F8041001EB09063A46314603A8B5
:106CA000FAF79EF8002824DBF019864213D0711EF3
:106CB000013811F8013F082284EA032423B2002B93
:106CC0004FEA4404B6BF85EA4303A4B29CB2013A3A
:106CD000F4D18142EDD1DDE90302BBF1030FADF840
:106CE000024003461146B9448AD121E7089B002B94
:106CF00009DA00200BB0BDE8F08F1548506000F1B4
:106D00008830506078E6079840B912490A6942F025
:106D100000420A61B3FA83F04009EBE7DDE9033290
:106D200003449342E5D806ABC0F1040200211844A5
:106D30007AF0EEF906A903A8F9F792FF00280346B6
:106D40000890D6DB9DF82420002AE3D0DDE700BFC1
:106D500023016745003C024008B5FFF739FE40B902
:106D6000FFF736FE28B9FFF733FE10B9052007F00C
:106D700033FDFFF7B9FD0028F8D008BD70B5458890
:106D80000B460446C5F30B052A46002118467AF047
:106D9000BFF90A4A21699142034606D3084A914243
:106DA00006D3BDE87040184608470029F9D170BDE8
:106DB0002A46BDE8704078F093BD00BF50870908AF
:106DC000778C09082DE9F04103EB4306964602EB68
:106DD000460612F9067B86B00346754692F8008097
:106DE000A3EB0804A3EB070C002CB8BF6442BCF172
:106DF000000FB8BFCCF1000C6445B8BF154602F1D6
:106E00000602B8BF4FFA88F7B242E7D16A889EF807
:106E10000000B842144614D1BEF80200A1EB0008ED
:106E2000A1EB020CB8F1000FB8BFC8F10008BCF12B
:106E3000000FB8BFCCF1000CE045BEBF754602465E
:106E400004460EF1060E7645E1D16A7904922A795C
:106E5000CDE902422878054ACDE90010032101203E
:106E6000FEF712FE284606B0BDE8F0817C0C09084A
:106E70004FF40063838170474FF400638381704750
:106E8000074B10B403F11001002453F8042B824285
:106E900008BF43F8044C8B42F7D15DF8044B7047B0
:106EA000407E002001207047012070472DE9F04FFF
:106EB000734D2869AB8AB5F920E0B5F91CC0B5F867
:106EC0001A80B5F9226085B0C3EB2014009204FB50
:106ED00004F4B5F91820CDF80CE0241302FB04F4F7
:106EE0005B00B5F916200296C3EBE00302FB03F347
:106EF000A41304EBE3242B6B0193A4F5FA30B5F94A
:106F00001E30EC6280FB00EA4FEAE37B03FB0AF9E8
:106F10008CFB00C20EFB0B99A3FB0E3BCB44120370
:106F20001B0A42EA1C5243EA0B634FEA0C3C13EB88
:106F30000C0342EB2B22A3FB083C02F5004208FBAA
:106F400002CC4FEAEC734FEA6C0953EA6C0C0F4623
:106F5000B5F9241000F09180029E019A86FB00088A
:106F6000C2F5801C01FB0AFA4A464FEA48484FEA3C
:106F7000E17948EAD0380EFB09A94004A1FB0E1EB6
:106F80004118F14449EB080900200CF00048039E29
:106F9000411848EA5C084FEACC7CBCEB010C09EBD9
:106FA000C60968EB09081CEB0C0E48EB08011EEB48
:106FB0000C0E48EB010188014FEA8E1940EA9E60F1
:106FC0001EEB090E41EB0001890041EA9E714FEA78
:106FD0008E0E1EEB0C0E48EB01014FEA8E0089006D
:106FE00010EB0C0041EA9E7148EB01017DF080F846
:106FF000B5F92A304FEA61384FEA503E4EEAC14EA9
:10700000DA1703FB08F984460EFB0299B5F928004C
:10701000B5F92620A3FB0E35A94403FB08F50EFBAA
:107020000955A3FB0E3E75445B0E43EAC51313EBF3
:107030000C0341EB65654FEAE07E00FB01F10EFBBE
:107040000C11A0FB0C0C6144C00C40EA41301B1831
:1070500045EBE1451B0A43EA056303EB02130FB15D
:107060001B0A3B60009B23B104EB84048034241290
:107070001C60012005B0BDE8F08F0023EFE700BFE2
:10708000407E002031B10A4BD3ED147AFDEEE77A51
:10709000C1ED007A52B1064B9FED067AD3ED157A19
:1070A00067EE877AFDEEE77AC2ED007A012070473D
:1070B000407E00200000C8420120704710B40E4BF3
:1070C0000E4C1B68A06D1B1AFA2B09D809B1236E50
:1070D0000B600AB1636E136001205DF8044B7047CA
:1070E000074A1368002023F0040384F85C0013604F
:1070F0005DF8044B704700BF60380020407E0020E0
:10710000AC00001001207047044B002200219A6659
:10711000DA661A6759670120704700BF407E002079
:107120000F4B104A1B68516F5B1AFA2B16D8D2ED21
:107130001A6A92ED1B7AD2ED1C7AFDEEE66ABDEE7C
:10714000C77A16EE903AFDEEE77AC38617EE103A4C
:10715000038717EE903A438701207047002070475D
:1071600060380020407E002000487047EC16002068
:1071700000487047B87E002030B50F4A83B092F8BF
:1071800088500191B5B9D2F88C509DB12B681A681E
:1071900082B19B6873B104462846984750B12B686A
:1071A000019922461C6828460B46214603B0BDE8DB
:1071B0003040084703B030BD407E00200B4B70B517
:1071C000D3F890608EB133681A6872B19B6863B16E
:1071D000054630460C46984738B133682A46196848
:1071E00030462346BDE87040084770BD407E002011
:1071F000437913F0010306D0D0E90731C268581A69
:10720000531E184070471846704700BF437913F06B
:10721000020307D0D0E909130269581E401A531E11
:1072200018407047184670474379024613F0010032
:1072300014D0106AD168D36901F1FF3C1B1A13EA1C
:107240000C030AD053691B5C00F1010CD8B2BCFBE3
:10725000F1F301FB13C3136270471846704700BF78
:1072600043799B070AD5436A8269D154436A02690C
:107270000133B3FBF2F102FB11334362704700BFED
:107280004171704781717047D0E90920101AB0FA36
:1072900080F04009704700BF024BD3F894305B6820
:1072A000184700BF407E0020024BD3F894300830CE
:1072B0009B681847407E00200120704701207047DE
:1072C00001207047012070470120704731B10C4BFD
:1072D000D3ED267AF8EEE77AC1ED007A7AB1084B61
:1072E000DFED086AD3F89C30A3F5D543333B07EEB6
:1072F000903AF8EEE77A87EEA67A82ED007A704748
:10730000407E00200000C8420120704701207047E5
:1073100010B4754C0023224692F90410012902F1A1
:107320000C023AD00133072BF6D12246002392F902
:107330000410022902F10C0245D00133072BF6D1CB
:107340002246002392F90410032902F10C0255D0C1
:107350000133072BF6D12246002392F904100429A9
:1073600002F10C025ED00133072BF6D1002394F911
:107370000420052A04F10C0468D00133072BF6D150
:107380005A4B5B685B067BD401795DF8044B20396E
:1073900001298CBF002001207047554A03EB4303AD
:1073A00002EB8303D3F8A03003B3524A037992F877
:1073B0003DC09C4503D092F83C209A42B5D10120B3
:1073C0005DF8044B70474A4A03EB430302EB830327
:1073D000D3F8A03063B1484A037992F83D1099423E
:1073E000EDD092F83C209A42AAD1E8E722469EE7E7
:1073F00022460C3212F9081C0329A9D13C4A03EB9E
:10740000430302EB8303D3F8A030002B36D03B4A72
:10741000037992F83D109942D1D092F83C209A42DB
:1074200099D1CCE7324A03EB430302EB8303D3F851
:10743000A030002B9BD0324A037992F83D1099423C
:10744000BDD092F83C209A4290D1B8E7284A03EB8D
:10745000430302EB8303D3F8A030002B90D0294ADA
:10746000037992F83D109942A9D092F83C209A42B3
:10747000A5D01E4B5B685B0686D501E022466CE713
:10748000214B00229C4619460C791A2C01F114015B
:1074900004D001320C2AF7D1002403E002EB82026F
:1074A0000CEB820400221979192903F114030BD083
:1074B00001320C2AF7D1002C3FF466AF2268036832
:1074C0009A427FF461AF7AE701681CB123688B426E
:1074D0003FF475AF0D4B02EB820203EB82031B6995
:1074E0008B427FF451AF6AE7E07E0020AC000010D1
:1074F000407E0020B4000020000300204C05002046
:1075000098070020E4090020FC160020EC1600205B
:107510000C4B10B5844603F1F00E002002E014334A
:107520009E450ED01A686245F9D1DA688A4218BFC2
:10753000D96000F1010403F1140318BFE0B29E45C5
:10754000F0D110BDFC160020704700BF044B40F284
:10755000FF7203EBC0039142A8BF114699807047A8
:10756000F83F0020112807D8044B03EB8003D3F821
:10757000F4300BB19B6819602AF054BE407E0020A5
:10758000112807D8044B03EB8003D3F8F4300BB178
:107590009B681960704700BF407E00200D4A92F83A
:1075A000003183B10C4B93F83C1161B193F83D115C
:1075B00061B1D2F804010022FA2883F83D21A8BF66
:1075C0004FF0FF3070476FF0010070476FF002001E
:1075D000704700BFEC160020407E00200C4B93F853
:1075E0003E218AB193F83F215AB10A49D1F80801E6
:1075F0000022B0F5967F83F83F21A8BF4FF0FF30FF
:1076000070476FF0020070476FF00100704700BFD5
:10761000407E0020EC160020024BD3F840315B681E
:10762000184700BF407E0020024BD3F840319B68D2
:10763000184700BF407E0020024BD3F84031DB6882
:10764000184700BF407E0020014BD3F80C01704763
:10765000EC1600204B1EDBB2062B98BF214A30B53A
:1076600098BF32F81350204BA3F1580488BF4FF451
:107670008075002808BF1C46A44620893CF8082BCA
:1076800087B04FFA82FE90B1A5EB0E022B1A002AAA
:10769000B8BF5242002BB8BF5B429A42C4BF644697
:1076A0004FFA80FE3CF8080F0028EDD122880F4BDE
:1076B0000F4893F844C1A3790593A38804930D4B15
:1076C000BCF1000F18BF0346A078CDE90015CDE945
:1076D00002200321084A0120FEF7D6F9204607B010
:1076E00030BD00BF305A080854180020407E0020EA
:1076F000B8250908B40D0908B80D090870B5066861
:10770000F0690D461446A0B3D0F80130CDB1D0F8E1
:1077100005209FED1B7ADFED1B5ADFED1B6A07EE9C
:10772000902AF8EE677AB7EE006A77EEC77A77EEBE
:10773000A77A87EEA57A77EE467A67EEE67AC5ED08
:10774000007AACB107EE903A9FED107ADFED106A47
:107750009FED106AF8EEE77A67EE877A87EEA67AF1
:10776000DFED0D6A77EE467A77EEA67AC4ED007A01
:1077700070BD09211420FEF7F9F9F061C4E700BFDC
:107780009AC9CC449AC94C460E76D7450000484366
:1077900000E0FF44000048423393884370B5066818
:1077A000F06982B00D461446002848D0D0F8053064
:1077B000DFED266A9FED267A07EE903AF8EE677ABB
:1077C000D0F8013077EEE67AF3EE096A67EE877A51
:1077D000B2EE047A67EEA67AF4EEC77AF1EE10FA0A
:1077E00020DCBAEE047AF4EEC77AF1EE10FA19D47E
:1077F0002DB19FED187A67EE877AC5ED007A7CB1DE
:1078000007EE903A9FED146ADFED146AB8EE677ADE
:10781000DFED137AE7EE067A77EEA67AC4ED007A0A
:1078200002B070BD17EE900A7BF07EFF0D4ACDE9E5
:10783000000104210320FEF727F902B070BD0921E1
:107840001420FEF793F9F061B0E700BF0000004696
:10785000000080380AD778430319C83D3393884322
:10786000000048C2040E0908244B254A30B5D3F85D
:10787000484194F91030A16803EB830302EB8302C3
:1078800083B08DF80700D2F8C8018A070AD5012312
:107890000DF10702002172F06FFDA3689B0714D55C
:1078A00003B030BD636913B11A689B885383154BCD
:1078B00015491A68154B4D68D200A3FB0232920994
:1078C0004B685B1B9A42FBD2E1E70E4B0E491A68EC
:1078D0000E4B4FF4FA7000FB02F2A3FB0232486831
:1078E00092094B681B1A9A42FBD26369002BD7D0CE
:1078F0001A689B88138303B030BD00BF407E002010
:10790000EC16002084390020001000E0D34D6210F6
:1079100070B52B4C94F84C3182B023B9012084F817
:107920004C3102B070BDD4F84851264A95F9103058
:10793000A96803EB830302EB83030522ADF8002063
:107940008A07D3F8C80111D502236A4601A972F04B
:1079500013FDAB689B071CD59DF8053003F00103B0
:1079600083F0010084F84C3102B070BD6B6913B133
:107970001A689B885383144B14491A68144B4E6839
:10798000D200A3FB023292094B689B1B9A42FBD2A6
:10799000DAE70D4B0D491A680D4B48684FF4FA763B
:1079A00006FB02F2A3FB023292094B681B1A9A42B1
:1079B000FBD26B69002BCFD01A689B881383CBE76F
:1079C000407E0020EC16002084390020001000E0EA
:1079D000D34D62102DE9F04782B060B9364D95F86D
:1079E0004C31D5F8507173B900230120C5F85031DE
:1079F00002B0BDE8F087314B2F4D1F6895F84C3130
:107A00000744002BF0D0DFF8BC802D4CDFF8B8A085
:107A1000DFF8B890D5F8486196F9103003EB83038E
:107A200008EB83030522D3F8C801B368ADF8002042
:107A30009A072FD502236A4601A972F09DFCB3680C
:107A40009B0712D59DF8053013F0010302D185F88C
:107A50004C31C9E7194B1B6801229F4285F84C2124
:107A6000D8D8002002B0BDE8F087DAF800206168BD
:107A70004FF4FA7303FB02F2A9FB02329209636826
:107A80005B1A9A42FBD27369002BDBD01A689B8881
:107A90001383D7E7736913B11A689B885383DAF8A5
:107AA00000206168D200A9FB0232920963685B1A68
:107AB0009A42FBD2BEE700BF407E00206038002023
:107AC000001000E0EC16002084390020D34D621035
:107AD00010B50020FFF77EFF00B910BD084C06204E
:107AE000FFF7C2FE0123C72084F84C31FFF7BCFE2C
:107AF000044B1B6803F5A4430833C4F8503110BD90
:107B0000407E002060380020F0B5044689B0002097
:107B10000E461546FFF75EFF10B9204609B0F0BDCE
:107B20001D4F0620FFF7A0FE012387F84C3197F880
:107B30005421CDF80CD00223009300238DF804309B
:107B40000293E2B1CDE9066505930522230E8DF877
:107B5000013004920DF10203220C1A70D7F848018B
:107B60009C70220A5A700379022B10D00B4B1B68B1
:107B70002C4406332046C7F8503109B0F0BDCDE99A
:107B80000526042207950DF101030492E4E702A9FA
:107B90006BF09AFCEAE700BF407E002060380020CE
:107BA00070B5054688B000200E461446FFF712FF58
:107BB000E8B103220092164ACDF80CD092F8541185
:107BC000059600238DF80430029391B9CDE906148F
:107BD00004210DF101030491D2F848019D702A0C93
:107BE0001A702A0A5A700379022B0CD0204608B06A
:107BF00070BD290E8DF801100521CDE906340491E0
:107C00000DF10203E8E702A96BF05EFC2046EEE707
:107C1000407E0020F0B5064683B00020FFF7DAFE74
:107C200008B903B0F0BD324C0620FFF71DFE01225B
:107C300094F8543184F84C21D82100228DF8042086
:107C4000D4F848510091C6F307420BBB70BA8DF8C7
:107C50000120ADF80200042395F91020254902EB1C
:107C6000820201EB8202A968D2F8C8018A0714D502
:107C70006A46002172F080FBAB689B0720D51E4B43
:107C80001B6803F59C530833C4F8503103B0F0BDB2
:107C900030BACDF801000523DEE76A6912B1116838
:107CA00092884A83154A164E1168164A7768C900A9
:107CB000A2FB012189097268D21B9142FBD2D7E74E
:107CC0000E4B0F491A680F4B48684FF4FA7606FBC3
:107CD00002F2A3FB023292094B681B1A9A42FBD2B2
:107CE0006B69002BCBD01A689B881383C7E700BF52
:107CF000407E0020EC1600206038002084390020EF
:107D0000001000E0D34D6210244B254A30B5D3F863
:107D1000584194F91030A16803EB830302EB83020E
:107D200083B08DF80700D2F8C8018A070AD501236D
:107D30000DF10702002172F01FFBA3689B0714D509
:107D400003B030BD636913B11A689B885383154B28
:107D500015491A68154B4D68D200A3FB02329209EF
:107D60004B685B1B9A42FBD2E1E70E4B0E491A6847
:107D70000E4B4FF4FA7000FB02F2A3FB023248688C
:107D800092094B681B1A9A42FBD26369002BD7D029
:107D90001A689B88138303B030BD00BF407E00206B
:107DA000EC16002084390020001000E0D34D621052
:107DB000274B284A30B5D3F8584194F9103003EBDB
:107DC000830383B002EB8302A3688DF804000025CF
:107DD000D2F8C8018DF8055049BA9A07ADF80610D7
:107DE0000AD504230DEB0302002172F0C5FAA36843
:107DF0009B0714D503B030BD636913B11A689B8823
:107E00005383154B15491A68154B4D68D200A3FBD7
:107E1000023292094B685B1B9A42FBD2E1E70E4BA0
:107E20000E491A680E4B4FF4FA7000FB02F2A3FBE6
:107E30000232486892094B681B1A9A42FBD2636966
:107E4000002BD7D01A689B88138303B030BD00BFC6
:107E5000407E0020EC16002084390020001000E055
:107E6000D34D621070B52D4D2D4AD5F8584194F977
:107E7000103003EB830302EB8303A26882B000207F
:107E80004CF2050192078DF80200ADF80010D3F80E
:107E9000C80119D503236A4601A972F06DFAA368D7
:107EA0009B0724D595F85C319DF806203BB102F084
:107EB000010383F0010085F85C3102B070BD012040
:107EC00085F85C3102B070BD636913B11A689B8894
:107ED0005383144B14491A68144B4E68D200A3FB09
:107EE000023292094B689B1B9A42FBD2D2E70D4BA0
:107EF0000D491A680D4B48684FF4FA7606FB02F2FA
:107F0000A3FB023292094B681B1A9A42FBD26369A7
:107F1000002BC7D01A689B881383C3E7407E0020DC
:107F2000EC16002084390020001000E0D34D6210D0
:107F300070B55A4D5A4E82B0FF20FFF7E5FE2C680F
:107F4000012304F5FA74C6F8604186F85C3103E059
:107F50002B681B1B002B06DAFFF784FF0028F7D0E5
:107F60000023C6F86031D6F858414E4D94F91030D0
:107F7000A2684AF2010103EB830305EB8303ADF82A
:107F8000041000218DF806109107D3F8C80120D500
:107F9000032301AA002172F0EFF9A3689A0743D5E1
:107FA00094F9103003EB830305EB83034BF20102DA
:107FB000ADF80420D3F8C80118228DF80620032359
:107FC00001AA002172F0D8F9A3689B0714D502B06A
:107FD00070BD636913B11A689B885383324B334970
:107FE0001A68334B4E68D200A3FB023292094B68E9
:107FF0009B1B9A42FBD2CBE72B4B2C491A682C4B8C
:108000004FF4FA7000FB02F2A3FB023248689209B7
:108010004B681B1A9A42FBD26369002BD7D01A68AF
:108020009B88138302B070BD1F4B20481A68204BF9
:1080300046684FF4FA7102FB01F1A3FB0131890993
:1080400043689B1B9942FBD294F91030616903EBA2
:10805000830305EB8305D5F8C801B1B10B688988A6
:10806000198359834BF20103ADF8043018238DF8BE
:1080700006300E490E4B4D68D200A3FB0232920926
:108080004B685B1B9A42FBD299E74BF20103ADF8B8
:10809000043018238DF80630EBE700BF603800206D
:1080A000407E0020EC16002084390020001000E003
:1080B000D34D621070B50B4D0B4E2C680123044458
:1080C000C6F8604186F85C3103E02B681B1B002B6F
:1080D00006DAFFF7C7FE0028F7D00023C6F86031A4
:1080E00070BD00BF60380020407E00202DE9F04FB9
:1080F000DFF8C48198F864918BB007468B4616462A
:10810000B9F1000F00F0A480D8F86851684CA8427B
:108110003AD1FFF7A7FE48B92268D8F86011521A81
:10812000002A06DAFFF79EFE0028F5D00022C8F8E4
:1081300060210620FFF7E8FD0122ABB288F85C2140
:108140000193C5F30A0AB9F1000F4FD105E0226887
:10815000D8F86011521A002A03DAFFF783FE0028CC
:10816000F5D08DF80EA04FEA1A2AD8F85801CDF8AC
:1081700020B08DF80DA00996022248E02268D8F8B8
:108180006011521A002A06DAFFF76CFE0028F5D0BB
:108190000022C8F860210620FFF7B6FD012288F80A
:1081A0005C21D8F86C214FEAD22905E02268D8F882
:1081B0006011521A002A03DAFFF754FE0028F5D0A6
:1081C00049461020FFF7F4FD226802324FF0000903
:1081D000C8F86021012288F8649188F85C21A1E741
:1081E0002268D8F86011521A002A03DAFFF73AFE23
:1081F0000028F5D0019BCDF820B0D8F858018DF8B3
:108200000EA0C3F3022B8DF80DB0099684228DF8D1
:108210000C20017900220492079203AA05920229F8
:108220004FF0030206923ED022680232C8F8602165
:108230000122354488F85C21012288F86421C5F3C5
:108240000A02C8F8685142B1B8190BB0BDE8F08F06
:10825000C8E95A00164C054664E7D8F86C214FEA85
:10826000D229144AC2F8189205E02268D8F86011A1
:10827000521A002A03DAFFF7F5FD0028F5D0494627
:108280001020FFF795FD2268C8F86C510232C8F83B
:10829000602101210022B81988F85C1188F8642156
:1082A0000BB0BDE8F08F04A96BF00EF9BCE700BF7E
:1082B00060380020EC160020407E002070B5134C82
:1082C00094F8643103B970BDD4F86C61104B114D52
:1082D000F60AC3F8186205E02B68D4F860219B1AEF
:1082E000002B03DAFFF7BEFD0028F5D03146102041
:1082F000FFF75EFD2B6801210022023384F85C1138
:10830000C4F8603184F8642170BD00BF407E002055
:10831000EC16002060380020F0B5314D314C83B0B0
:10832000064605E02B68D4F860219B1A002B03DA7F
:10833000FFF798FD0028F5D0D4F858712A4A062393
:108340008DF8073097F9103003EB830302EB8303BA
:10835000D3F8C801BB689A0715D501230DF10702B0
:10836000002172F009F8BB689B0721D5F10AD820DB
:10837000FFF71EFD2B6801220F3384F85C21C4F83F
:10838000603103B0F0BD7B6913B11A689B885383D9
:10839000164B17491A68174BD1F804C0D200A3FB3B
:1083A000023292094B68A3EB0C039A42FAD2D4E74B
:1083B0000E4B0F491A680F4B4FF4FA7000FB02F294
:1083C000A3FB0232486892094B681B1A9A42FBD2FF
:1083D0007B69002BCAD01A689B881383C6E700BF4D
:1083E00060380020407E0020EC16002084390020F8
:1083F000001000E0D34D62102DE9F04F5D4DB5F84F
:10840000783083B0002B55D0D5F858715A4EDFF82C
:1084100074A15A4CDFF870B14FF000094FEA494897
:1084200005E03368D5F860219B1A002B03DAFFF7CB
:1084300019FD0028F5D097F91030BA6803EB8303D3
:1084400006210AEB83038DF804109107D3F8C801C5
:108450007ED5012301AA002171F08EFFBB684FEA8F
:10846000D8209A07C8F3C748C0B23CD5D823ADF886
:10847000043097F910308DF8070003EB83030AEB03
:1084800083038DF80680D3F8C80104230DEB0302A3
:10849000002171F071FFBB689B070ED50121336885
:1084A000B5F8782085F85C1189440F334A45C5F842
:1084B0006031B3D803B0BDE8F08FDBF800306168FD
:1084C0004FF4FA7203FB02F22D4BA3FB0232920926
:1084D00063685B1A9A42FBD27B69002BDED01A6874
:1084E0009B881383DAE7DBF80020254BD4F804C01F
:1084F0004FF4FA7102FB01F1A3FB013189096368B2
:10850000A3EB0C039942FAD24FF0000368F3070380
:1085100060F30F23ADF8063097F91030796903EB5B
:1085200083030AEB8303D3F8C80119B10B68898868
:1085300019835983D823ADF80430114B6168D200F8
:10854000A3FB0232920963685B1A9A42FBD29CE752
:108550007B6913B11A689B885383DBF8003061682C
:10856000DA00074BA3FB0232920963685B1A9A4256
:10857000FBD26EE7407E002060380020001000E053
:10858000D34D6210EC160020843900202DE9F04F05
:10859000DFF8AC81D8F81832B3EBD02F8BB005469A
:1085A0008946174661D1614C614ECDF81C90D6F8D2
:1085B00058910023C5F30A05C5F5006003228DF824
:1085C0000F300493089399F804308DF80C20B842CA
:1085D00003AAB4BF87B2BFB28DF80E5005922D0A20
:1085E0000422022B8DF80D500997069200F0998015
:1085F000256801230235C6F8605186F85C3103E036
:1086000023685B1B002B2CDAFFF72CFC0028F7D02B
:108610004CF20503ADF8043099F9103003EB8303F5
:1086200008EB8308D9F80830D8F8C8010022C6F84A
:1086300060218DF806209A075FD5032301AA02A9BD
:1086400071F09AFED9F808309B073ED59DF80A30A4
:10865000C3F30113013B022B33D938460BB0BDE8FD
:10866000F08F00200BB0BDE8F08F304C304E4FEA59
:10867000D02A05E02368D6F860219B1A002BF0DA97
:10868000FFF7F0FB0028F5D04FF0FF3351461320E1
:10869000C8F81832FFF78CFB012386F85C31236899
:1086A00003F1020BC6F860B104E02368A3EB0B03EF
:1086B000002BD6DAFFF7D6FB0028F6D0C8F818A2B0
:1086C00073E7FFF735FC3846C8E71A4B1A491A68B2
:1086D0001A4B48684FF4FA7404FB02F2A3FB02320F
:1086E00092094B681B1A9A42FBD2D9F81430002B1E
:1086F000ACD01A689B881383A8E7D9F8143013B15B
:108700001A689B8853830B4B0B491A680B4B4C68B8
:10871000D200A3FB023292094B681B1B9A42FBD288
:108720008BE704A948466AF0CFFE61E76038002075
:10873000407E002084390020001000E0D34D6210FC
:10874000EC1600202DE9F0410C4E356873691D4090
:1087500011D0DFF82C800127B5FA85F4C4F11F048D
:1087600008EB840307FA04F4D3F870010368984710
:10877000A5437461F0D1BDE8F08100BF003C014029
:10878000407E002070B583681C686379DB0748D59C
:10879000A37994F85C22E06B03F001010E461ABB4A
:1087A00094F85F32012B3DD0002B3FD194F85E321C
:1087B00094F85DE29E450ED9B4F86622012505FACB
:1087C00003FC013342EA0C025FFA83FCE64592B2F5
:1087D000F5D8A4F86622012384F85F3286EA030103
:1087E000BDE870406AF072BC43681A68D36AC3F38C
:1087F0004E03536294F86D32012B07D094F8613226
:1088000023B1B4F868320133A4F8683286F001016C
:108810006AF05CFC00224FF08073A4F86622C4F872
:108820005C3270BD94F85D3284F85E32002384F8C7
:108830005F32BDE870406AF049BC00BFF0B52DED75
:10884000028B4D4E16F84C3C022B83B00D4614465D
:1088500019D0DFED4A7A7DB19FED497A9FED496AE3
:10886000DFED496A67EEA77A67EE877A87EE867A48
:1088700077EE267AC5ED007A0CB1444B236003B045
:10888000BDEC028BF0BD424B317C9B6803F00202D1
:1088900039BB5B0525D42AB3B6F9363007EE903ADA
:1088A000B6F93430F8EEE77A06EE903A27EEA77A7A
:1088B000F8EEE66AB6F93830A6EEA67A07EE903AF8
:1088C000F8EEE77AA7EEA77AB5EEC07AF1EE10FAE5
:1088D000BFDBF1EEC77AF4EE677AF1EE10FABAD7A1
:1088E000B7E71AB9336DD3ED337AB4E7294F0DF1F9
:1088F00006002EF01BFBBDF80630D7F89C259FED37
:10890000266ADFED266A9FED267A9B1A07EE903ADB
:10891000F8EEE77AB0EE408A67EE867AA7EEA67A9E
:10892000FDEEC77AB0EE470A17EE903A2033402B9F
:108930001FD8FCF7EBFE1B4B97F8C211D6ED077A58
:10894000A3F12C021846443B002918BF134693EDAF
:10895000057AD0ED006A77EE877AE8EE406A27EE76
:10896000A77AA6EEA67AB5EEC07AF1EE10FAB0DAE2
:108970006FE79FED020ADEE7388F0020000000005D
:10898000CDCC9C3F00409C4682E6C54733139043C4
:10899000AC000010407E00200AD7233C35FA8E3C04
:1089A000DB0FC93FF083002010B50B4B82B053F8AA
:1089B000304001916CB107EE901A94ED047A94ED79
:1089C000030AF8EEE77AA7EE870A73F009F8A368BE
:1089D000186002B010BD00BFF83F0020184B53F8DC
:1089E000200048B310B5174C00EB400004EB8003A7
:1089F00093F955C0BCF1FF3F1FD093F85D00D0B193
:108A000004EB0C0293F85C0092F8A8E08C2314218C
:108A100003FB0CFC00220CEB000304EB43030139C5
:108A2000B3F8AC30704412FA83F2F4D1064BA3FBD6
:108A30000230C0F30F1010BD7047002010BD00BF02
:108A4000407E0020388F0020CDCCCCCC30B5032028
:108A500083B00D461446FFF7C1FF01909DB107EEAC
:108A6000900A9FED0B7AF8EE677AF0EE006A67EEF7
:108A7000877AB8EE047AA7EEA67ADFED067A67EE7B
:108A8000277AC5ED007A0CB1034B236003B030BDEB
:108A90006740533A00007A4433139043E8B170B50D
:108AA00006680E4B06F13F4202F57E0203EB92236D
:108AB0000C4682B00546187C6AF0BEFB6209C4F31E
:108AC0000013A9883046CDE90032C4F3810304F0D5
:108AD000030271F0F7FB02B070BD7047305A08080E
:108AE00070B5104B104CA3421AD2054602E00C336D
:108AF000A34215D293F805C08C45F8D193F804C071
:108B0000AC4501D0002DF2D1D8799042EFD1186850
:108B100090F804E0E645EAD106689E42E7D170BDD0
:108B2000002070BD788C0908348E09080379022B67
:108B300000D0704710B490F910201D481D4C83B030
:108B400002EB82020831694400EB82020094D2F801
:108B5000C82111F8084C18498A4225D0A1F578415E
:108B60008A4223D001F580618A4219D1118821F00F
:108B70004001090403EB8303090C118000EB83001F
:108B80001388D0F8D41123F0380331F824101B04D3
:108B90001B0C0B43138013889BB243F040031380DC
:108BA00003B05DF8044B70470023DFE70123DDE7E6
:108BB000EC160020000102030030014010B504460D
:108BC000C06900B110BD09211420FCF7CFFFE0619E
:108BD00010BD00BF034690F910002DE9F041244C70
:108BE00000EB800016469A6804EB80009207D0F8EC
:108BF000C88109D5404671F057FC3146404671F0B6
:108C000053FC0120BDE8F0815D69084615B12B6871
:108C1000AA885A83174B184F1C68184B7A684FEA7A
:108C2000C40CA3FB0C3C4FEA9C1C7B689B1A9C4524
:108C3000FBD20146404671F037FC3146404671F0A8
:108C400033FC0E4B78680C494FF4FA7204FB02F2C5
:108C5000A3FB023292094B681B1A9A42FBD2002DE9
:108C6000CFD02B68AA881A830120BDE8F08100BF0D
:108C7000EC16002084390020001000E0D34D621073
:108C800010B50379012B84B08E460DD0022B02D093
:108C9000002004B010BD8368DB0758BF01F07F01DE
:108CA00004B0BDE8104095E7144682688DF80F4087
:108CB00002F0010201920DF10F020092417C90F945
:108CC00010007246FAF7C4FC04B010BD2DE9F04163
:108CD000076888B08046B6227E213846FFF7D0FF6D
:108CE000642605F01DFD04460D4605F019FD001B28
:108CF00061EB0501B0F57A7F71F10001F5D3013E1A
:108D0000EFD102213846FFF711FF7B6913B11A68D2
:108D10009B88538305F004FD04460D4605F000FDD5
:108D2000001B61EB0501B0F57A7F71F10001F5D30D
:108D30007B6913B11A689B8813830A2605F0F0FC3F
:108D400004460D4605F0ECFC001B61EB0501B0F597
:108D50007A7F71F10001F5D3013EEFD132467C21DB
:108D60003846FFF78DFF05F0DBFC04460D4605F0A5
:108D7000D7FC001B61EB0501B0F57A7F71F10001B2
:108D8000F5D3002259213846FFF77AFF05F0C8FCD9
:108D900004460D4605F0C4FC001B61EB0501B0F56F
:108DA0007A7F71F10001F5D35E22002371498DF8BD
:108DB00007200DF10702CDE902320122CDE905318C
:108DC000049202A94FF4A472384607926AF07CFB21
:108DD0000A2605F0A5FC04460D4605F0A1FC001B83
:108DE00061EB0501B0F57A7F71F10001F5D3013E29
:108DF000EFD1012259213846FFF742FF05F090FCE0
:108E000004460D4605F08CFC001B61EB0501B0F536
:108E10007A7F71F10001F5D38C2240213846FFF7AB
:108E20002FFF05F07DFC04460D4605F079FC001B84
:108E300061EB0501B0F57A7F71F10001F5D30322F2
:108E400041213846FFF71CFF05F06AFC04460D4639
:108E500005F066FC001B61EB0501B0F57A7F71F14E
:108E60000001F5D3444CD8F8382098F83500B4FB0D
:108E7000F2F2032391B2414AFDF7A4FF4388B4FB09
:108E8000F3F4C8F840400279422142F0C00238466B
:108E9000FFF7F6FE05F044FC04460D4605F040FCE5
:108EA000001B61EB0501B0F57A7F71F10001F5D38C
:108EB000082243213846FFF7E3FE05F031FC044663
:108EC0000D4605F02DFC001B61EB0501B0F57A7F26
:108ED00071F10001F5D3042258213846FFF7D0FE86
:108EE00005F01EFC04460D4605F01AFC001B61EB64
:108EF0000501B0F57A7F71F10001F5D30A22532103
:108F00003846FFF7BDFE05F00BFC04460D4605F0A4
:108F100007FC001B61EB0501B0F57A7F71F10001E0
:108F2000F5D300227C213846FFF7AAFE05F0F8FBB6
:108F300004460D4605F0F4FB001B61EB0501B0F59E
:108F40007A7F71F10001F5D306227D213846FFF7C3
:108F500097FE05F0E5FB04460D4605F0E1FB001B1E
:108F600061EB0501B0F57A7F71F10001F5D308B02E
:108F7000BDE8F081485A080840420F00905B08089D
:108F8000F8B57822074600210068FFF779FE05262C
:108F900005F0C6FB04460D4605F0C2FB001B61EB65
:108FA0000501B0F57A7F71F10001F5D3013EEFD1F3
:108FB000386820220121FFF763FE052605F0B0FB8B
:108FC00004460D4605F0ACFB001B61EB0501B0F556
:108FD0007A7F71F10001F5D3013EEFD13246386856
:108FE0000221FFF74DFE642605F09AFB04460D466C
:108FF00005F096FB001B61EB0501B0F57A7F71F17E
:109000000001F5D3013EEFD10120F8BD70B5242257
:10901000044641210068FFF733FE90B9052605F0AC
:109020007FFB04460D4605F07BFB001B61EB050151
:10903000B0F57A7F71F10001F5D3013EEFD1012047
:1090400070BD206820223021FFF71AFE0028E5D0ED
:10905000206806223121FFF713FE0028DED02068A9
:1090600000223421FFF70CFED8E700BFF8B5072235
:1090700007460A210068FFF703FE052605F050FBAE
:1090800004460D4605F04CFB001B61EB0501B0F5F5
:109090007A7F71F10001F5D3013EEFD138682422C7
:1090A0004121FFF7EDFD052605F03AFB04460D468C
:1090B00005F036FB001B61EB0501B0F57A7F71F11D
:1090C0000001F5D3013EEFD13868C0224221FFF7FD
:1090D000D7FD052605F024FB04460D4605F020FBD0
:1090E000001B61EB0501B0F57A7F71F10001F5D34A
:1090F000013EEFD10120F8BD10B504460022212128
:109100000068FFF7BDFD2068FC222021FFF7B8FDB5
:10911000206840222421FFF7B3FD20680C22232180
:10912000FFF7AEFD206800222221FFF7A9FD0120F4
:1091300010BD00BFF8B50122074610210068FFF7F7
:109140009FFD00B9F8BD142605F0EAFA04460D4665
:1091500005F0E6FA001B61EB0501B0F57A7F71F1CD
:109160000001F5D3013EEFD13868A022BDE8F840F8
:10917000112185E52DE9F041802207460B21006889
:10918000FFF77EFD1E26804605F0CAFA04460D460E
:1091900005F0C6FA001B61EB0501B0F57A7F71F1AD
:1091A0000001F5D3013EEFD1B8F1000F02D100204C
:1091B000BDE8F081386806222921FFF761FD00280B
:1091C000F5D0386808220B21FFF75AFD0028EED0B1
:1091D0003868CF22BDE8F0410A2151E510B50446B8
:1091E00094220B210068FFF74BFD206871220121BA
:1091F000FFF746FD206800220421FFF741FD2068AB
:10920000C8220521FFF73CFD206800220621FFF758
:1092100037FD2068C8220721FFF732FD20680022B1
:109220000821FFF72DFD2068C8220921FFF728FD3E
:10923000012010BD00B500680379012B85B012D064
:10924000022B03D0012005B05DF804FB8368DB0727
:109250004FF031024CBFF4217421FFF7BBFC012019
:1092600005B05DF804FB826890F910C0417C02F003
:10927000010201920DF10F0200926046F4224FF0BC
:10928000310C8DF80FC0FAF7E3F9012005B05DF855
:1092900004FB00BF10B5044600680379012B84B0BD
:1092A00011D0022B02D0002004B010BD01220B21EE
:1092B000FFF790FC0028F6D020681D22092104B099
:1092C000BDE81040DCE4826890F910C0417C8DF864
:1092D0000F3002F0010201920DF10F020092604680
:1092E0000B22FAF7B5F9E5E72DE9F04105461F46EF
:1092F00095F91030244803EB830300EB8300AB683F
:10930000D0F8C88116469A070ED5404671F0CCF8C1
:109310003B4632460021404671F02EF8AB689B0771
:1093200018D50120BDE8F0816B6913B11A689B88DC
:109330005383164B164A1B684FEAC30E154BA2FB0C
:109340000E2E5A684FEA9E1E5C68A4EB020CE6459E
:10935000FAD2DAE70D4B0F491A680D4B4FF4FA7049
:1093600000FB02F2A3FB0232486892094B681B1A09
:109370009A42FBD26B69002BD3D01A689B88138367
:109380000120BDE8F08100BFEC16002084390020E8
:10939000D34D6210001000E030B50579012D83B087
:1093A0008E460DD0022D02D0002003B030BD84685F
:1093B000E40758BF41F0800103B0BDE8304093E7B7
:1093C00014468268009402F00102417C90F910007A
:1093D00001927246FAF73CF903B030BD10B5164C55
:1093E00084F8F513017984F8F62301294FF000027F
:1093F00082B084F8F42310D0022903D06FF00C005F
:1094000002B010BD032304F57D72FF21FFF76CFF4E
:109410000028F3D0002002B010BD8268417C90F992
:10942000100004F57D7402F00102CDE9004203232F
:10943000FF22FAF70DF9EBE7388F00200068037977
:10944000012B0AD0022B00D0704783680D4A13F01D
:10945000010314D00023512146E700B58368094A6F
:10946000417C90F9100083B003F00103CDE90023A3
:1094700000235122FAF7ECF803B05DF804FBD12188
:1094800032E700BF2C9400202DE9F04105461F462D
:1094900095F91030244803EB830300EB8300AB689D
:1094A000D0F8C88116469A070ED5404670F0FCFFEA
:1094B0003B4600223146404670F05EFFAB689B079A
:1094C00018D50120BDE8F0816B6913B11A689B883B
:1094D0005383164B164A1B684FEAC30E154BA2FB6B
:1094E0000E2E5A684FEA9E1E5C68A4EB020CE645FD
:1094F000FAD2DAE70D4B0F491A680D4B4FF4FA70A8
:1095000000FB02F2A3FB0232486892094B681B1A67
:109510009A42FBD26B69002BD3D01A689B881383C5
:109520000120BDE8F08100BFEC1600208439002046
:10953000D34D6210001000E030B50579012D83B0E5
:109540008E460DD0022D02D0002003B030BD8468BD
:10955000E40758BF41F0800103B0BDE8304093E715
:1095600014468268009402F00102417C90F91000D8
:1095700001927246FAF77CFA03B030BD10B504468A
:109580000068037982B0022B0CBF4321032106231C
:109590006A46FFF7D1FF68B1BDF80010BDF80220A0
:1095A000BDF8043049BA52BA5BBAE18662872387B4
:1095B00002B010BDC4F83600608702B010BD00BF15
:1095C00070B50668F56982B00446002D59D00023B5
:1095D0002B7004230DEB03023046FF21FFF7ACFF95
:1095E00010B9002002B070BD206804236A46FF2134
:1095F000FFF7A2FF0028F4D09DF804309B09023B3E
:10960000012BEED9BDF80430BDF80620BDF80010DE
:10961000BDF802605BBA43F6FF74C3F30D03A342C7
:10962000DFD0002BDDD052BAC2F34A1240F2FF7CE9
:109630006245D6D0002AD4D049BAC1F30D01A14267
:10964000CFD00029CDD076BAC6F34A166645C8D029
:10965000002EC6D05C1A002CB8BF6442FF2CC0DCC0
:10966000941B002CB8BF6442FF2CBADC0B445B1087
:1096700032445210C5F805300123C5F801202B7083
:10968000B0E709211420FCF771FAF061054626685D
:109690009DE700BF70B50668F46982B0F4B100239D
:1096A000237004230DEB0302FF213046FFF744FF34
:1096B00010B39DF804309B0919D1BDF80420BDF802
:1096C000063052BA5BBA92B2C3F34A130121217039
:1096D000C4F80520C4F8013002B070BD0546092168
:1096E0001420FCF743FAF06104462E68D7E7044AD9
:1096F00004210320FCF7C8F9002002B070BD00BFB0
:10970000280E09082DE9F041104C04F57D7884F805
:10971000F5131746002502234246FF21064684F82A
:10972000F453FFF739FE68B1424630460223FF2169
:10973000FFF702FF30B1B4F8F4335BBA28463B8040
:10974000BDE8F0816FF00C00FAE700BF388F002011
:1097500030B51A4D95F83E3183B00BB903B030BD2A
:1097600004460DF1050100686FF0CEFF9DF805304D
:1097700083B9134A206801214FF4064482F8F61396
:10978000A2F8F443032302F57D72FF2103B0BDE884
:10979000304001E60DF1060296212068FFF7B2FF86
:1097A000084ABDF806300849A2FB0323DB08012262
:1097B000C1F8083185F83F21DBE700BF407E00207B
:1097C000388F0020CDCCCCCCEC16002010B5044650
:1097D00000680379012B84B02DD0022B01D000202A
:1097E00027E0836813F0010F02AA4FF0060314BFAD
:1097F0001F219F21FFF748FE0028F0D0BDF8081078
:10980000BDF80A20BDF80C30C9BA07EE901AD2BADA
:10981000F8EEE76A07EE902ADBBAB8EEE77A07EED1
:10982000903AF8EEE77AC4ED046A84ED057AC4ED67
:10983000067A04B010BD8368417C90F9100003F0F3
:109840000103019302AB00931F220623FAF710F9DC
:10985000D2E700BF10B5044600680379012B84B03D
:109860002DD0022B01D0002027E0836813F0010FD8
:1098700002AA4FF0060314BF2521A521FFF704FE1D
:109880000028F0D0BDF80810BDF80A20BDF80C3053
:10989000C9BA07EE901AD2BAF8EEE76A07EE902A34
:1098A000DBBAB8EEE77A07EE903AF8EEE77AC4ED65
:1098B000076A84ED087AC4ED097A04B010BD8368A4
:1098C000417C90F9100003F00103019302AB009377
:1098D00025220623FAF7CCF8D2E700BF10B50068BE
:1098E0000379012B84B00C4625D0022B01D0002037
:1098F0001FE0826812F0010F18BF1D2103AA08BFE4
:109900009D21FFF7C1FD0028F1D0BDF80C309FED7F
:10991000116ADFED116ADBBA07EE903AB8EEE77A2A
:10992000C7EE067A77EEA67AFDEEE77A17EE903A62
:10993000238004B010BD8368417C90F9100003F0CF
:109940000103019303AB00931D220223FAF790F861
:10995000D9E700BFCFF7534100007A4300B5006854
:109960000379012B85B030D0022B0BD01E4AD2F8E0
:10997000F434D2F8F82400201C490A610B6305B0C6
:109980005DF804FB062302AAF721FFF77DFD0028FE
:10999000ECD09DF809309DF808C09DF80C209DF88A
:1099A0000A109DF80BE01B0143EA0C3312019DF8ED
:1099B0000DC043EA111342EA0E320B4942EA1C126F
:1099C000C1F8F434C1F8F824D6E78368417C90F9F3
:1099D000100002AA03F00103CDE900230623F722B9
:1099E000FAF746F8D3E700BF388F0020407E00200A
:1099F00010B5044600680379012B84B043D0022BD4
:109A000007D0002213461046C4F83620638704B0FE
:109A100010BD836813F0010F02AA4FF0060314BFB4
:109A200011219121FFF730FD0028EAD0BDF908206F
:109A3000BDF90A3006EE902A5B42BDF90C2007EE14
:109A4000103AF8EEE66AB7EE086A07EE902A66EE7C
:109A5000866AB8EEC77AFDEEE66A27EE067AF8EE79
:109A6000E77A16EE903A67EE867ABDEEC77AFDEE9B
:109A7000E77AE38617EE103A238717EE903A1BB287
:109A8000638704B010BD8368417C90F9100003F037
:109A90000103019302AB009311220623F9F7E8FFBB
:109AA000C2E700BF10B5044600230068C4F8363092
:109AB00063870379012B84B022D0022B01D00020D0
:109AC0001CE0836813F0010F02AA4FF0060314BFD5
:109AD00003218321FFF7D8FC0028F0D0BDF90A301C
:109AE000BDF80810BDF80C205B4201EB410103EB0F
:109AF000430302EB4202E1862387628704B010BD74
:109B00008368417C90F9100003F00103019302ABDC
:109B1000009303220623F9F7ABFFDDE710B50446F7
:109B20004FF0000C0068C4F836C0A4F83AC00379BE
:109B3000012B84B018D0022B01D0002012E08368E2
:109B400013F0010F02AA4FF0060314BF61468021F3
:109B5000FFF79AFC0028F0D0029ABDF80C30C4F848
:109B60003620638704B010BD836890F910E0417C13
:109B700003F00103019302AB009362460623704693
:109B8000F9F776FFE6E700BF10B584B0002304467E
:109B900000680293CDF80B300279012A1ED0022A08
:109BA00019D1836813F0010F02AA4FF0070314BF05
:109BB0004E21CE21FFF768FCBDF80910BDF80B203F
:109BC000BDF80D30C9BAD2BADBBA0120E1862287CE
:109BD000638704B010BD1A461946F6E7836890F90A
:109BE00010C0417C02AA03F00103009201934E22AF
:109BF00007236046F9F73CFFDEE700BF00B50068C9
:109C00000379012B85B00DD0022B07D1012303AAC4
:109C1000FF21FFF739FC05B05DF804FB002005B01B
:109C20005DF804FB8268417C90F9100002F00102AB
:109C3000019203AA0092FF22F9F71AFF05B05DF81E
:109C400004FB00BF30B5044600680379012B85B0E2
:109C50002DD0022B0ED0224B6FF00102C3F80C2145
:109C60002049214AD1F8FC3415683233AB422CD359
:109C700005B030BD826812F0010F18BF512103AA50
:109C800008BFD121FFF700FC0028E4D0BDF80C305C
:109C9000134A5BBA9BB2C2F80C31D2F80C31B3F55F
:109CA000C87FDDDD4FF0FF33C2F80C31D8E78368A1
:109CB000417C90F9100003F00103019303AB009382
:109CC00051220223F9F7D4FEDEE701F2F442C1F893
:109CD000FC54206800235121FFF75EFB05B030BD26
:109CE000EC160020388F00206038002070B5044644
:109CF000234894F9103003EB830300EB8300A3683F
:109D0000D0F8C86115469A070DD5304670F0CCFBE7
:109D1000012300222946304670F02EFBA3689B07E2
:109D200016D5012070BD636913B11A689B885383EF
:109D3000144B154A1B6850684FEAC30C134BA3FB26
:109D40000C3C4FEA9C1C53681B1A9C45FBD2DCE779
:109D50000C4B0D491A680D4B4FF4FA7000FB02F2E0
:109D6000A3FB0232486892094B681B1A9A42FBD245
:109D70006369002BD5D01A689B881383012070BDBE
:109D8000EC16002084390020001000E0D34D621052
:109D900010B50379012B82B08E460DD0022B02D074
:109DA000002002B010BD8368DB0758BF41F080017E
:109DB00002B0BDE8104099E714468268009402F0B2
:109DC0000102417C90F9100001927246F9F750FEB1
:109DD00002B010BD2DE9F043836B0768A04AA14C87
:109DE000B4FBF3F183B08046052389B290F83500C7
:109DF000FCF7E8FF00214388B4FBF3F48146C8F880
:109E000040403846FEF792FE002276213846FEF7A3
:109E100037FF0F224E213846FEF732FF0F2604F09F
:109E20007FFC04460D4604F07BFC001B61EB050142
:109E3000B0F57A7F71F10001F5D3013EEFD199F8C9
:109E400005204F2102F00F023846FEF719FF0F26BA
:109E500004F066FC04460D4604F062FC001B61EB56
:109E60000501B0F57A7F71F10001F5D3013EEFD124
:109E700099F80520502102F00F023846FEF700FF46
:109E80000F2604F04DFC04460D4604F049FC001B6F
:109E900061EB0501B0F57A7F71F10001F5D3013E68
:109EA000EFD1FF2252213846FEF7EAFE0F2604F0DA
:109EB00037FC04460D4604F033FC001B61EB050142
:109EC000B0F57A7F71F10001F5D3013EEFD198F83A
:109ED0003510072941D0644D95F84401FDF7BAFBD0
:109EE0000446012276213846FEF7CAFEA2780C21EC
:109EF0003846FEF7C5FE22790D213846FEF7C0FE32
:109F0000A279A388120142EA1322D2B20E21384666
:109F1000FEF7B6FE4FF4807195F84401FDF79AFB09
:109F20000446022276213846FEF7AAFEA2785200A5
:109F3000032102F0FE023846FEF7A2FE2279042138
:109F40003846FEF79DFEA279A388120142EA132249
:109F50000521D2B23846FEF793FE0022762138461C
:109F6000FEF78EFE032214213846FEF789FE0F26E7
:109F700004F0D6FB04460D4604F0D2FB001B61EB57
:109F80000501B0F57A7F71F10001F5D3013EEFD103
:109F9000324663213846FEF773FE642604F0C0FBA8
:109FA00004460D4604F0BCFB001B61EB0501B0F557
:109FB0007A7F71F10001F5D3013EEFD108226521CE
:109FC0003846FEF75DFE64210DF107023846FFF7C3
:109FD000DFFE9DF8072022F0100242F060026421AB
:109FE00038468DF80720FEF74BFE0F2604F098FB4D
:109FF00004460D4604F094FB001B61EB0501B0F52F
:10A000007A7F71F10001F5D3013EEFD10DF1060227
:10A010004D213846FFF7BCFE9DF8062002F03F02B6
:10A0200042F040024D2138468DF80620FEF728FE0A
:10A030000F2604F075FB04460D4604F071FB001B6F
:10A0400061EB0501B0F57A7F71F10001F5D3013EB6
:10A05000EFD103213846FEF769FD03B0BDE8F08378
:10A06000A45B080840420F00407E0020F0B583B09A
:10A0700015460DF107021C4606460F46FFF788FEFF
:10A080009DF8072005EA0203A34201D103B0F0BD09
:10A0900022EA050222433946304603B0BDE8F040CB
:10A0A000FEF7EEBD10B582B004466A46006808218E
:10A0B000FFF76EFE9DF80030DB0602D4002002B0F0
:10A0C00010BD206806236A460021FFF735FA0028F4
:10A0D000F4D09DF801309DF800109DF802209FED0E
:10A0E0004B6A1B0203EB01439DF804101C029DF810
:10A0F00003401A444FEA01219DF8053001EB044169
:10A1000048BF02F17F420B4407EE902A090248BF84
:10A1100003F17F43B8EEE77A07EE903AF8EEE77A7C
:10A12000C7EE066A3A4BB3F94020B3F94610C7EEC2
:10A13000863A07EE102A374A93ED0F6A92F80045E7
:10A14000B3F94220D3ED0E7AF8EEC65A06EE102A85
:10A15000B3F9442005EE102AB3F9482004EE901A12
:10A1600004EE102AB8EEC77A112CF8EEE77AB8EEB2
:10A17000C66AB8EEC55AF8EEE44AB3F94A10B3F924
:10A180004C20B8EEC44A27EE237A26EEA32A23D029
:10A19000A6EE845AA6EEA46AE5EE265AE5EEA67A65
:10A1A00077EE877AE6EE027AB3F9362007EE102AC8
:10A1B000B3F93420C3ED147A06EE902AB8EEC77ACC
:10A1C000F8EEE66A27EE237AB6EE006AA6EE867A05
:10A1D00083ED157A02B010BD03EE102AF8EEC32A03
:10A1E00003EE101AA6EEA24AB8EEC33AA4EE265A1F
:10A1F000E6EE834AE5EE265AA4EEA66AE5EEA67AD6
:10A2000077EE877AE6EE027ACEE700BF0000784864
:10A21000407E0020388F0020F0B5002283B0074632
:10A220000A210068FEF72CFD142604F079FA044692
:10A230000D4604F075FA001B61EB0501B0F57A7F5D
:10A2400071F10001F5D3013EEFD138680F220A21E8
:10A25000FEF716FD0A2604F063FA04460D4604F0E4
:10A260005FFA001B61EB0501B0F57A7F71F1000127
:10A27000F5D3013EEFD13868032301AA1021FFF77F
:10A280005BF90A2604F04CFA04460D4604F048FA3D
:10A29000001B61EB0501B0F57A7F71F10001F5D388
:10A2A000013EEFD19DF804209DF805009DF80610B1
:10A2B000194B803280308031A3F80425A3F80605BD
:10A2C0003246A3F8081538680A21FEF7D9FC0A2699
:10A2D00004F026FA04460D4604F022FA001B61EB56
:10A2E0000501B0F57A7F71F10001F5D3013EEFD1A0
:10A2F0000DF1030238680221FFF74AFD0DF1030258
:10A3000038680921FFF744FD386811220A21FEF759
:10A31000B7FC012003B0F0BD388F0020F0B500225B
:10A3200083B007460A210068FEF7AAFC142604F051
:10A33000F7F904460D4604F0F3F9001B61EB050143
:10A34000B0F57A7F71F10001F5D3013EEFD13868A5
:10A350000F220A21FEF794FC0A2604F0E1F90446D4
:10A360000D4604F0DDF9001B61EB0501B0F57A7FC5
:10A3700071F10001F5D3013EEFD13868032301AA42
:10A380001021FFF7D9F80A2604F0CAF904460D4651
:10A3900004F0C6F9001B61EB0501B0F57A7F71F19D
:10A3A0000001F5D3013EEFD1324638680A21FEF7AD
:10A3B00067FC0A2604F0B4F904460D4604F0B0F92F
:10A3C000001B61EB0501B0F57A7F71F10001F5D357
:10A3D000013EEFD10DF1030238680221FFF7D8FCEE
:10A3E0000DF1030238680921FFF7D2FC3868012219
:10A3F0000A21FEF745FC012003B0F0BD30B5002373
:10A4000085B00446C0F8363043870DF10702006876
:10A410000221FFF7BDFC18B19DF80730DB0703D41C
:10A420000025284605B030BD062302AA0321206876
:10A43000FFF782F820680DF107020921FFF7A8FC59
:10A4400005460028ECD09DF8073013F00C0FE7D13B
:10A45000BDF80820BDF80C30BDF80A102068C2EB2A
:10A460008232C3EB83339B0092008900E28621870E
:10A47000638701220A21FEF703FC284605B030BDA0
:10A48000F0B583B0002307468DF80230142604F09F
:10A4900047F904460D4604F043F9001B61EB050142
:10A4A000B0F57A7F71F10001F5D3013EEFD131466D
:10A4B0000DF102023868FFF76BFC0DF102028021FA
:10A4C0003868FFF765FC4FF4F842ADF804203868AF
:10A4D0008DF80660032301AA6021FEF75DFF1426B4
:10A4E00004F01EF904460D4604F01AF9001B61EB56
:10A4F0000501B0F57A7F71F10001F5D3013EEFD18E
:10A5000031460DF1030238688DF80360FFF740FC17
:10A510004CF26243ADF8043004238DF806303868FD
:10A52000032301AA6021FEF737FF142604F0F8F890
:10A5300004460D4604F0F4F8001B61EB0501B0F58C
:10A540007A7F71F10001F5D3013EEFD131460DF173
:10A55000030238688DF80360FFF71AFC4FF4E853E4
:10A56000ADF8043008238DF80630386801AA0323BB
:10A570006021FEF711FF142604F0D2F804460D46C0
:10A5800004F0CEF8001B61EB0501B0F57A7F71F1A4
:10A590000001F5D3013EEFD10DF1030231463868D9
:10A5A0008DF80360FFF7F4FB38680DF102021E21FD
:10A5B000FFF7EEFB012003B0F0BD00BF2DE9F04135
:10A5C0004D4F97F83C3182B043B14C4E96F80A5546
:10A5D000012D04463BD0022D5AD015B102B0BDE882
:10A5E000F081012280210068FEF74AFB20680122E9
:10A5F000FF21FEF745FB2A4629462068FEF740FB6F
:10A6000096F80B2520689121FEF73AFB2946206831
:10A610000122FEF735FB2A462068FF21FEF730FBBA
:10A620002A4620688021FEF72BFB2946206801225C
:10A63000FEF726FB324B33491A6881F800010123EB
:10A64000C6F80C2586F80A3502B0BDE8F08101AAEB
:10A650000068DFF8B0800021FFF79AFB9DF8043016
:10A6600088F80001DA073ED5D6F81035002BB5D0B2
:10A67000234AD6F80C15126892B2521A9342ADD200
:10A680004FF0FF320023C8F8042186F80A35A5E709
:10A690000068DFF8708001AA1321FFF779FB9DF8AD
:10A6A000043088F800015B07DED020682B4601AA41
:10A6B0001E21FEF741FFBDF80430206801220B2166
:10A6C0005CBAFEF7DDFA104B88F80001A4B2A3FBD8
:10A6D0000434E40801220023C8F8044187F83D212E
:10A6E00086F80A357AE7064A02231268C6F80C256E
:10A6F00086F80A3572E700BF407E0020388F0020C0
:10A7000060380020EC160020CDCCCCCC30B504460F
:10A7100000680379012B85B062D0022B03D000259D
:10A72000284605B030BD826802AD12F0010F18BF97
:10A7300019462A4608BF8221FFF7D8FA0028EED032
:10A740009DF80830DA07EAD52A4620680723032156
:10A75000FEF7F2FE05460028E1D0206811220A210A
:10A76000FEF78EFA9DF80E301B07D8D42A49BDF8A3
:10A770000830B1F8042513FB02F3284A93423FDB6B
:10A78000B3F5000F3ADA002BB8BFFF331B125B4260
:10A790001BB2BDF80A20E386B1F8063512FB03F3BD
:10A7A0001E4A934230DBB3F5000F31DA002BB8BFFD
:10A7B000FF3343F30F22BDF80C30B1F808152287A0
:10A7C000164A13FB01F393421CDBB3F5000F1DDAAD
:10A7D000002BB8BFFF331B125B421BB263879FE79E
:10A7E000826890F910C0417C02F0010202AD019232
:10A7F000009560460222F9F73BF99FE7084BC8E74E
:10A80000084BC6E7074BE9E7064AD4E7044BE5E700
:10A8100047F6FF72CFE700BF388F002001FF7FFFB0
:10A820000180FFFF0080FFFF10B5044686B000687E
:10A8300000238DF80F300379012B31D0022B02D089
:10A84000002006B010BD8368D9070DF10F024CBF80
:10A850002721A721FFF74AFA0028F1D09DF80F30F1
:10A860001B07EDD52068062304AA2821FEF764FE05
:10A8700028B3BDF91030BDF91220002BB8BF033347
:10A880009B10E386BDF91430002AB8BF0332002BB9
:10A89000B8BF033392109B102287638706B010BDA8
:10A8A000826890F910C0417C02F0010201920DF122
:10A8B0000F02009260462722F9F7DAF8CCE7C4F8D5
:10A8C000360060870020BCE730B504464FF0000C2E
:10A8D0000068C4F836C0A4F83AC00379012B87B0E9
:10A8E0002AD0022B02D0002007B030BD8368D907E0
:10A8F0000DF10F024CBF61468021FFF7F7F90028E8
:10A90000F1D09DF80F301B07EDD52068062304AA6F
:10A910000121FEF711FE0028E5D0BDF81430BDF886
:10A920001010BDF812205BBA49BA52BA5B42E186F8
:10A930002287638707B030BD8568417C90F910009D
:10A9400005F0010501950DF10F0562460095F9F737
:10A950008FF8D4E710B5044600230068C4F83630F9
:10A9600063870379012B86B023D0022B02D000200D
:10A9700006B010BD8368D9070DF10F024CBF062148
:10A980008621FFF7B3F90028F1D09DF80F30DB07DF
:10A99000EDD52068062304AA0021FEF7CDFD00288E
:10A9A000E5D0049ABDF81430C4F83620638706B0A9
:10A9B00010BD826890F910C0417C02F00102019242
:10A9C0000DF10F02009260460622F9F751F8DAE71E
:10A9D00010B5044600230068C4F836306387037955
:10A9E000012B86B029D0022B02D0002006B010BD6A
:10A9F0008368D9070DF10F024CBF09218921FFF7A8
:10AA000075F90028F1D09DF80F30DB07EDD52068EF
:10AA1000062304AA0121FEF78FFD0028E5D0BDF82A
:10AA20001210BDF81020BDF81430494252425B426A
:10AA3000E1862287638706B010BD826890F910C056
:10AA4000417C02F0010201920DF10F02009260467A
:10AA50000922F9F70DF8D4E710B504460023006881
:10AA6000C4F8363063870379012B86B012D0022BED
:10AA70000DD18368DB070DF10B024CBF3421B421EB
:10AA8000FFF734F918B19DF90B30002B11DB0020D2
:10AA900006B010BD826890F910C0417C02F001023E
:10AAA00001920DF10B02009260463422F8F7E0FFAC
:10AAB000E8E72068092303AA2421FEF73DFD0028CA
:10AAC000E5D09DF810209DF80F109DF8133012046A
:10AAD00042EA0162C2F30F429DF8121022871B0462
:10AAE0009DF80D2043EA01639DF80C10120442EA20
:10AAF0000162C2F30F42C3F30F43E286638706B0DD
:10AB000010BD00BF2DE9F041DFF8BC802C4E2D4D6B
:10AB100041F0010284B000210446FEF7B1F8D8F8F4
:10AB20000070C6F80C7519E0022B3FD1A368DB0753
:10AB30000DF10F024FF0130120465EBF0DF10F0221
:10AB400093212046FFF7D2F89DF80F3085F80001D9
:10AB500013F0070319D1D6F810254ABB2379012B2E
:10AB6000E2D1A268617C94F9100002F00102019226
:10AB70000DF10F0200921322F8F77AFF9DF80F30C3
:10AB800085F8000113F00703E5D001220B212046D0
:10AB9000FEF776F8002211462046FEF771F80123F1
:10ABA00085F80001184604B0BDE8F0810020CBE72D
:10ABB000D8F8001089B2C91B8A42CFD2F2E700BF91
:10ABC000388F0020EC1600206038002010B5036894
:10ABD000DA6B82B0044612B1904740B123685B6BD8
:10ABE0001BB1214601A8984718B9FF23E38202B0A0
:10ABF00010BDBDF80630013B9BB2F7E7F0B5044647
:10AC000083B018460D4616461F4678F039FB284497
:10AC1000D4F800C0A073E673204600240094DCF84A
:10AC200014403B4632462946A04703B0F0BD00BF62
:10AC300038B58B68016004460D46984700230B4ADF
:10AC4000226123752B6B13B1204698472075084B62
:10AC500093F814351BB1237D23F0010323750023E2
:10AC6000E3822046BDE83840B0E700BF0001FF00A6
:10AC7000388F002010B5154BD3F8184584B084B137
:10AC80002379012B10D0022B0BD1A16811F0010107
:10AC9000024618BF8021204604B0BDE81040FDF7F1
:10ACA00099BF002004B010BDA268617C8DF80F0030
:10ACB00002F0010294F910000DF10F04CDE90042F9
:10ACC0008022F8F7C5FC04B010BD00BF388F00200B
:10ACD000F0B5294BD3F8185585B09DB1B02280212D
:10ACE0002846FDF7CDFF402280212846FDF7C8FF0A
:10ACF000002280212846FDF7C3FF1022802128462C
:10AD0000FDF7BEFF4FF480642DB9013CA4B2002CC6
:10AD1000FBD105B0F0BD00270DF10F062B79012BFB
:10AD200008D0022B04F1FF3217D094B2002CF0D0DF
:10AD3000012BF6D1AA6895F91000697C8DF80F7087
:10AD400002F00102013CCDE90062A4B24022F8F712
:10AD50007FFC002CE2D105B0F0BDAA68013C12F0E6
:10AD6000010218BF002240212846A4B2FDF732FF9D
:10AD7000002CD3D105B0F0BD388F00200B4B10B59F
:10AD8000D3F818458CB15038C2B280212046FDF767
:10AD900077FF002280212046FDF772FF2046102217
:10ADA000BDE810408021FDF76BBF10BD388F00203B
:10ADB000F0B5264B264CD3F81855203800EB800010
:10ADC000661D85B00444064425B90134A642FCD171
:10ADD00005B0F0BD0DF10F072B792278012B1BD0A8
:10ADE000022B0AD00134A642F7D100224021284686
:10ADF00005B0BDE8F040FDF743BFAB68DB074FF09F
:10AE00004001284619D50134FDF7E4FEA642E3D1FE
:10AE1000002DEAD105B0F0BD8DF80F20AA6895F994
:10AE20001000697C02F00102CDE900720134402279
:10AE3000F8F70EFCB442CFD1D7E70134FDF7CAFED4
:10AE4000B442C9D1002DE5D0CFE700BF388F002034
:10AE5000C45B0808F0B5754BD3F8185585B0002DC4
:10AE600000F09680D42280212846FDF709FF802239
:10AE700011462846FDF704FFA82280212846FDF749
:10AE8000FFFE3F2280212846FDF7FAFED3228021D3
:10AE90002846FDF7F5FE002280212846FDF7F0FE4A
:10AEA000402280212846FDF7EBFE8D228021284696
:10AEB000FDF7E6FE142280212846FDF7E1FEA122DF
:10AEC00080212846FDF7DCFEC82280212846FDF7B8
:10AED000D7FEDA2280212846FDF7D2FE12228021F9
:10AEE0002846FDF7CDFE812280212846FDF7C8FEC9
:10AEF000CF2280212846FDF7C3FED9228021284693
:10AF0000FDF7BEFEF12280212846FDF7B9FEDB22C7
:10AF100080212846FDF7B4FE402280212846FDF717
:10AF2000AFFEA42280212846FDF7AAFEA62280219A
:10AF30002846FDF7A5FEAF2280212846FDF7A0FE9A
:10AF4000A62280212846FDF79BFEAE2280212846BE
:10AF5000FDF796FE202280212846FDF791FE002273
:10AF600080212846FDF78CFEB02280212846FDF77F
:10AF700087FE402280212846FDF782FE00228021A4
:10AF80002846FDF77DFE102280212846FDF778FE39
:10AF90004FF4806435B9013CA4B2002CFBD10120F0
:10AFA00005B0F0BD00270DF10F062B79012B2AD03B
:10AFB000022B04F1FF3214D094B2002CF6D181227E
:10AFC00080212846FDF75CFEC82280212846FDF737
:10AFD00057FEAF2280212846FDF752FE012005B022
:10AFE000F0BDAA68013C12F0010218BF0022402106
:10AFF0002846A4B2FDF7EEFD002CD6D1002DDED1FF
:10B00000012005B0F0BDAA6895F91000697C8DF8A3
:10B010000F7002F00102013CCDE90062A4B24022AF
:10B02000F8F716FB002CC0D1C9E700BF388F00200D
:10B03000FDF788BBFDF786BBFDF784BBFDF782BB40
:10B04000FDF780BBFDF77EBB38B52B4C2B48362275
:10B05000002176F05DF8D4F81C320020984728B91A
:10B06000D4F840329847012108B938BD0021242086
:10B070004A42234B234D024000FB01441344C5F8D0
:10B080005435D4F83C229047836853B305F21C5CD6
:10B0900004886246614600230878032801F106010E
:10B0A00021D00133092BF7D1601E80B20023117823
:10B0B000022902F1060209D00133092BF7D1D5F894
:10B0C0005835082B0DD05A1CC5F85825062202FB0E
:10B0D00003CC022200238CF80020ACF80230ACF83C
:10B0E0000400012038BD062101FB0353B3F81E05FF
:10B0F000013880B2DAE700BFEC160020549400203B
:10B1000008190020388F002001207047034620B125
:10B11000026812B1D26902B1104793ED017A084B6F
:10B12000B8EEC77AD3ED016AF6EE007AE7EE267A3A
:10B13000FDEEE77A17EE900A00F30B00704700BFB0
:10B1400094940020034620B1026812B1126A02B141
:10B15000104793ED027A084BB8EEC77AD3ED026A36
:10B16000F6EE007AE7EE267AFDEEE77A17EE900A21
:10B1700000F30B00704700BF94940020034628B1F1
:10B1800002681AB1516A09B19369184793ED037ABD
:10B19000074BB8EEC77AD3ED036AF6EE007AE7EE16
:10B1A000267AFDEEE77A17EE900A00F30B0070475F
:10B1B0009494002010B5044630B1036823B1DB68D5
:10B1C00013B1BDE81040184703F0AAFAD4E90423EC
:10B1D0009042994134BF0120002010BD38B50409C8
:10B1E000013C042C1CD8104D05EB440200F00F0369
:10B1F000B2F8380440FA03F212F0010212D0012230
:10B2000002FA03F3013B1840254478F0D9FF95F882
:10B210004434064A184400EB400002EB800038BD7D
:10B22000002038BD104638BD305A0808582C002080
:10B230002DE9F04F542204460021BE4895B075F028
:10B2400067FFBD49621EE01C0C4612F8013F5D1EFF
:10B25000052D88BF0023904244F8043BF5D1B74A3E
:10B26000A2F1100353F8040B012800F059819A420F
:10B27000F8D151F8043B022B00F048819142F8D1FB
:10B280000320FBF7FDFD0420FBF7FAFD0520FBF78B
:10B29000F7FD0620AA4FA74DFBF7F2FD1A264FF047
:10B2A000000BA7F24C4A2C7B002C41D02046FFF724
:10B2B00095FF95F90D800246002800F0FF80D0F838
:10B2C0000090C6710523837109F13F4303F57E03A6
:10B2D0000AEB9323CDE9022A187C0023137267F04E
:10B2E000ABFF029A92880023114601220092484641
:10B2F000019303226EF0E6FF002317F83320A242E9
:10B300002ED00133102BF8D100218E4B296108EB90
:10B31000480803EBC8080122D8F878322B7513448B
:10B32000C8F878320723AB756A7588F8742293449D
:10B330000136F6B2202E05F10C05B4D1BBF1000F99
:10B340000BD0814D814F00262B7C7BB90136032E1B
:10B3500005F1180507F58C77F6D115B0BDE8F08F2B
:10B36000039A02EBC309D9F85014CEE7687967F065
:10B3700063FF287967F060FFD5F808904846F7F733
:10B38000D7FAD5F814802C680797142303FB08F329
:10B3900009930023CDE91033CDE9123308930A93C2
:10B3A000EB68059304F14C034FF4806206934FF46D
:10B3B0000063CDE90B234FF400514FF48073CDE9C6
:10B3C0000D1348464FF4003305A90F9367F008FFAB
:10B3D000D9F800205E495F4B42F00102C9F8002015
:10B3E0004A68134043F440334B606268B8F1010F80
:10B3F00022F04072D4BF0023012322F4807242EA7B
:10B4000003226260A168544A0A4042F00202A2602C
:10B41000E26A08F1FF33DBB222F4700242EA03531E
:10B42000E362444B4FF0010C03F148004FFA86FEF3
:10B4300002E00C33834230D05A7D002AF9D093F9D0
:10B440000D207245F5D11A7C997D092A39D8D4F896
:10B45000108002EB420A4FF0070909FA0AF901FAD3
:10B460000AF128EA090841EA08012161BCF1060F46
:10B4700039D80CF1FF31D4F8348001EB81014FF061
:10B480001F098A4009FA01F128EA01010A436263AF
:10B490000CF1010C5FFA8CFCCBE7A36843F400735A
:10B4A000A360A36843F48073A360A36843F001031F
:10B4B000A360A36843F08043A36047E7274B03934F
:10B4C0001AE7A2F10A08D4F80C9008EB48084FF0EC
:10B4D000070A01FA08F10AFA08F829EA080841EA15
:10B4E0000801E160C2E7BCF10C0F3BD8ACF10701E9
:10B4F000D4F8308001EB81014FF01F098A4009FA2E
:10B5000001F128EA01010A432263C1E7144B93F8D1
:10B51000A8202121013283F86C1083F8A820AFE61F
:10B520000F4B93F8A8002024013083F8604083F883
:10B53000A8009EE68C8F0020407E0020507E0020D8
:10B540007C5E0808EC16002050190020E48F0020D3
:10B5500000230140E030FCFFFDF7FFC0305A08082F
:10B56000388F0020ACF10D01D4F82C8001EB810163
:10B570004FF01F098A4009FA01F128EA01010A4344
:10B58000E26285E710B503681A79022A044603D0FF
:10B5900000232371236010BD987AFFF71FFE002857
:10B5A000F6D040F61A610022C18002722021FDF718
:10B5B00075FA00232371236010BD00BFF0B5066843
:10B5C000194B144606F13F4202F57E0203EB92232B
:10B5D000074683B0187C0D4667F02EFEB988B1FA95
:10B5E00081F3C3F11F03C3F3CC0206EB820203F025
:10B5F000070330469B00166A0F279C4007FA03F3A7
:10B6000026EA03031362136A1C431462C5F3001392
:10B610006A09CDE90032C5F3810305F003026EF03B
:10B6200051FE03B0F0BD00BF305A08082DE9F04FBD
:10B63000B44EB54CA64285B057D21D4602E00C363A
:10B64000A64252D273798B42F9D13379834201D029
:10B650000028F4D1F3799342F1D13468002C44D01E
:10B6600000236360A360E36023616361A361E3611E
:10B6700026603379237196F80690C4F80890327AE0
:10B68000E260012B33D0022B2FD1F07AFFF7A6FD19
:10B6900096F90970A061B07A2774FFF79FFD0646FE
:10B6A0006061F8B1DFF880A207EB87030AEB830340
:10B6B000BA00D3F8C8810092B8F1000F12D093F805
:10B6C000DA21EAB10E220023F2713372B571092139
:10B6D0003046FDF7E3F93368B2881A83204605B097
:10B6E000BDE8F08F2046FFF74DFF0024F6E7F07A23
:10B6F000FFF774FD727AB37A6374A0612274EDE788
:10B7000093F8D0B1584667F097FD4FEA5B120123DA
:10B710000BF01F0B023A03FA0BF3032A08D8DFE8F9
:10B7200002F0ADA7B30279494A6922EA03034B61EB
:10B73000BB003B440AEB830393F8CD01FFF74EFDBA
:10B74000791C0246C9B218B140F60A330172C380AF
:10B75000BB003B440AEB8303CDE9002193F8CF0102
:10B76000FFF73CFDDDE90021834620B1017240F680
:10B770000A50ABF8060009F004030093BB0003EB8A
:10B7800007090AEB8909CDE9022199F8CE01FFF7F3
:10B7900025FDDDE9022199F8D1910190002800F002
:10B7A000D580019B197240F60A41D980009B002B7D
:10B7B00070D0002A00F0C58010464A214A46FFF7A3
:10B7C000FDFEBBF1000F04D058464A462A21FFF780
:10B7D000F5FE01984A460A21FFF7F0FEBB003B4404
:10B7E0000AEB830393F8CCB1BBF1000F6AD1484B4D
:10B7F000984571D0474B984500F09880464B984546
:10B8000075D0464B984500F0BE80454B984500F0FA
:10B81000AF80444B984500F0D180009BB8F80020E1
:10B82000002B02F441520CBF03230023134343F4C3
:10B830004573A8F80030B8F81C3023F400631B04EB
:10B840001B0CA8F81C300723A8F81030B8F80030FB
:10B850009BB243F04003A8F80030BBF1000F28D1A1
:10B86000BB003B440AEB8303012283F8DA2129E77A
:10B8700026490A6A22EA03030B6259E723494A6A06
:10B8800022EA03034B6253E720490A6922EA0303D1
:10B890000B614DE722B110460A214A46FFF78EFEA2
:10B8A000BBF1000F95D058464A460A21FFF786FEA5
:10B8B0008FE75846FFF792FC0028D1D002688388B2
:10B8C0001383CDE75846FFF789FC00288FD04A46FE
:10B8D0000921FFF773FE8AE703F584335A6A42F4BD
:10B8E00080525A625A6A22F480525A6295E703F5EE
:10B8F000FE331A6A42F400421A621A6A22F40042C3
:10B900001A628AE7788C0908348E090800380240E8
:10B910000030014000380040003C0040003401404D
:10B920000050014000540140EC16002003F50033A4
:10B930001A6A42F480421A621A6A22F480421A6237
:10B940006BE7BBF1000F7FF43FAF42E7009B2BB3E7
:10B9500022B110464A214A46FFF730FEBBF1000FE4
:10B960003FF43CAF58464A462A21FFF727FE35E709
:10B9700003F568435A6A42F480125A625A6A22F402
:10B9800080125A6249E703F582335A6A42F4005240
:10B990005A625A6A22F400525A623EE7CAB110460D
:10B9A0000A214A46FFF70AFEBBF1000F3FF416AF2B
:10B9B00058464A460A21FFF701FE0FE703F56443A4
:10B9C0005A6A42F400125A625A6A22F400125A6207
:10B9D00023E7BBF1000FEBD100E700BF2DE9F047F3
:10B9E000C2B282B00E2333210220FFF71FFEDFF820
:10B9F0005CA10746CAF84801002864D00321FDF77E
:10BA000095F84FF00008C146322602F089FE044640
:10BA10000D4602F085FE001B61EB0501B0F57A7F53
:10BA200071F10001F5D3013EEFD19F23019397F906
:10BA30001030404C8DF8016003EB830304EB83036B
:10BA4000D3F8C801BB689A0758D504230DEB03024D
:10BA500069466EF091FCBB689B0738D59DF80210D3
:10BA60009DF80130344A0902002741EA03419DF85C
:10BA700003302780C4E901771943304BA7819942ED
:10BA800004D1B2F80480B2F80690012752F8083FBA
:10BA9000002BF4D1002F44D0A4F80080A4F80C901F
:10BAA000B8F1000F3DD04FEA0922A37302FB08F35F
:10BAB000C4E90123B3F1807F4FF48072628032D8F1
:10BAC00001238AF84C31384602B0BDE8F0871C4BA0
:10BAD0001C491A681C4B4FF4FA7000FB02F2A3FBDE
:10BAE0000232486892094B681B1A9A42FBD27B6962
:10BAF000002BB3D01A689B881383AFE77B6913B11F
:10BB00001A689B8853830E4B0E491A680E4B4D687A
:10BB1000D200A3FB023292094B685B1B9A42FBD214
:10BB200093E70027CFE70123B7208AF85431FBF7CA
:10BB30009BFEC5E7EC160020FC5E08081620C2003C
:10BB400084390020001000E0D34D6210407E0020B8
:10BB50002DE9F041C2B282B00E2334210220FFF75A
:10BB600065FDDFF8B8800746C8F8580180B30023A8
:10BB70000193322602F0D4FD04460D4602F0D0FDBA
:10BB8000001B61EB0501B0F57A7F71F10001F5D37F
:10BB9000013EEFD104230DEB03029F213846FDF750
:10BBA000CBFC9DF806309DF805101B4A1B0243EAAA
:10BBB00001439DF807100B4393420CD0013293428E
:10BBC00025D0C8E91F66A8F87860A8F884603046D8
:10BBD00002B0BDE8F0814FF480634FF00061A8F837
:10BBE00078304FF4006301274022A8F87A304FF4F0
:10BBF0000033C8E91F31A8F8842088F8867088F8D7
:10BC00005C71FCF795F9384602B0BDE8F0814FF45D
:10BC100000634FF08051E2E721AAEF00407E002050
:10BC20002DE9F04F85B007460093BDF838300293F8
:10BC30009DF83C3001938A469146F9F7D5FF0028DC
:10BC400000F08181C14E96F86C450B2C00F2768194
:10BC50005C2202FB04620021C2F8701582F87415A0
:10BC6000621C04EB4401D2B2C4EBC101804606F56C
:10BC7000AE6B387986F86C2503920BEB810BFFF7DE
:10BC8000ADFA054628B1039A0272022280F806A096
:10BC9000C2715C2000FB04600099C0F870854A46C0
:10BCA0004046F6F779FCD8F804309A7902F00201A0
:10BCB000003918BF012112F0040210D149004FF4DD
:10BCC000807C91464FF0010E58791B68032800F2E2
:10BCD0006F81DFE810F0E500A2005F000C004FF07C
:10BCE000000C4A004FF004096146E646ECE71A8C66
:10BCF00022F480521204120C1A841A8C988822F4AE
:10BD0000005212044EEA010E120C42EA0E319A8BD6
:10BD1000DFF840E222F4E6421204120C734580B2CE
:10BD200042F4C04200F025810EF5806E734500F0AC
:10BD3000208198809A83029A1A6419849A8B22F43B
:10BD400000621204120C42F400629A83B3F8442099
:10BD50006FEA42426FEA524292B2A3F844201A8834
:10BD600092B242F0010223F8402B5C2202FB0466EF
:10BD70000022C6F878351A60019B002B00F0D080B5
:10BD800025B13A7A02212846FFF718FC584605B03B
:10BD9000BDE8F08F4EEA0100198C21F4807109048E
:10BDA000090C1984198C21F400710904090C41EA69
:10BDB00000219888B3F81CE02EF0730E4FEA0E4E67
:10BDC0004FEA1E4E4EF06008DFF888E1734580B2FE
:10BDD00000F0C2800EF5806E734500F0BD80029ABF
:10BDE0009880A3F81C80DA6319849A8B22F00802E9
:10BDF0001204120C42F008029A83B3F844206FEA4E
:10BE000042426FEA524292B2A3F844201A8892B298
:10BE100042F0010223F83C2BA7E74EEA0100198CFF
:10BE200021F010010904090C1984198C21F020015A
:10BE30000904090C41EA00119888B3F818E02EF4BF
:10BE4000E64E4FEA0E4E4FEA1E4E4EF4C048DFF863
:10BE500004E1734580B200F09E800EF5806E73455C
:10BE600000F09980029A9880A3F818809A63198448
:10BE70001A8B22F400621204120C42F400621A833C
:10BE8000B3F844206FEA42426FEA524292B2A3F8FA
:10BE900044201A8892B242F0010223F8382B64E75A
:10BEA0004EEA0100198C21F001010904090C1984E2
:10BEB000198C21F002010904090C01439888B3F898
:10BEC00018E02EF0730E4FEA0E4E4FEA1E4E4EF063
:10BED0006008DFF880E0734580B24FD00EF5806EC9
:10BEE00073454BD0029A9880A3F818805A6319843E
:10BEF0001A8B22F008021204120C42F008021A8374
:10BF0000B3F844206FEA42426FEA524292B2A3F879
:10BF100044201A8892B242F0010223F8342B24E71D
:10BF200011212846FCF7BAFD002D3FF42FAF2B68F6
:10BF3000AA885A83584605B0BDE8F08F044A00210C
:10BF40000420F9F7A1FD4FF0000B1FE7388F002008
:10BF50004C0E09080000014021F4006141EA022171
:10BF600021F4806120F4405041EA092140EA0C109C
:10BF700035E720F4804040EA8C10DAE620F4407087
:10BF80004CEA00004FF6F37C01EA0C0C4CEA020C80
:10BF900049EA0C01A6E721F0800141EA021121F0F3
:10BFA000400120F4406041EA091140EA8C0059E761
:10BFB000B3F844206FEA42426FEA524292B2A3F8C9
:10BFC00044201A885C20002100FB046092B242F0F9
:10BFD00001021A80C0F878150960FFDE30B50368E9
:10BFE000284D294C2DED028BAB42246883B0F0EE36
:10BFF000408AB0EE608A10D005F58065AB420CD067
:10C0000005F57055AB4208D005F58065AB4204D00C
:10C0100005F58065AB4218BF6408B4FBF1F303F586
:10C020007F43FF331B0CB4FBF3F40023B4FBF1F5A7
:10C03000019200932246ABB20221FFF7F1FDE0B17D
:10C04000B5EE408A07EE904AF1EE10FAF8EE677A04
:10C050000ABF07EE105A28EE278AB8EE478A9FEDEE
:10C060000B7AC8EE076A0123037127EE667AC0EDEA
:10C07000046AA8EEA77A80ED037A03B0BDEC028BC8
:10C0800030BD00BF00000140300C002000007A44A9
:10C09000074B53F8203021B14BB11A689B8853836A
:10C0A0007047002BFCD01A689B8813837047704739
:10C0B000245A08082DE9F04F864FA7B000210A2620
:10C0C0000C4607F51C654FF0050B01968BE0BAF1A5
:10C0D000000F19D143F04003BEF18C0F87F8C43D27
:10C0E00000F2E48004F1010C98340DEB040A0CF129
:10C0F00098040DEB040C74464FF0040E0AF88CEC17
:10C100000CF88C3C04F1020EBEF18C0F42F0020CD4
:10C1100000F2CC8004F198036B4403F88BCC04F15B
:10C12000040CBCF18C0F03F88CBC00F2BF800EF144
:10C1300098060DEB060E4FF0060A0EF88CAC04EBD9
:10C140000A0E4FEA8909BEF18C0F5FFA89F603F8EF
:10C15000890C00F2AB8004F19C0CEC444FF0070911
:10C160000CF88C9C04F1080CBCF18C0F03F8876C64
:10C1700000F29C800EF198060DEB060E0EF88CBCBA
:10C1800003F8852C04F10A028C2A00F28F8004F156
:10C19000A0060DEB060C0CF88CAC03F8830C04F134
:10C1A0000C008C2800F2828004F1A20204F1A303A7
:10C1B0006A446B4402F88C9C044603F88C8C480952
:10C1C00001F01F0C55F82030012202FA0CF223EA8C
:10C1D000020345F82030019B013B01936ED00131F1
:10C1E000B1F5F07F6AD23C222846F8F71FFF011E06
:10C1F0005FDB07EB410297F8C43DB2F8FCC91CF0C5
:10C20000040FC1F30722C8B25FFA8CF94FEA1C2869
:10C2100003F0400A04F1020E7FF459AFBAF1000FA7
:10C2200003D103F0380CCC4519D003F0870343EA5F
:10C230000903BEF18C0F87F8C43D37D804F1010C17
:10C240000CF1980698346C440DEB060C4FF0040981
:10C2500004F88C9C74460CF88C3C0EF1020EBEF176
:10C260008C0F23D804F198030DEB030C231D8C2BAA
:10C270000CF88B2C0CF88CBC18D80EF198020DEB36
:10C28000020E06220EF88C2C0CF8890CA0188C28B3
:10C290000CD804F19C0304F19D026B446A4407240A
:10C2A00003F88C4C044602F88C8C88E76FF000444D
:10C2B00085E7204614B927B0BDE8F08FD7F8BC0D4C
:10C2C000234603AA00216EF0A7F8012027B0BDE89D
:10C2D000F08F00BF388F0020F0B5284CD4F8BC0D8B
:10C2E00083B010B194F8C23D0BB103B0F0BD01238F
:10C2F0000DF10702842184F8C23DFDF749FD94F851
:10C30000C42DD4F8BC0D04210A43FCF7B9FCD4F8C1
:10C31000BC0D0DF107028421FDF73AFD9DF80730B1
:10C3200013F00406F3D1164D84F8C43D3C22314687
:10C33000284674F0EDFE3246124E05F13A0005F241
:10C34000FA374FF0010E30F8023F334002F01F0180
:10C350009BB24FEA521C0EFA01F1013223B155F89B
:10C360002C300B4345F82C30B842ECD1FFF7A2FE3D
:10C370000028FBD184F8C20D03B0F0BD388F002037
:10C38000F898002004DFFFFF70B5414DD5F8BC4D93
:10C3900082B09CB395F8C03D012B43D0022B2FD126
:10C3A000082194F910303B4A85F8C31D03EB830341
:10C3B00002EB8303A2688DF80510002040F20441CF
:10C3C00092078DF80400ADF80610D3F8C80142D5E5
:10C3D00004230DEB030200216DF0CEFFA3689B0741
:10C3E00022D52D483C22FF2174F092FE95F8C13DE4
:10C3F00023B9FFF771FF012385F8C13D02B070BD7D
:10C400000DF10302A0212046FDF7C2FC9DF8033088
:10C4100003F00503012B37D0002B2FD1D5F8BC4DED
:10C420000821BEE74821BCE71C4B1D491A681D4B7B
:10C4300048684FF4FA7606FB02F2A3FB0232920937
:10C440004B681B1A9A42FBD26369002BC9D01A6849
:10C450009B881383C5E7636913B11A689B8853836C
:10C460000E4B0F491A680F4B4E68D200A3FB0232E5
:10C4700092094B689B1B9A42FBD2A9E70A4A1268B1
:10C4800040F2DC539A42B9D9D5F8BC4D482188E72F
:10C49000388F0020EC160020F89800208439002006
:10C4A000001000E0D34D6210603800202DE9F0410B
:10C4B000334D95F8C23D82B003B1FEE7012285F805
:10C4C000C22D95F8C32D044602F0F702D5F8BC0D35
:10C4D00085F8C32D0E461946FCF7D2FBE2B207469B
:10C4E0000921D5F8BC0DFCF7CBFBB4F5807F3FD01C
:10C4F000D5F8BC0DDFF88C8050220821FCF7C0FB7A
:10C50000D5F8BC0D0DF10702A021FDF741FC48B99B
:10C51000D8F88C31B8F8902159690A4214BF5A836F
:10C520001A83EDE79DF8074014F02004F0D1E2B241
:10C530000A21D5F8BC0DFCF7A3FB3219D5F8BC0DC8
:10C54000C0210134FDF724FC362CF0D157B995F801
:10C55000C32DD5F8BC0D02F0F702394685F8C32D7E
:10C56000FCF78EFB002385F8C23D02B0BDE8F081E8
:10C57000D5F8BC0D40220A21FCF782FBB8E700BFCA
:10C58000388F0020582C00202DE9F04F604D95F891
:10C59000C27DC3B007B1FEE795F8C32D044602F093
:10C5A000F7020123D5F8BC0D85F8C32D0E46394698
:10C5B00085F8C23DFCF764FBFF2C4FF009038DF8B2
:10C5C000054088BFA40801AA8CBF04F0C008B84683
:10C5D00002204FF0000C4FF00A0B0DF1050A4FF04E
:10C5E0000B09137014E0B1F5827F02F800B00AF86D
:10C5F000003016F80C3017D80CF1010CBCF1360FD6
:10C6000002F8079004F1060402F80E30084614D030
:10C61000871C48EA0C03B7F5827F00F10401044649
:10C62000DBB200F1030EDED90CF1010C6FF000411A
:10C63000BCF1360F374C0846EAD1B4F5827F63D897
:10C64000082353540DF10503A0211954831CD5F878
:10C65000BC4D314E94F9101001EB810106EB8101C4
:10C66000D1F8C801A168890722D500216DF084FEA8
:10C67000A3689B0731D5294CD5F8BC0D0DF10302F9
:10C68000A021FDF785FB48B9D4F88C31B4F890218E
:10C6900059690A4214BF5A831A83EDE79DF80330A3
:10C6A00013F02003F0D185F8C23D43B0BDE8F08F10
:10C6B000616911B10E68898871831949194F0E6833
:10C6C0001949D7F804C0F600A1FB0616B609796827
:10C6D000A1EB0C018E42FAD2C7E7114B11491A683F
:10C6E000114B48684FF4FA7606FB02F2A3FB0232C4
:10C6F00092094B681B1A9A42FBD26369002BBAD08D
:10C700001A689B881383B6E76FF000439FE700BF6A
:10C71000388F002001000080EC160020582C0020EB
:10C7200084390020001000E0D34D621038B58379C1
:10C7300013F0010F044603F02002C36B406B1FD0BF
:10C74000002A5D680CBF4221022110B12A7AFEF74F
:10C7500035FF012384F86032A4F85C326A790C4812
:10C76000296810440A8C90F8840583409BB292B2E9
:10C7700022EA03020A840A8C92B213430B8438BD66
:10C78000002A5D680CBF222102210028DED1E0E7EB
:10C79000305A0808F8B583681C686579A80744D43E
:10C7A000ED0700D4F8BD94F85C32002BFAD194F870
:10C7B0005D320133DBB2092B84F85D3277D00A2B6E
:10C7C000F0D194F85F52B4F86632002D00F08D80FD
:10C7D000980502D4DA0700F1F580B4F86A32013323
:10C7E000A4F86A3201239D42A4F85C32DAD1E66BE8
:10C7F000A179002384F85F3201F00101304666F030
:10C8000065FC7268764B5079116803440A8C93F882
:10C81000843505FA03F39BB292B222EA03020A843A
:10C820000A8C92B213430B84F8BD94F8611200296C
:10C8300034D1A26A636A94F86002934200F0918056
:10C84000531CA669A362B65C2269A779934228BFEC
:10C8500000237600A3620A2346F4007684F862324D
:10C860000123A4F8646284F8613208B13A074CD419
:10C870007B0695D50922402087EA06037608A4F8AE
:10C880006462DE07A16B2AD411B10B6889885983D1
:10C8900084F86222002883D02AB181E794F96222C9
:10C8A000002A40F09580002384F8613278E794F8FC
:10C8B0005F32002B7FF476AF94F85E32082B3FF6A0
:10C8C00071AFB4F86622012000FA03F101330A4384
:10C8D000D9B2082992B2F7D9A4F86622F8BD002986
:10C8E000D6D00B6889881983D2E743F001009905F7
:10C8F000A4F866024AD4E36A4008002B53D0216BA7
:10C90000C0B2984794F85F526CE7E26BD2F804E04B
:10C91000334A9EF80500DEF800C00244606B92F8CE
:10C9200084259340BCF8202092B222EA0303ACF89D
:10C930002030BCF820309BB2ACF8203018B19EF803
:10C940000820FEF73BFE002384F86032236CA06BC6
:10C950002BB35B681A7A00288AD00121FEF72EFEDD
:10C9600086E700287FF41CAFA37919077FF518AF7D
:10C97000216CA36B41B32BB14A680146127A184669
:10C98000FEF71CFE2046FFF7D1FE09E7B4F86A3235
:10C9900001221344A4F85C22A4F86A32F8BD0121F4
:10C9A000FCF77CF864E7E3696269C0B2D054E369DC
:10C9B000E26894F85F520133B3FBF2F102FB1133EA
:10C9C000E3610FE7184696E71846FCF767F8D9E7E2
:10C9D000A779B4F86462013A07F0400052B24BE71D
:10C9E000305A080838B504464068304B0568304A6C
:10C9F0009D421268084610D003F580639D420CD01A
:10CA000003F570539D4208D003F580639D4204D026
:10CA100003F580639D4218BF52081346B3FBF0F143
:10CA2000B1F5803F0FD289B22046F5F7B5FD2368F6
:10CA30001A685379DBB993794BB92B889BB243F0D1
:10CA400001032B8038BD012BEAD95B08E6E71A0603
:10CA50001ED41849CA18302082F800035809012250
:10CA600003F01F0302FA03F341F82030E5E719064B
:10CA700015D410485C0900EB030C012103F01F03DF
:10CA800001FA03F330218CF8001340F82430D2E788
:10CA9000094A03F00F031A4430231376CDE7064901
:10CAA00003F00F03194430230B76C4E70000014064
:10CAB000300C002000E100E0FCEC00E00346C06B1D
:10CAC00099608FE7002ABCBF80185242002B30B516
:10CAD00003EB010503DA0C465B4229462546002894
:10CAE000B7BF121A841814460020A4F11D0C0029A7
:10CAF000BCBF2B460021BCF1000FC4BFA2EB0C024F
:10CB00001418A5F10F02002AC4BF9B1A5D188442B5
:10CB10001EDBC1F1010C0F4AAC44C1EB0113CCEB9D
:10CB20000C1C00EB430301344FEA4C0C02EB4302B4
:10CB30004FF0200E8D42A8BF002304DB22F813E043
:10CB40001E339C45FAD10130A04202F10202F1D11C
:10CB500030BD00BF349900201B4B1C48196C1C4A87
:10CB600010B441F080510124196404625321FF2460
:10CB7000CA205462506251625B6FDB0085B013D4EF
:10CB80000023144902930291029A1348043202923C
:10CB9000029A136003930391039B0393039B186012
:10CBA00005B05DF8044B70470A4B002201920193D7
:10CBB000019B0193019A084B12689A42E0D105B09B
:10CBC0005DF8044B704700BF0038024000000E4281
:10CBD000002800405028004076614E692DE9F04F52
:10CBE0002DED028BAC4BAD4E1B78AD4DDFF8D0A2D6
:10CBF000B1B000270293B146BB46A6F11008D9F8A0
:10CC00000040002355F83320944203D001330E2B0B
:10CC1000F8D1FF23534493F8C83D022B00F0BD80A8
:10CC2000032B00F0B180012B09D1D9F80C3023F08F
:10CC3000807323F0080343F00403C9F80C3048461E
:10CC4000FAF766FB48B90BEB8B0308EB8303D96952
:10CC500001F00C03042B00F0AB800BF1010BBBF1D6
:10CC60000C0F09F11409CAD1DDF8088006F1F005AE
:10CC7000344608E02068E260FAF74AFC4844C7B24C
:10CC80001434A5421FD02046FAF742FB0028F7D102
:10CC9000E368590703F00C02F2D5042AF0D023F020
:10CCA000080242F00402781CB84511465FFA80F988
:10CCB00023F00403DED82068E36019461434FAF741
:10CCC00027FCA542DFD10023764FDFF8F8911D46FF
:10CCD0001C4698469B463046FAF71AFB002840F05F
:10CCE000AA80F06843076BD5029B57F80C2C43458C
:10CCF00000F2A880030765D4002D57F80C3C40F3E0
:10CD0000BF8023A900229C4602E0AA4200F0B7801F
:10CD100051F8043F1B689C4502F10102F5D1C301A3
:10CD200065D40BF1010BBBF10C0F06F1140607F1F2
:10CD30001407D0D1584B029593F80090B9F10C0F1D
:10CD400000F36B82584B594A1B791370032B40F246
:10CD5000BB801A1F022A00F29482052B00F0828207
:10CD6000062B0CBF4FF47A564FF47A66504951485F
:10CD700000224A600027504AB2FBF6F200260A6001
:10CD8000C0E900674D4AA0E0D9F80C3023F00C034D
:10CD900043F08073C9F80C3051E7D9F80C3023F018
:10CDA000807323F0040343F00803C9F80C3046E70E
:10CDB0002046FAF7ADFB0137FFB20744FFB24CE75C
:10CDC0000207ACD5002C57F80C3C4CDD17A900220B
:10CDD0009C4601E0A24245D051F8043F1B689C45A7
:10CDE00002F10102F6D1420786D4C30199D5002C85
:10CDF00057F80C3C0ADD17A9002251F8040F00680F
:10CE0000834202F101028CD0A242F6D1002D0BDD4B
:10CE100023A9002251F8040F0068834202F10102A5
:10CE20003FF47FAFAA42F5D14FF080711846F16010
:10CE3000FAF76EFB75E75B464A4601210420F8F7D6
:10CE400023FE6EE720F00801F1601046FAF760FB60
:10CE5000F06808F1010801075FFA88F8B2D44207C8
:10CE6000C3D549E76346184630AB03EB850208217A
:10CE7000F16042F8306C0135FAF74AFB51E763463E
:10CE8000184630AB03EB84020421F16042F8606C79
:10CE90000134FAF73DFB44E7A4000010FC16002023
:10CEA000084D0808081700203C410020B23F002030
:10CEB000B83F0020C03F002040420F004D750008E1
:10CEC000388F0020880E09087F4ACAF8D82D7F4A7B
:10CED00012F81330002B00F0CE81A14500F3D3816E
:10CEE000B9F1000F5CD09FED7A8ADFF828B2794E55
:10CEF0000DF15C080024784BDBF804201B7858F80F
:10CF0000040FC2F30072062B00F21F82DFE803F069
:10CF10006C635A3704040400052B00F08A816F49C2
:10CF20006F4D062B08BF29460025019200950A4641
:10CF300014230221FEF774FE0390002800F07B8189
:10CF4000039AD2F800C0DCF804E02B46DEF800704B
:10CF5000DEF81050590106EB431072586A4012F483
:10CF60007C5F03F1010300F0D780102BF2D1002386
:10CF7000CCF80C305B4B039A43F834200DE0DFED26
:10CF80005A0A5A4BB0EE600A5988FFF727F8554BFA
:10CF900043F83400002800F051810134A145AAD1A2
:10CFA0009AF8DC3D4BBB524A02210420F8F76CFD95
:10CFB0009AF8D60DB0FA80F0400931B0BDEC028B82
:10CFC000BDE8F08FDFED4B0A9FED4B0A4FF4FA619D
:10CFD000FFF704F8DBE7DFED490A4FF47A71B0EEB2
:10CFE000600AFEF7FBFFD2E79FED390AF0EE480A30
:10CFF0004FF4C871FEF7F2FFC9E79AF8DD8D9AF891
:10D00000DE3D08F10108A8EB0308B8F1120F0BDDB3
:10D010001223022100933A4A8AF8D61D4346002182
:10D020000420F8F731FDC3E79AF8E83D012B00F042
:10D030001E81022B40F00C8167F016FF314A9AF8EE
:10D04000E83DCAF8EC2D002B00F00F81022B40F0D8
:10D050000381029B122BB8BF12239BB2984500F3A9
:10D060001681029B9845A8BF9846B8F1000F9FDD36
:10D07000254EDFF8A0B0254F23AD002404E0013495
:10D08000444546F8040B93D0DBF80430BAF8E01DB1
:10D09000C3F30072BAF8E23D01920091B7FBF3F3DB
:10D0A0001A4A55F8040F9BB20321FEF7B9FD002878
:10D0B000E5D105250146164A8AF8D65D23460420A7
:10D0C000F8F7E2FC74E700BFA9890008F84C0808EB
:10D0D0006F12833A340C0020B23F0020C0C62D00EE
:10D0E000001BB700F83F0020000000003C4100207A
:10D0F000500F0908ACC5A737ACC5A7366F12033966
:10D100006C0F090865750008347F002040420F004D
:10D110000C100908AC000010037FCCF80C00002BA9
:10D120007FF428AFB7F844306FEA43436FEA5343C4
:10D130009BB2A7F844303B889BB243F080033B800E
:10D140009EF80520834B9EF806E004929A181EF084
:10D15000040F92F88425B7F820E014BF04230123BC
:10D1600093409BB21FFA8EFE2EEA030EA7F820E032
:10D170003A8C92B213433B843B8842689BB243F0A3
:10D1800001033B80744B9A4200F09380734B7448C8
:10D190001A6B42F480021A6301F118024FF0070E75
:10D1A00020F802E01A6B42F480021A6372186D488C
:10D1B00092F91430C2F818C0002BD06072DB6A4AB2
:10D1C000580902EB030C4FF0010E03F01F030EFA97
:10D1D00003F34FF0300E8CF800E342F82030314476
:10D1E0008B6805931846F5F7A3FB059B1A6822F098
:10D1F00001021A601846F5F79BFBDDE904130022D3
:10D20000CDE91222CDE914220C921092032900F2EA
:10D210009A80DFE801F096949260544ACDF800B00D
:10D2200001218AF8D61D4B4600210420F8F72CFC7A
:10D23000B6E64F4978E64F4B43F8340005218AF8AB
:10D24000D61D4D4A234600210420F8F71DFCA7E611
:10D250004A4ACAF8EC2D43B1494A02210420F8F7A2
:10D2600013FCA5E64FF4FA5680E5029BF5E667F05D
:10D27000FBFD444AE3E6444A02210420F8F704FC9B
:10D280008EE6424A21E6424A00940321C9E7029B06
:10D29000009304203F4A8AF8D60D43460021F8F750
:10D2A000F3FB85E63C4A03F00F031A443023137660
:10D2B00095E7A3F520532A481A6B42F400121A632B
:10D2C00001F118024FF0070E20F802E01A6B42F449
:10D2D00000121A636AE740371E4A0897EDB202EB64
:10D2E0008502039FD2F88825079212220B924FF4F1
:10D2F00080624FF4804C0D924FF48052CDE90E2C99
:10D300004022184607F114050A9207A94FF400328B
:10D3100011920393099565F063FF039B1A6842F02D
:10D3200010021A6028464822002173F0F1FE012302
:10D330003B71104B43F834702FE63C37CCE738375D
:10D34000CAE73437C8E70027C6E70A4A002342F88D
:10D35000343073E7305A0808006002400038024059
:10D36000380C0020D102000800E100E0A00E0908FE
:10D37000808D5B00F83F0020280F090881750008A8
:10D38000980F090825220308CC0E090849750008E2
:10D39000EC0E0908D40F0908FCEC00E010B5104CA5
:10D3A000D4E90423A16882B002FB03F38B428DF819
:10D3B000070012D06368E0680DF10701184472F0AD
:10D3C0008FFA63682269A16813446269B3FBF1F0C4
:10D3D000013201FB10336360626102B010BD00BF17
:10D3E000D03F002010B50379012B84B00C4627D024
:10D3F000022B23D18368DB070DF10F024CBF012103
:10D400008121FCF773FC9DF80F300022C3F300115B
:10D4100061F30702C3F3800161F30F220F49C3F3E5
:10D42000C00C6CF3174281F80001C3F3801161F363
:10D430001F62DB092260237104B010BD0020E2E707
:10D4400082680DF10F0102F00102CDE900121A46C7
:10D45000417C90F91000F6F70BFBD4E7EC160020A6
:10D460002DE9F04182B014460E4601AA502105462E
:10D47000FCF78EFC9DF80430DFF8F080394F013363
:10D480005B00DBB24621238001AA2846FCF780FC22
:10D4900023789DF8042008FB03F303F5FA73A7FB38
:10D4A000031301329909DB0902FB0133A280A7FBB8
:10D4B00003239B0901AAE360512102232846FCF7BC
:10D4C0003BF82378BDF8040008FB03F340BA03F5EA
:10D4D000FA73A7FB0323C2B2C0F3072082400132D4
:10D4E00092B29809DB0902FB0033A7FB03739B0987
:10D4F0007021E280238201AA2846FCF749FC9DF8AE
:10D50000043001335B00DBB201AA63807121022386
:10D510002846FCF711F8BDF80430134AF17882F878
:10D5200000015BBADAB2C3F307239A40013292B228
:10D53000228119B1E388D21A92B222810B48A378D2
:10D54000084900FB03F303F5FA73A1FB03039809F1
:10D55000DB0902FB0033A1FB03139B09638202B0CA
:10D56000BDE8F081D34D6210EC160020002F3A0088
:10D570002DE9F04FDFF89C82DFF89C92DFF89CA247
:10D58000A34F8DB0054600264FF4FA7307AA8921F0
:10D590000068C8F8103589F83C61FCF7F9FB9DF884
:10D5A0001C202868892142F00102FBF769FB324602
:10D5B00088212868FBF764FB012280212868FBF79B
:10D5C0005FFB0122FF212868FBF75AFB32463146F8
:10D5D0002868FBF755FB07AA91212868FCF7D8FBC0
:10D5E0009DF81C30286888F80B3531460122FBF77E
:10D5F00047FB3246FF212868FBF742FB3246802179
:10D600002868FBF73DFB07AA60212868FCF7C0FBF0
:10D610009DF81C202868602142F01202FBF730FBC5
:10D620004FF40053ADF81C3007AA022344212868A8
:10D63000FBF7B2FEFF2201212868FBF721FB2C68D3
:10D64000012280212046FBF71BFB0122FF212046FF
:10D65000FBF716FB324631462046FBF711FB06224C
:10D66000FF212046FBF70CFB07AA83212046FCF78D
:10D670008FFB9DF81C20832142F004022046FBF71B
:10D68000FFFA0722FF212046FBF7FAFA0122812147
:10D690002046FBF7F5FA012280212046FBF7F0FA3D
:10D6A0006B2294212046FBF7EBFA32468321204679
:10D6B000FBF7E6FADAF80060C8F80C652379012B6D
:10D6C00000F09880022B0FD000209DF81C3087F8C6
:10D6D0000001DBB9DAF800309BB29B1BB3F5FA7F8F
:10D6E000ECD90DB0BDE8F08FA368DB0707AA4FF0B7
:10D6F000830120465EBF07AA83212046FCF7F6FA85
:10D700009DF81C3087F80001002BE3D00122832113
:10D710002046FBF7B5FA07AA92212046FCF738FB12
:10D720000022812120469DF81CB0FBF7A9FA0622B1
:10D73000FF212046FBF7A4FA07AA83212046FCF725
:10D7400027FB9DF81C20832102F0FB022046FBF7FB
:10D7500097FA0122FF212046FBF792FA01220021CD
:10D760002046FBF78DFA0022FF212046FBF788FABE
:10D77000204600228021FBF783FA0623B02105AA68
:10D780002868FBF7D9FE0122FF212868FBF778FA09
:10D7900000224F212868FBF773FA2C224E212868BB
:10D7A000FBF76EFA0022FF212868FBF769FA4FEABF
:10D7B000DB162868B422B621FBF762FA0024002E9B
:10D7C00018BF0C260BF07F0BA2464FF0010EC4F3DE
:10D7D000C40330336B44E2B213F81C0C04F0070CA2
:10D7E0000EFA0CF1964220EA010119D903F81C1C2B
:10D7F0000134ECE7A268617C94F9100002F00102A8
:10D80000019207AA00928322F6F732F95DE700BF82
:10D81000EC160020388F0020407E00206038002069
:10D82000DA4540FA0CF200F01183D30744BF0AF145
:10D83000010A5FFA8AFA0134302CC8D1062305AAFE
:10D84000B0212868FBF7A8FD0122FF212868FBF71B
:10D8500017FA002211462868FBF712FA0022FF216E
:10D860002868FBF70DFA002209212868FBF708FA5F
:10D87000002210212868FBF703FA002211212868F2
:10D88000FBF7FEF9012224212868FBF7F9F9FF22B2
:10D8900025212868FBF7F4F9002275212868FBF799
:10D8A000EFF90122FF212868FBF7EAF92C224E212B
:10D8B0002868FBF7E5F9002248212868FBF7E0F922
:10D8C000214620222868FBF7DBF90022FF21286887
:10D8D000FBF7D6F9214609222868FBF7D1F9002287
:10D8E00054212868FBF7CCF9042231212868FBF782
:10D8F000C7F9032232212868FBF7C2F983224021AD
:10D900002868FBF7BDF9252246212868FBF7B8F9FE
:10D91000002260212868FBF7B3F90022272128683C
:10D92000FBF7AEF9062250212868FBF7A9F900227F
:10D9300051212868FBF7A4F9962252212868FBF7A9
:10D940009FF9082256212868FBF79AF922465721A9
:10D950002868FBF795F9002261212868FBF790F908
:10D96000002262212868FBF78BF9002264212868D5
:10D97000FBF786F9002265212868FBF781F9A022D0
:10D9800066212868FBF77CF90122FF212868FBF754
:10D9900077F9322222212868FBF772F914224721F5
:10D9A0002868FBF76DF9FF2249212868FBF768F921
:10D9B00000224A212868FBF763F90022FF2128682A
:10D9C000FBF75EF90A227A212868FBF759F9002251
:10D9D0007B212868FBF754F9212278212868FBF77E
:10D9E0004FF90122FF212868FBF74AF9342223214D
:10D9F0002868FBF745F9002242212868FBF740F927
:10DA0000FF2244212868FBF73BF92622452128689C
:10DA1000FBF736F9052246212868FBF731F9402249
:10DA200011462868FBF72CF906220E212868FBF71F
:10DA300027F91A2220212868FBF722F940224321E6
:10DA40002868FBF71DF90022FF212868FBF718F969
:10DA5000032234212868FBF713F944223521286872
:10DA6000FBF70EF90122FF212868FBF709F90422D0
:10DA700031212868FBF704F909224B212868FBF7BC
:10DA8000FFF805224C212868FBF7FAF804224D2103
:10DA90002868FBF7F5F80022FF212868FBF7F0F86B
:10DAA000002244212868FBF7EBF820224521286852
:10DAB000FBF7E6F8082247212868FBF7E1F828225F
:10DAC00048212868FBF7DCF8002267212868FBF76B
:10DAD000D7F8042270212868FBF7D2F801227121BF
:10DAE0002868FBF7CDF8FE2272212868FBF7C8F8FA
:10DAF000002276212868FBF7C3F8002277212868E6
:10DB0000FBF7BEF80122FF212868FBF7B9F80122D4
:10DB10000D212868FBF7B4F80022FF212868FBF7E5
:10DB2000AFF8012280212868FBF7AAF8F82201212A
:10DB30002868FBF7A5F80122FF212868FBF7A0F869
:10DB400001228E212868FBF79BF80122002128681A
:10DB5000FBF796F80022FF212868FBF791F80022D6
:10DB600080212868FBF78CF804220A212868FBF73B
:10DB700087F82C68842107AA2046FCF709F99DF84C
:10DB80001C20204602F0EF028421FBF779F80122E5
:10DB90000B212868FBF774F82C6803A92046FFF7CF
:10DBA00021FC07AA03A92046FFF75AFC9DF80C3078
:10DBB000002B00F05C810A9C04F684549DF80E3022
:10DBC000002B00F04A810A9B03F2B22304EB4304CA
:10DBD0009DF80F3023B1BDF82C3003F525731C449C
:10DBE0009DF8103023B1BDF82E3003F226231C44DB
:10DBF000E82201212868C8F8F04DFBF741F82868B1
:10DC000021466BF0B7FD012211462868FBF738F872
:10DC1000402187F800012868FCF774FF00283FF4D2
:10DC200060AD012128680222FBF72AF8002187F85D
:10DC300000012868FCF766FF00283FF452ADE82297
:10DC400001212868FBF71CF84FF4005307AAADF830
:10DC50001C30442102232868FBF79EFB2C6803A993
:10DC60002046FFF7BFFB07AA03A92046FFF7F8FBF2
:10DC7000502257212046FBF703F808225621204660
:10DC8000FAF7FEFF082250212046FAF7F9FFBDF807
:10DC90002C204FF47A7148F20E6301FB0233794A6B
:10DCA000934240F2EB80784AA2FB0332120C013A15
:10DCB000FF2A4FF0000306DD52080133FF2A9BB212
:10DCC000FAD81B029BB21343C3F30722DBB28DF8D1
:10DCD00008208DF8093002AA022351212046FBF7C3
:10DCE0005BFB0A9A4FF47A7148F20E6301FB023330
:10DCF000664A934200F2C080634AA2FB0332120CD0
:10DD0000013AD2B246212046FAF7BAFF2046D8F8A7
:10DD1000F01D6BF02FFD02AA01212046FCF738F818
:10DD200002229DF8086001212046FAF7A9FF002190
:10DD30002046FCF7E7FE324620460121FAF7A0FF15
:10DD40002C6803A92046FFF74DFB07AA03A920462C
:10DD5000FFF786FB482211462046FAF791FF08227A
:10DD600047212046FAF78CFF032232212046FAF79A
:10DD700087FF072230212046FAF782FF0122FF2188
:10DD80002046FAF77DFF202230212046FAF778FF5F
:10DD90000022FF212046FAF773FF06227021204659
:10DDA000FAF76EFFBDF82E10394A4FF47A7046F636
:10DDB000440300FB0133A2FB03239DF80F201B0B40
:10DDC0001AB1BDF8222013449BB2002B52D05A1E28
:10DDD000FF2A4FF0000306DD52080133FF2A9BB2F1
:10DDE000FAD81B029BB21343C3F30722DBB28DF8B0
:10DDF00008208DF8093002AA022371212046FBF782
:10DE0000CBFAD8F8F01D20466BF0B4FC02AA012131
:10DE10002046FBF7BDFF9DF8085002220121204655
:10DE2000FAF72EFF00212046FCF76CFE2A4620461A
:10DE30000121FAF725FF6422012387F80001C8F8C1
:10DE4000102589F83C310DB0BDE8F08F0EFA0CFCBE
:10DE500020EA0C0003F81C0CEDE49DF80D30002BBB
:10DE60003FF4B6AE0A9B03F525731C44B0E640F6BA
:10DE70003634A3E61A46BAE7FF2243E700231A46E0
:10DE800025E700BF1B0C0100950370F41B280D0152
:10DE90004963A41310B5174C84F8F513017952BAED
:10DEA000A4F8F62301294FF0000282B084F8F4238D
:10DEB00010D0022903D06FF00C0002B010BD042373
:10DEC00004F57D72FF21FBF70FFA0028F3D0002044
:10DED00002B010BD8268417C90F9100004F57D7499
:10DEE00002F00102CDE900420423FF22F5F7B0FB66
:10DEF000EBE700BF388F00202DE9F04F9E4F9F4B7E
:10DF00009F4D06683C464FF0000885B0834683F875
:10DF10003E815B37C4F12D0905F57D7A13E0022BB4
:10DF20000FD1B26812F0010F4FF0030352464FF0C9
:10DF3000FF01304601BF03235246FF213046FBF765
:10DF4000D3F9A7421AD0337985F8F48309EB040199
:10DF5000012B14F8012F85F8F51385F8F623DED18F
:10DF6000B368717C96F9100003F00103CDE900A3BA
:10DF7000FF220323F5F76CFBA742E4D14FF40743DC
:10DF8000A5F8F433402385F8F63352460323FF21E6
:10DF90003046FBF701FA00238DF80E300DF10E012B
:10DFA00030466BF0B1FB9DF80E30002BF6D04FF4ED
:10DFB0000643A5F8F4330123724A85F8F633FF21AE
:10DFC00003233046FBF7E8F94FF407436D4AA5F801
:10DFD000F43300240323FF21304685F8F643FBF792
:10DFE000DBF94FF40063A5F8F4330923654A85F89B
:10DFF000F633FF2103233046FBF7CEF94FF43063AD
:10E00000A5F8F4335F4A85F8F64330460323FF2131
:10E01000FBF7C2F9002800F0AD80DBF800400DF1FD
:10E020000E025E212046FBF76DFBBDF80E30B3F506
:10E03000D77F00F08D806BD8512B00F0858079D888
:10E040001D2B7FD10F2608BB0A224B212046FBF750
:10E05000C5F90F2260212046FBF7C0F90D2263218C
:10E060002046FBF7BBF9B82269212046FBF7B6F939
:10E0700040F60D7278212046FFF70CFF40F60E6245
:10E080007A212046FFF706FF00286ED0DBF800005B
:10E0900021216BF08FFADBF800400DF10E02DE213A
:10E0A0002046FBF72FFBBDF80E309FED377AC3F308
:10E0B000090303EB8303DB0007EE903AF8EEE77AFF
:10E0C0004FF4D84367EE877AA5F8F433FCEEE77A8D
:10E0D000524617EE903A1BBAC5F8F633FF210623D5
:10E0E0002046FBF759F94FF40743DBF80000A5F889
:10E0F000F433402385F8F63352460323FF21FBF720
:10E100004BF9B8B31D4B83F83E0105B0BDE8F08F65
:10E1100040F2E132934219D01CD840F2D922934206
:10E1200014D040F2E122934202D0B3F5E67FADD1A4
:10E13000642688E7AD2B0BD0D62B01D0602BA5D160
:10E14000212680E71E2BA1D114267CE7C8267AE77A
:10E15000322678E740F28F42934203D040F2915248
:10E16000934293D14FF4FA766DE7314620466BF037
:10E1700021FA8BE70020C5E7D75F0808407E002022
:10E18000388F00202C9300209A99893F044B1B78EC
:10E1900013B1044B186870476FF00100704700BF5F
:10E1A00098A400209819002070B52D4C0546032333
:10E1B0000068221D0021FBF7BFF948B96FF0010389
:10E1C000A360284AE368116832338B423ED370BDA6
:10E1D000A388A0795BBA9BB207EE903AF8EEE77A93
:10E1E000F2EE046A87EEA67A23790821BDEEC77A9B
:10E1F00084ED027A4FFA83FCBCF1000F4FEA4C0227
:10E20000A8BF5B0082F00702B4BFD3B2DBB2013912
:10E21000F0D16279082153405AB2002AB8BF5200A7
:10E220004FEA4303B6BF82F00702DBB2D3B2013933
:10E23000F2D19842C5D1A36823B1A2684FF6FF730B
:10E240009A42BED14FF0FF33A360BAE7E16028687D
:10E25000054ABDE8704001233121FBF79DB800BF9E
:10E2600098A4002060380020A8A40020014B9868E2
:10E27000704700BF98A40020437A5A1C0344D2B2CE
:10E2800042729972037A934200D97047002AFCD0F7
:10E2900010B5044604F10A01D0E900309847002384
:10E2A000637210BD2E4E3569F06980B52CF042FBCB
:10E2B00028462CF03FFBF76979798B0747D5002179
:10E2C0000846FDF7E5FE00210120FDF7E1FE254CA3
:10E2D0003B6838465B68984758B92B6828465B68A6
:10E2E0009847F8B9F7693B6838465B689847002853
:10E2F000F3D0F069D4F88C210368B4F89011DB688E
:10E30000518398472B6801461B6828469847D4F8E4
:10E310008C31B4F890211A832B6828465B689847A3
:10E320000028DFD0D4F880212B68B4F88411DB6892
:10E330005183284698470146F06903681B6898474F
:10E34000D4F88031B4F88421F7691A83C0E73B68B8
:10E3500038469B6941F002019847F769AFE700BF73
:10E3600098A40020582C002000B500680379012BE8
:10E3700085B02BD0022B23D1826812F0010F18BF79
:10E38000002103AA08BF8021FBF77EF81A4B187002
:10E3900098B1BDF80C305BBA9BB2B3F5FA6F23D2DB
:10E3A000164A1749A2FB0323DB0807EE903AF8EE62
:10E3B000E77AFDEEE77AC1ED007A05B05DF804FB7F
:10E3C0000D4B00221A7005B05DF804FB8368417C98
:10E3D00090F9100003AA03F00103CDE90023022302
:10E3E0000022F5F745FBD1E7054B4FF0FF321A60ED
:10E3F00005B05DF804FB00BF98A40020CDCCCCCCC8
:10E400009819002010B500680379012B84B00C46E0
:10E410001FD0022B02D0002004B010BD826812F081
:10E42000010F18BF002103AA08BF8021FBF72CF8B9
:10E430000028F0D05CB19DF80D309DF90C20DB096F
:10E4400003EB830302EB820203EB4203238004B05D
:10E4500010BD8368417C90F9100003F00103019323
:10E4600003AB009300220223F5F702FBE0E700BFB5
:10E4700000680379012B0CD0022B00D07047836811
:10E480000E4A13F0010F4FF0010313D00021FAF7E9
:10E490002BBF00B58268417C90F9100083B002F078
:10E4A00001020192054A00920022F5F7D1F803B06B
:10E4B0005DF804FB8021FAF717BF00BFA8A4002075
:10E4C0000FB410B582B004AB0B4C53F8042BA06C06
:10E4D0000A49019366F014FFA46C627A32B1D4E960
:10E4E000003004F10A0198470023637202B0BDE8CE
:10E4F000104004B0704700BF98A4002079E20008E3
:10E50000F8B504460F46164600252046202174F033
:10E5100077FD0446C8B10378202B03D114F8013FDE
:10E52000202BFBD02046F7F76DFFB0F5617F10DBA5
:10E5300040F63403984211DD30231A46C5B17B7092
:10E540003378013333702046F8BD002DFBD101250F
:10E55000DBE700231A46002DF1D109E0074AA0F5B8
:10E560006173A2FB0323DA08C3F3C703002DE6D1CE
:10E570003A70337801333370E9E700BF1F85EB5100
:10E5800070B5054608460E4674F07AFE31460446DC
:10E5900002462846F7F71AFC68B92B5DA3F1300252
:10E5A000092A00D870BD23F02003413B192BF9D96B
:10E5B0000134281970BD002070BD00BF03682DE92B
:10E5C000F0411F6A1FB13B46BDE8F0411847002AE1
:10E5D000164611DD04460D460E4400E023689B6894
:10E5E000204698470028F9D0236815F8011B1B68BE
:10E5F00020469847B542F1D1BDE8F081DEE700BF83
:10E60000BFF34F8F0549064BCA6802F4E06213431B
:10E61000CB60BFF34F8F00BFFDE700BF00ED00E010
:10E620000400FA0508B572B600224FF0FF319300DE
:10E6300003F1604303F561430132082AC3F88010F7
:10E64000C3F88011F3D1FFF7DBFF00BF00B583B043
:10E650000D49002200920091009B04330093009B1F
:10E660001B68012B02D003B05DF804FB01920191FD
:10E67000019B064904330193019B1A600B6883F3E5
:10E6800008884B689847FEE7502800400000FF1FAD
:10E6900010B4EFF31183102282F31288084C09485A
:10E6A00022684FF0E021013222608A69C2640022B0
:10E6B00002650A69DBB283F311885DF8044B704789
:10E6C0006038002098A4002030B4EFF311821023AA
:10E6D00083F312884FF0E023D2B29969186910F4DD
:10E6E000803F0C481EBF0121016599690A4B1D68D6
:10E6F000036D82F31188094804684FF47A7202FBB3
:10E7000004F02B44401A0021B0FBF4F030BCE3FBD2
:10E710000201704798A4002060380020843900204E
:10E72000124B5B68C3F30803F3B9EFF31183DBB952
:10E7300030B40F4A0F4C4FF0E02C1368DCF818008F
:10E7400011688B42F9D1E16C8842F6D80A4A156803
:10E750004FF47A7404FB05F20021101AB0FBF5F0B7
:10E76000E3FB040130BC7047AEE700BF00ED00E002
:10E770006038002098A400208439002090B170B542
:10E78000461EFFF7CDFF04460D46FFF7C9FF001BED
:10E7900061EB0501B0F57A7F71F10001F5D3013E1F
:10E7A000EFD270BD704700BF70B50068012209212B
:10E7B000FAF766FA6426FFF7B3FF04460D46FFF743
:10E7C000AFFF001B61EB0501B0F57A7F71F100012D
:10E7D000F5D3013EEFD170BD2DE9804883B0431CD5
:10E7E0000193DFF838810A230093D8F88011D8F814
:10E7F0008C31B8F88401B8F89021DDF804B0488372
:10E800004FF0320A1A834FF00509D8F88031B8F872
:10E81000842159690A4214BF5A831A83D8F88C316B
:10E82000B8F8902159690A4214BF5A831A83564690
:10E830005746FFF775FF04460D46FFF771FF001BB3
:10E8400061EB0501B0F57A7F71F10001F5D3013F6D
:10E85000EFD1D8F88031B8F8842159690A4214BF41
:10E860005A831A83D8F88C31B8F8902159690A4232
:10E8700014BF5A831A83FFF753FF04460D46FFF770
:10E880004FFF001B61EB0501B0F57A7F71F10001CC
:10E89000F5D3013EEFD1B9F1000F1CD0B9F1010958
:10E8A000B3D14FF4FA76FFF73BFF04460D46FFF76E
:10E8B00037FF001B61EB0501B0F57A7F71F10001B4
:10E8C000F5D3013EEFD14FF0FA0ABBF1000F07D0AC
:10E8D0004FF0000999E70BF1FF3BBBF1000FF7D1B7
:10E8E0004FF47A76FFF71CFF04460D46FFF718FF3A
:10E8F000001B61EB0501B0F57A7F71F10001F5D3E2
:10E90000013EEFD1009B013B00937FF46EAF0121EC
:10E910000846F5F723FEFFF785FE00BF582C0020C0
:10E9200018B103685B6903B11847704718B10368F1
:10E930001B6A03B118470020704700BF38B50B4D64
:10E940000C4620B10368DB6A0BB1984760B9002020
:10E95000C4E90000C4E90200C4E906552D223023B1
:10E960002061227584F8203038BD00BF5C6D090835
:10E970000178F1B1F8B50F4F0546002602E015F811
:10E98000011FA9B1BC6C637A5A1C2344D2B26272D3
:10E990009972237A9342F2D804F10A01002AEED048
:10E9A000D4E900309847667215F8011F0029E9D1B3
:10E9B000F8BD704798A4002070B504460F48FFF7D3
:10E9C000D7FF2046FFF7D4FF0D48FFF7D1FF0D4BCF
:10E9D000B3F8546016B970BD013EFCD0FFF7A0FE3D
:10E9E00004460D46FFF79CFE001B61EB0501B0F5E8
:10E9F0007A7F71F10001F5D3EEE700BF341009080A
:10EA00004811090898A4002070B5114C05460E461F
:10EA10001048FFF7ADFF2A460F49A06C334666F059
:10EA20006FFCA56C6A7A32B12B68686805F10A013F
:10EA3000984700236B7294F856303BB194F85830E5
:10EA40000122134484F8572084F8583070BD00BF69
:10EA500098A400203C10090879E200080FB470B5B2
:10EA600082B006A951F8040B0191FFF7CDFF0E48C3
:10EA7000FFF77EFF0D4BB3F8546036B902B0BDE826
:10EA8000704004B07047013EF8D0FFF749FE0446DD
:10EA90000D46FFF745FE001B61EB0501B0F57A7FDF
:10EAA00071F10001F5D3EEE74811090898A40020A0
:10EAB00070B5C379044603F007008CB015460628EC
:10EAC00000F29680DFE800F0092433353840040076
:10EAD0004C480CB0BDE87040F2E40E7813F0C0036F
:10EAE0001BD0402B21D13146237A4C2B5DD8464A8E
:10EAF00002EBC30393F8B821914256D2D3F8B43154
:10EB000053F82100002850D00CB0BDE87040D7E485
:10EB100013F0C00391F90060E3D13C483146FFF7A0
:10EB2000CFFC15B1E3793F2B4DD90CB070BD0E88E9
:10EB3000D4E7B1F90060D1E7096813F0C0030E46CD
:10EB40003DD0402BD0D0F0E791ED000A6846F7F7B2
:10EB500035FB01462B48FFF7B3FC002DE5D0E379E8
:10EB60003F2BE2D8237A284D35F9233000EE103AB6
:10EB70006846B8EEC00AF7F721FB01462448FFF7C4
:10EB80009FFCE37903F0C003402B28D0637A05EBA8
:10EB9000830393ED000AB8EE400A6846F7F70EFBD0
:10EBA00001461B48FFF78CFCBFE7694620461EF074
:10EBB00035F818486A463146FFF750FFB5E7164862
:10EBC000FFF77EFCADE7104B627A217A53F82220E2
:10EBD00033F9211011480CB0BDE8704070E4237A7D
:10EBE00005EBC30595F8B831013B00EE103AD2E7CA
:10EBF00013F0C00304D0402B97D100210E4673E7D9
:10EC00001E468AE7D81F090864600808D81D09084D
:10EC100070410908501009085416090848100908DD
:10EC2000D8B10378CBB12DE9F04F87B0704905AA70
:10EC300070F0DEFD8246002800F0CE800024DFF870
:10EC4000ECB16B4EA1462546A0464FF0FF37032C92
:10EC500032D8DFE804F0676C21046648FEE65046CF
:10EC600074F00EFB032867D19AF80020382A63D18C
:10EC70009AF80120452A00F081804E2A5CD10022BA
:10EC80009AF80230312B00F08980322B54D149EAB6
:10EC9000020242F002090FE05946504674F0FAF8B9
:10ECA000002874D045F001055349504674F0F2F83D
:10ECB000002865D045F0020505AA3146002070F015
:10ECC00097FD013482460028C1D178B24B4A002317
:10ECD00092F90010814232D00133072B02F10C026D
:10ECE000F6D1B8F1000F5CD0002D08BF032500233A
:10ECF000EDB2CDE90085CDF808901A4619462BF003
:10ED0000B5FB064600286ED03D483E4C424639468B
:10ED1000F6F780FE39463C48F6F77CFE206931461E
:10ED200062F00CFD5046F7F76DFB0746C4E750460E
:10ED3000F7F768FB8046BFE74FF0FF09BCE7314CAF
:10ED400003EB430304EB83031E6E002EC9D02F4850
:10ED50003946F6F75FFE15B17179A94228D1B9F1AC
:10ED6000000F02D0B17949452CD1F36A002BD1D0E4
:10ED70002748F6F74FFE0023F362CBE704227FE734
:10ED80002449504674F086F8002893D194E722492C
:10ED9000504674F07FF8002884D185E749EA0209DB
:10EDA0008AE71E483946F6F735FE07B0BDE8F08F12
:10EDB0002A461B48F6F72EFE3368E9B29B693046B7
:10EDC0009847CCE74A461748F6F724FE3368494689
:10EDD000DB6930469847C8E781464FF0FF3055461B
:10EDE000D046074672E739460F48F6F713FEDCE7D0
:10EDF000C87009087010090880100908F4A40020E0
:10EE0000D010090898A4002064110908F01009081E
:10EE10004C110908841009083439090888100908B8
:10EE20000811090828110908B01009087C10090800
:10EE3000A0B32DE9F04F037887B005463BB300F14E
:10EE40000040514C0138294603E09F422AD18142BB
:10EE500012D011F8013BA3F14102192A14F8012B39
:10EE6000A2F1410698BF2033192E02F12007ECD9F8
:10EE70009A4217D1002BEAD1444B0022C3F8242E2A
:10EE800083F82D2EA3F82B2E07B0BDE8F08F0021BC
:10EE9000012007B0BDE8F04F62F0AABC00210120BC
:10EEA00062F0A6BC3A4C294603E09F421AD1814247
:10EEB00012D011F8013BA3F14102192A14F8012BD9
:10EEC000A2F1410698BF2033192E02F12007ECD998
:10EED0009A4207D1002BEAD1012007B0BDE8F04FDC
:10EEE00052F06CBA2B4C294603E09F4258D1814224
:10EEF00012D011F8013BA3F14102192A14F8012B99
:10EF0000A2F1410698BF2033192E02F12007ECD957
:10EF10009A4245D1002BEAD11C4B002293F92B4E8B
:10EF200083F8242E1846164693F8D6140129A1F129
:10EF3000030509D0052D07D90EB180F82B4E1648D0
:10EF400007B0BDE8F04F89E593F8D714A52903F180
:10EF5000140303D00132782AE6D1EDE7012C03D067
:10EF6000013C64B20126F5E70C4980F8244E0023E9
:10EF7000013280F8252E81F8B03080F82B3E07B0A2
:10EF8000BDE8F04F52F07CBA94110908F07F0020E0
:10EF90009C1109085C2509087010090898A4002034
:10EFA000DFF8C8B22846F7F72DFA9BF9B0A00AFAA5
:10EFB00080F6772E074600F2DB802846202174F089
:10EFC0001FF80446002800F02A810378202B03D183
:10EFD00014F8013F202BFBD02046F7F713FA012548
:10EFE0005FFA80F82046202174F00AF804460028D1
:10EFF00000F013810378202B03D114F8013F202B5C
:10F00000FBD02046F7F7FEF901350190EDB220461E
:10F01000202173F0F5FF0446002800F0FC800378FF
:10F02000202B03D114F8013F202BFBD02046F7F70B
:10F03000E9F901350290EDB22046202173F0E0FF9E
:10F040000446002800F0E5800378202B03D114F853
:10F05000013F202BFBD02046F7F7D4F90135039070
:10F06000EDB22046202173F0CBFF0446002800F0CB
:10F07000CE800378202B03D114F8013F202BFBD046
:10F080002046F7F7BFF9013503B20493EDB22046ED
:10F09000202173F0B5FF0446002800F0B08003780B
:10F0A000202B03D114F8013F202BFBD02046F7F78B
:10F0B000A9F920210346204605931CB273F0A0FF56
:10F0C0000135059BEDB20246002859D01378202B5C
:10F0D00003D112F8013F202BFBD010460592F7F721
:10F0E00091F9059A0FFA80F92021104673F088FFF4
:10F0F00000284CD00378202B03D110F8013F202B9F
:10F10000FBD0F7F77FF905F0FD05042D08BFC3B26A
:10F110007FF415AFB8F1010F0AD9B8F1040F07D089
:10F12000A8F10502032A03D9B8F1030F7FF407AF52
:10F1300023B1A52B44D0482B7FF401AF002E39D149
:10F14000474A82F82B6E82F8D6840199C2F8C4141B
:10F150000299C2F8C8140399C2F8CC140499A2F811
:10F16000D014A2F8D244A2F8D49482F8D7348BE613
:10F170003C493D487723002207B0BDE8F04F6DE4DD
:10F18000062D7FF4DCAE8146DBB20446C2E7052DD6
:10F190007FF4D5AEB8F1010F0AD9B8F1040F07D04A
:10F1A000A8F10503032B03D9B8F1030F7FF4C7AE11
:10F1B0000346C3E72A4A06EB860602EB8602C2E74D
:10F1C00086BB2748019AC0F8C424029AC0F8C82414
:10F1D000039AC0F8CC24049A80F8D73480F8D684F7
:10F1E000A0F8D024A0F8D244A0F8D49401230AF1C6
:10F1F00001023A448BF8B02080F82B3E44E62021EF
:10F2000073F0FEFE024600287FF460AF97E604909C
:10F210003DE7039025E702900EE70190F7E60546EB
:10F220008046DFE60E48019906EB860600EB860273
:10F23000C2F8C41482F8D734029990F82B3EC2F871
:10F24000C8140399C2F8CC140133049982F8D68407
:10F25000A2F8D014A2F8D244A2F8D4945BB2C6E7C4
:10F26000F07F0020A4110908B011090898A400201B
:10F270002DE9F04782B03C4901AA70F0B9FA0028A4
:10F2800063D04FF0000A4FF0FF34374DD146564659
:10F29000D0462746BAF1040F37D8DFE80AF0423CDF
:10F2A000310B03000378482B41D0562B2DD14FF062
:10F2B000010904E0F7F7A6F83F28064625D8002004
:10F2C00001AA29460AF1010A70F092FA0028E1D158
:10F2D000BAF1040F2ED0BAF1050F40D1234AB30181
:10F2E000A92103F47C6308F03F0801FB074443EACB
:10F2F000080302EB440243EA4933A2F8B43007E0C2
:10F30000F7F780F83F288046D9D91948FFF7A6FBC0
:10F3100002B0BDE8F087F7F775F8A8280446CED903
:10F32000F3E7F7F76FF803280746C8D9EDE74FF082
:10F330000009C4E70D4AA92303FB074302EB43037B
:10F34000B3F8B490C9F34039C9E74FF0FF373C46F2
:10F35000084923463A46012062F0D6FAD8E7BAF1C6
:10F36000030FD2D0F4E700BFC870090898A40020AA
:10F37000701009084CA500202DE9F04F8FB0DFF880
:10F38000AC829E4E9E4C0091074603E00C344445EF
:10F3900000F0AF80B56C6A7A32B12B68686805F10D
:10F3A0000A01984700236B72E27902F03803BB42EE
:10F3B000ECD1934BA4EB030C924B4FEAAC0C03FB48
:10F3C0000CFC1FFA8CFCBCF11B0F40F20A818E4D25
:10F3D00001201C2302E0332800F0D68015F8011F1D
:10F3E0000B449BB29C45014600F10100F3D2874BD0
:10F3F00003EB4103B3F81C548548864B834204D386
:10F40000F8E01433834280F0F5801988C1F30B01D2
:10F41000A942F6D12046D3F808B001921DF078FC3D
:10F4200081460BEB000A20461DF0C8FC019A0146FC
:10F43000009802F0070300F02005062B14D8DFE83F
:10F4400003F0828A7A715B049300D1ED007A9AED21
:10F45000007AB4EE677AF1EE10FA0CBF01230023B4
:10F46000002D52D0002B91D102AD294620461DF02F
:10F47000D5FB009B5A0615D567482946FFF720F8AB
:10F480002B68664A934200F0828000225146204653
:10F49000FFF70EFB6248FFF76BFAB6F85430002B0B
:10F4A00040F08A805F482946FFF70AF8002251465B
:10F4B0002046FFF7FDFA5A48FFF75AFAB6F85430DB
:10F4C000002B3FF463AF9A46FFF72AF905468946B9
:10F4D000FFF726F9401B61EB0901B0F57A7F71F166
:10F4E0000001F5D3BAF1010AEED10C3444457FF4A2
:10F4F00051AF0FB0BDE8F08F0A685BF809309B1A76
:10F50000B3FA83F35B09002DACD102AD2946204646
:10F5100001931DF083FB009B5B06C3D5019B002B71
:10F52000C0D1A9E7B1F900203BF909309B1AB3FA21
:10F5300083F35B0994E70A883BF809309B1AB3FA16
:10F5400083F35B098CE70A781BF809309B1AB3FA3E
:10F5500083F35B0984E791F900201BF909309B1ABA
:10F56000B3FA83F35B097BE702F0C002402A274B22
:10F5700039D0627A53F822200132504670F0EAFC0A
:10F58000B0FA80F35B096BE74FF6FF7534E72B7930
:10F59000002B7FF47AAF1BF80930202B7FF475AF76
:10F5A00021485146FEF78CFF1D48FFF7E1F9B6F8F8
:10F5B0005430002B3FF476AF9B460194FFF7B0F830
:10F5C00004468946FFF7ACF8001B61EB0901B0F572
:10F5D0007A7F71F10001F5D3BBF1010BEED1019CF3
:10F5E00060E70A2508E7227A03EBC20393F8B82103
:10F5F000013AC1E700239B68FFDE00BF98A400200A
:10F6000058760808ABAAAAAAE86408086460080843
:10F6100050870908EC810908DC1109086E616D65E5
:10F6200048110908D0110908E8110908309508089F
:10F6300080B51848184DFFF79BF91848FFF798F95F
:10F64000AC6C627A32B12146606851F80A3B984747
:10F65000002363722F693B6838465B699847B0B9ED
:10F660000A26FFF75DF804460D46FFF759F8001B20
:10F6700061EB0503B0F57A7F73F10003F5D3013E2A
:10F68000EFD13B6838465B6998470028E8D00120F5
:10F690000BF068F8F011090898A400200C12090872
:10F6A000174B93F8FC25012A00D0704710B593F84A
:10F6B0000126062A84B00FD00A2A07D131F054FD62
:10F6C000104804B0BDE81040FFF752B90E4804B02E
:10F6D000BDE81040FFF74CB9D3F820464CB10B4AB7
:10F6E00007CA01AB03C301A91A7020460922FEF71D
:10F6F00065FF074804B0BDE81040FFF739B900BF07
:10F7000098A4002028120908181209086012090894
:10F710004412090880B52D482D4FFFF729F92D48CF
:10F72000FFF726F9B7F85460002E40D1BC6C627A1E
:10F7300032B12146606851F80A3B98470023637252
:10F74000254B00251D7087F82456C7F8645621F014
:10F7500009FC2248FFF70CF9BC6C627A2AB12146F9
:10F76000606851F80A3B984765723F693B683846C4
:10F770005B699847B0B90A26FEF7D2FF04460D46EA
:10F78000FEF7CEFF001B61EB0503B0F57A7F73F146
:10F790000003F5D3013EEFD13B6838465B699847DB
:10F7A0000028E8D000200AF0DDFF013EBED0FEF7C1
:10F7B000B7FF04460D46FEF7B3FF001B61EB0501E2
:10F7C000B0F57A7F71F10001F5D3EEE76C1209080C
:10F7D00098A4002048110908C87E00200C120908CE
:10F7E000F0B5374C94F8563091B01BB194F85730BF
:10F7F000002B4FD13348FFF7BBF8012384F86B3659
:10F8000084F8A436F7F7E4F840B9F7F7E1F828B937
:10F81000F7F7DEF810B90520FEF7DEFFF7F764F81A
:10F820000028F8D0284B29481A68C4F87826002602
:10F83000012384F8A46684F86B6684F89A36FFF78F
:10F8400097F8A56C6A7A2AB1D5E9003005F10A016A
:10F8500098476E7227693B6838465B699847B0B92C
:10F860000A26FEF75DFF04460D46FEF759FF001B12
:10F8700061EB0501B0F57A7F71F10001F5D3013E2E
:10F88000EFD13B6838465B6998470028E8D00020F4
:10F890000AF068FF94F858200D4901A8F6F7DCF843
:10F8A00001A8FFF7DBF80B48FFF7D8F8002384F82E
:10F8B000563084F8573084F8583011B0F0BD00BF8E
:10F8C00098A40020FC120908603800200C120908D6
:10F8D00098120908DC120908F8B52C4C05462C488A
:10F8E000FFF746F806F000F9012384F86B3684F838
:10F8F000A436F7F76DF840B9F7F76AF828B9F7F7C3
:10F9000067F810B90520FEF767FFF6F7EDFF00284E
:10F91000F8D0204A1168C4F878160023012228463E
:10F920001D4984F8A43684F86B3684F89A2684F846
:10F930005730FEF725FE054600B1F8BD1748FFF722
:10F9400017F8A66C727A2AB1D6E9003006F10A01DE
:10F950009847757227693B6838465B69984788B94C
:10F960000A26FEF7DDFE04460D46FEF7D9FE001B13
:10F9700061EB0501B0F57A7F71F10001F5D3013E2D
:10F98000EFD1E8E700200AF0EDFE00BF98A40020C8
:10F9900004130908603800201C1309080C12090818
:10F9A000F8B53A4B3A4F1B68D7F8A846002B6AD0F7
:10F9B0001B6A9847A28861884468521A02FB044473
:10F9C000002C4BD03348FEF7D3FF3348FEF7D0FF6F
:10F9D0003248FEF7CDFFB7F8546086BB3048FEF7DB
:10F9E000C7FFBC6C627A002A45D14FF47A76FEF7E5
:10F9F00097FE04460D46FEF793FE001B61EB0501E2
:10FA0000B0F57A7F71F10001F5D3013EEFD138698D
:10FA10002AF090FF234B1A784AB12349304651F817
:10FA200036300BB19B68186001369642F7D102213F
:10FA30000120F4F793FDFEF7F5FD013ECED0FEF771
:10FA40006FFE04460D46FEF76BFE001B61EB0501E1
:10FA5000B0F57A7F71F10001F5D3EEE71348FEF7B8
:10FA600087FFBD6C6A7A2AB12B68686805F10A01C4
:10FA700098476C72F8BD2368606804F10A019847E2
:10FA800000236372B1E70A4894E700BF8C9400201A
:10FA900098A40020341009082813090848110908FF
:10FAA0000C120908A4000010F83F002048130908B0
:10FAB00088A400202DE9F84F1A4FDFF870A0DFF876
:10FAC00070B0DFF8709007F54C7802E010374745CA
:10FAD00026D03868FEF74CFF796811B15846FEF71A
:10FAE000EFFCB96811B11048FEF7EAFC4846FEF792
:10FAF0003FFFBAF85460002EE8D0FEF711FE04462E
:10FB00000D46FEF70DFE001B61EB0501B0F57A7F97
:10FB100071F10001F5D3013EEFD110374745D8D13F
:10FB2000BDE8F88F1C6508088013090898A4002018
:10FB3000781309084811090870B50C48FEF718FF3A
:10FB40000B4BB3F8546016B970BD013EFCD0FEF704
:10FB5000E7FD04460D46FEF7E3FD001B61EB0501E2
:10FB6000B0F57A7F71F10001F5D3EEE7481109088D
:10FB700098A400202DE9F041304F3B68002B5BD06A
:10FB80001B6A98478368002B50D02D48DFF8C4804B
:10FB9000FEF7EEFE2B48FEF7EBFEB8F85460D6B940
:10FBA0003BF0A4FE3B6813B15B68984710BB64262A
:10FBB000FEF7B6FD04460D46FEF7B2FD001B61EBF5
:10FBC0000501B0F57A7F71F10001F5D3013EEFD167
:10FBD000E8E7013EE4D0FEF7A3FD04460D46FEF73C
:10FBE0009FFD001B61EB0501B0F57A7F71F100010B
:10FBF000F5D3EEE71448FEF7BBFE1248FEF7B8FE59
:10FC0000B8F854601EB9BDE8F081013EFBD0FEF7A4
:10FC100087FD04460D46FEF783FD001B61EB0501E1
:10FC2000B0F57A7F71F10001F5D3EEE70748FEF7F2
:10FC30009FFEBDE8F0417FE70548A3E78C940020D4
:10FC40009C13090848110908A81309088813090812
:10FC500088A4002098A4002070B52D4990B00522FA
:10FC6000044673F0CBFA38BB2A4C94F85630DBB11B
:10FC70002948FEF77DFE2948FEF77AFEB4F8546065
:10FC80001EB910B070BD013EFBD0FEF749FD044621
:10FC90000D46FEF745FD001B61EB0501B0F57A7FCF
:10FCA00071F10001F5D3EEE7012284F8562084F8C3
:10FCB000573084F85830DBE719490322204673F0A7
:10FCC0009DFAF0B9134C94F8563013B194F85730AC
:10FCD0006BB91448FEF74CFEFFF72EFF002384F8A3
:10FCE000563084F8573084F8583010B070BD94F80E
:10FCF00058200D4901A8F5F7AFFE01A8FEF7AEFEAA
:10FD0000ECE70A4810B0BDE87040FEF7A7BE00BFA0
:10FD1000B013090898A40020B8130908481109086D
:10FD2000682E0908D013090898120908E413090875
:10FD3000800601D5002931D10CB470B5184C194991
:10FD4000A06C82B007AB069A019365F0D9FAA56C56
:10FD50006A7A32B12B68686805F10A019847002376
:10FD60006B721148FEF704FEB4F854603EB90120EE
:10FD700002B0BDE8704002B07047013EF7D0FEF718
:10FD8000CFFC04460D46FEF7CBFC001B61EB0501E2
:10FD9000B0F57A7F71F10001F5D3EEE700207047EE
:10FDA00098A4002079E2000848110908F0B505463A
:10FDB00083B060B304785CB300F1004E444C0EF1A4
:10FDC000FF3E014603E0984236D1714513D011F849
:10FDD000013BA3F14102192A14F8012BA2F1410CB5
:10FDE00098BF2033BCF1190F02F12000EBD99A42E1
:10FDF00022D1002BE9D1374B374AC3F8AC26C3F8E0
:10FE0000B026C3F8B426C3F8B82603B0F0BD044644
:10FE1000324D334E35F8243005EB840200215288F0
:10FE20000120CDE90032234632460134FFF780FF3E
:10FE3000042CEFD103B0F0BD2846F6F7E3FA03280F
:10FE4000064639D82021284673F0DAF804460028FF
:10FE50003BD00378202B03D114F8013F202BFBD09B
:10FE60002046F6F7CFFA012705462021204673F0F9
:10FE7000C7F8D8B10378202B03D110F8013F202B0D
:10FE8000FBD0F6F7BFFA8FB1A5F2EE2240F2DC53B9
:10FE90009A420BD8A0F2EE229A4207D80D4B03EB00
:10FEA0008603A3F8AC56A3F8AE06AEE70D4803B040
:10FEB000BDE8F040FEF7D2BD0B490C4803230022F9
:10FEC00003B0BDE8F040FEF7C9BD05460746CCE7E4
:10FED0009411090898A40020E803D00744AB00203F
:10FEE000F41309087010090808140908B01109086A
:10FEF0002DE9F04385B040B3037806462BB300F1FB
:10FF0000004C574C0CF1FF3C014603E0984232D1C3
:10FF1000614512D011F8013BA3F14102192A14F8EE
:10FF2000012BA2F1410598BF2033192D02F12000C9
:10FF3000ECD99A421FD1002BEAD14A486022002115
:10FF400005B0BDE8F04371F0E3B8464D464E0024DD
:10FF5000D5E9012115F80C3B0093CDE90121234699
:10FF60003246002101200134FFF7E2FE082CEFD1D8
:10FF700005B0BDE8F0833046F6F744FAC3B2072B6C
:10FF8000054657D82021304673F03AF80446002839
:10FF900059D00378202B03D114F8013F202BFBD03C
:10FFA0002046F6F72FFA071E18BF01270126204624
:10FFB000202173F025F8044600284ED00378202B2A
:10FFC00003D114F8013F202BFBD02046F6F71AFA94
:10FFD00001368046F6B22046202173F011F804461F
:10FFE000A0B30378202B03D114F8013F202BFBD0C2
:10FFF0002046F6F707FA0136814620212046F6B260
:020000040801F1
:1000000072F0FEFF08B10136F6B2032E05D0174894
:1000100005B0BDE8F043FEF721BD154B6DB205EB11
:10002000450503EB850383F8BC76C3F8C086C3F8A7
:10003000C4969DE70F4910480723002205B0BDE88C
:10004000F043FEF70BBD06460746B0E7202172F0ED
:10005000D7FFA1460028D6D1D9E78046BBE700BF2D
:100060009411090854AB00201014090870100908F5
:1000700098A4002028140908B011090870B588B0A8
:10008000002841D003780446002B3DD000252D2BBD
:1000900054D0A3F13002092A50D9202B62D16378C1
:1000A0000134002BF3D1052DBDF914305AD19AB289
:1000B000112A57D8BDF91610A1F5FA7292B2B2F50D
:1000C000FA6F4FD8BDF91800A0F5FA7292B2B2F5E6
:1000D000FA6F47D8BDF91A40A14243DCA04241DB88
:1000E000BDF91C5005F17D0292B2FA2A3AD8204A95
:1000F00002EBC303A3F81C17A3F81E07A3F82047BD
:1001000083F8225708B070BD1A4C1B4E002594F995
:100110000600B4F90410B4F9022034F9083BCDE923
:100120000210CDE9003200212B4632460120013574
:10013000FFF7FEFD122DEAD108B070BD042D11DCD1
:100140002046F6F75FF908AB03EB4503013523F8CA
:100150000C0C14F8013FA3F13002092AF9D9002B45
:1001600095D1A0E7054808B0BDE87040FEF776BC21
:1001700098A40020B4AB00203814090870100908B6
:1001800070B58AB0064673F07BF810F0FF0414D106
:100190003B4D3C4EAB68D5E900210120CDE9012162
:1001A00000933246234600210134FFF7C1FD082C9D
:1001B00005F10C05EED10AB070BD334C06F1050C0B
:1001C000314603E098422AD1614512D011F8013B33
:1001D000A3F14102192A14F8012BA2F1410598BF9D
:1001E0002033192D02F12000ECD99A4217D1002BAF
:1001F000EAD12648264A904238BF40F2FF3103D365
:10020000D9E714309042D6D20388C3F30B038B4254
:10021000F7D11B490AB0BDE87040F6F7AFBD1D49E4
:1002200005AA30466FF0E4FA78B11A4E06AD002404
:10023000F6F7E8F805AA45F8040B3146002001342A
:100240006FF0D6FA30B1042CF2D11348FEF706FC59
:100250000AB070BD042CF8D1069B072BF5D80849CD
:10026000DDE9074003EB430301EB830241F8230080
:100270009460099B09485360FFF782FF9BE700BF2A
:1002800044AC00205014090894110908EC810908B5
:1002900050870908C8700908701009081C780908F7
:1002A0002DE9F04184B0654903AA6FF0A1FA002856
:1002B00070D0F6F7A7F80D2805462AD85F4903AA9B
:1002C00000206FF095FA002866D05D495D4E044627
:1002D00003E09E4523D1B14213D011F8013BA3F1B5
:1002E0004102192A14F8012BA2F1410C98BF2033C6
:1002F000BCF1190F02F1200EEBD99A420FD1002B5D
:10030000E9D100244D4903AA00206FF071FA0028BA
:100310007BD04D48FEF7A2FB04B0BDE8F0814B490D
:100320004B4F044603E09C4516D1B94212D011F858
:10033000013BA3F14102192A14F8012BA2F1410655
:1003400098BF2033192E02F1200CECD99A4203D128
:10035000002BEAD10124D5E73E49DFF810C104465D
:1003600003E09F4235D1614512D011F8013BA3F162
:100370004102192A14F8012BA2F1410698BF20333B
:10038000192E02F12007ECD99A4222D1002BEAD192
:100390000224B7E74FF0FF35DFF8CC802E4F2F4E09
:1003A00000240EE03B5D08EB83033246D3F8E837C8
:1003B00000930021234601200134FFF7B9FC0E2CE5
:1003C000AAD06B1CEED0AC42ECD001340E2CFAD18A
:1003D000A2E72349234F03E09E429AD1B94212D0AB
:1003E00011F8013BA3F14102192A10F8012BA2F1E7
:1003F000410498BF2033192C02F12006ECD99A420F
:1004000087D1002BEAD103247CE7134E164FDFF887
:100410004C8074550446AC420BD1335D07EB83032B
:100420004246D3F8E8370093002123460120FFF726
:100430007FFC01340E2CEED16EE700BFC8700908B6
:100440006414090863140988701009086C140908F9
:100450006B140988F86A0908009D002074140908C3
:100460001C6709081B67098864600808F76A09881F
:1004700010F040002FD00CB470B50C4682B029B1FA
:10048000002002B0BDE8704002B07047174EB56C56
:100490006B7A5A1C2B44D2B223216A7299722B7A3E
:1004A000934219D9069A124907AB2846019364F082
:1004B00027FFB46C627A32B1D4E9003004F10A014A
:1004C000984700236372FFF737FB012002B0BDE8B5
:1004D000704002B070477047002AE3D0D5E9003081
:1004E00005F10A0198476C72B56CDBE798A400200F
:1004F00079E200082DE9F04FDFF8F0A087B09346CD
:1005000081460D46164600270AF2FC744FF0190882
:1005100095F800C0BBF1000F52D03078604551D043
:100520000021002302E001333D2B5AD004EBC3022B
:100530004FEAC30C12798242F5D1F37805914FF45A
:10054000617218FB03230393B378D44418FB03238D
:1005500002939CF8013872784846CDE90032224A6D
:100560003B46FFF785FF95F800C00599002302E0A0
:1005700001333D2B35D004EBC302D800127962451C
:10058000F6D1EB784FF4617218FB03230393AB7839
:10059000504418FB032302936A7890F801384846C8
:1005A000CDE900323B46104A0137FFF7C1FB282F47
:1005B00005F1040506F10406AAD107B0BDE8F08FE5
:1005C0005946D3E76A7873789A42A9D1AA78B37862
:1005D0009A42A5D1E978F378C91AB1FA81F14909AB
:1005E0009FE700235B79FFDE8C140908646008082C
:1005F000002871D0F0B5037883B00446002B43D0B7
:10060000F5F700FF272805466ADC0023601C20213F
:100610008DF8073072F0F4FCAE00044658B1037850
:10062000202B03D114F8013F202BFBD02046F5F7F7
:10063000E9FE002834DA2046202172F0E1FC04466D
:10064000A0B10378202B03D114F8013F202BFBD05D
:100650002046F5F7D7FE1D2808D8264B334483F8EB
:100660000D089DF8073001338DF80730224FB11C7B
:100670000DF1070239442046FDF742FF9DF807308F
:10068000042B08D103B0F0BD1B490022012003B0A8
:10069000BDE8F0402EE7002347F8253003B0F0BD59
:1006A000164FC2B2002307F2FC7001E03D2BC2D00E
:1006B00000EBC3014FEAC30C4979914203F10103F6
:1006C000F4D101238DF807300A4B6744334497F87F
:1006D000002883F80C28AEE707490022012009E72B
:1006E000074908482723002203B0BDE8F040FEF781
:1006F000B5B900BF98A40020A4AC0020646008082D
:1007000040170908B01109082DE9F04F89B0434E90
:10071000434F079092460C46154602F1540894F94F
:100720000430404A92F90010994202F10C0209D0BB
:100730009642F7D10C35454504F10C04EFD109B0D0
:10074000BDE8F08FBAF1000F51D095F904E0D5F86B
:1007500000B06A79A879297A95F807C0734548D01E
:100760004FF0000907EB8C0C07EB8101DCF8E43952
:10077000049307EB8000D1F8E439039307EB82027E
:10078000D0F8E4390293D2F8E4390193264A079865
:10079000CDF800B073464946FFF76AFE94F904307D
:1007A000E279D4F800C007EB82024946D2F8E42986
:1007B0000492227A07EB82020C35D2F8E4290392E4
:1007C000A27907EB82020C34D2F8E429029214F8E1
:1007D000070C154ACDF800C007EB8000D0F8E409FB
:1007E00001900798FFF7A4FA454598D1A7E7D146AD
:1007F000D6E723685B45B3D163799342B0D1A3793F
:100800008342ADD1237A8B42AAD194F80790A9EB09
:100810000C09B9FA89F94FEA5919A3E748A500204C
:1008200064600808F4A40020A0140908D8B1027874
:10083000CAB12DE9F04F87B0451CF5F7E3FD5A4CDE
:10084000014647B22246002392F90460BE4202F1FB
:100850000C020CD00133072BF6D1544807B0BDE889
:10086000F04FFEF7FBB85049002201204CE703EBA4
:10087000430304EB830494E8070003AE86E8070013
:1008800007462021284672F0BBFB834600287DD016
:100890000278202A03D11BF8012F202AFBD02B2A13
:1008A00039D02D2A66D05846F5F7ACFD022307460D
:1008B0000093E37994F8059094F8068094F808A0E2
:1008C000019300255846202172F09AFB83460028A8
:1008D00045D00278202A03D11BF8012F202AFBD013
:1008E0005846F5F78FFD002203461146304804E0D4
:1008F0000132112A1AD050F8041F9942F8D1022D62
:100900005FFA82FC16D0032D16D0012D14BFE146EC
:10091000E0460135D6E70BF1010B5846F5F772FDBD
:1009200001228240022317430093C2E7BBB9022D84
:100930009C46E8D1E246ECE7002369F3070368F33D
:100940000F236CF317436AF31F630397CDF811303D
:1009500096E8070084E8070007B0BDE8F08F009B29
:100960002B44DBB2012B14D1124807B0BDE8F04F85
:10097000FEF774B80BF1010B5846F5F743FD012261
:100980008240022327EA0207009392E701230093A3
:100990008FE70023019A69F3070368F30F2362F3DB
:1009A00017436AF31F63D0E7E07E0020C0140908F4
:1009B000486A0808701009082DE9F04F89B0DFF87F
:1009C000D0A0079281460C46154600264FF0190824
:1009D0004FF461773AE0A97894F802B02B786A78FE
:1009E000E87895F804C095F805E08B4534D04FF0D1
:1009F000000B18FB027218FB0373CDE90232CDE93C
:100A0000040CCDE900E13346524659464846FFF70B
:100A10002FFD23790593E37804936278237818FBFC
:100A2000027218FB0373CDE90232A3780193637954
:100A3000009352463346594648460136FFF778F947
:100A4000142E04F1060405F106051ED0079B002BA9
:100A5000C1D1DDF81CB0DCE794F800B09B45C6D1ED
:100A600094F801B09345C2D194F803B08345BED148
:100A700094F804B0E345BAD194F805B0ABEB0E0B93
:100A8000BBFA8BFB4FEA5B1BB3E709B0BDE8F08F05
:100A9000D4140908002800F0AD802DE9F047037850
:100AA00082B00446002B71D0F5F7ACFC1328054644
:100AB00000F3A48000EB40060023601C20218DF889
:100AC000073072F09DFADFF850814FEA46096F0057
:100AD00008EB4606044658B10378202B03D114F8DE
:100AE000013F202BFBD02046F5F78CFC032877D95B
:100AF0002046202172F084FA044658B10378202B56
:100B000003D114F8013F202BFBD02046F5F77AFCE7
:100B10001D2859D920460DF107023146FDF7F0FC9A
:100B2000202172F06DFA0446002870D00378202B43
:100B300003D114F8013F202BFBD02046F5F762FCCF
:100B40003C289DF807A032D92046202172F058FA9F
:100B5000B0B10378202B03D110F8013F202BFBD03C
:100B6000F5F750FC1D280BD82A4B2F440AF1010A37
:100B700003EB47035FFA8AFA8DF807A083F8B00801
:100B8000BAF1060F09D102B0BDE8F0872249002270
:100B9000012002B0BDE8F0470EE72048002348F8E6
:100BA0000930B38002B0BDE8F047FDF757BF194BDD
:100BB0007A190AF1010A03EB42035FFA8AFA8DF807
:100BC00007A083F8AF08BFE79DF80720114B01325B
:100BD0008DF807207A1903EB420383F8AE0899E7F2
:100BE0000C4B7A1903EB420383F8B10801238DF80B
:100BF00007307DE7084900220120DDE60849094861
:100C00001323002202B0BDE8F047FDF727BF9DF88F
:100C100007A099E798A4002044AD002070100908AF
:100C200040170908B01109082DE9F04F2DED088B88
:100C300099B082460C461546002607925DE0F4EE18
:100C40004A8AF1EE10FA74D1B4EE6A9AF1EE10FA13
:100C50006FD1F4EE4B9AF1EE10FA0CBF0121002196
:100C600014A80691F5F7AAFAB0EE4A0A074610A8AA
:100C7000F5F7A4FA0DF130098346B0EE6A0A48464A
:100C8000F5F79CFA0DF120080590B0EE4B0A4046AE
:100C9000F5F794FA059A0390CDE901B206992B4A2B
:100CA000009733465046FFF7E3FBB0EE480A14A81E
:100CB000F5F784FAB0EE680A074610A8F5F77EFA51
:100CC000B0EE490A83464846F5F778FAB0EE690A6D
:100CD00081464046F5F772FA3346CDE90290CDE9F8
:100CE000007B1A4A002150460136FFF721F80C2EEE
:100CF00004F1100405F1100522D094ED008AB5EE40
:100D0000408AF1EE10FA1BD0079BD4ED018A94EDD6
:100D1000029AD4ED039A73B195ED000A95ED01AAFC
:100D2000D5ED02AA95ED03BAB4EE408AF1EE10FAC1
:100D300085D0002194E70DF130090DF12008B4E7CA
:100D400019B0BDEC088BBDE8F08F00BFF4140908A2
:100D50002DE9F04198B30378054683B36D4C00F15B
:100D6000050E014603E0984237D1714513D011F8C2
:100D7000013BA3F14102192A14F8012BA2F1410C05
:100D800098BF2033BCF1190F02F12000EBD99A4231
:100D900023D1002BE9D1604A92F87E1C4FF4D67023
:100DA00000FB01F102F6241302F6E4120B440A449C
:100DB0000021596110339342FBD1BDE8F0815649BF
:100DC00091F87E3C4FF4D67000FB0311BDE8F04172
:100DD000002201F63811012026E72846F5F712FB1C
:100DE0000B28064600F28B802021284672F008F975
:100DF0000446002800F08B800378202B03D114F8E0
:100E0000013F202BFBD02046F5F748FA424B93F8E0
:100E10007E2C4FF4D670711C00FB02F203F62413F3
:100E200002EB0112134483ED010A01252046202123
:100E300072F0E6F80446C8B10378202B03D114F809
:100E4000013F202BFBD02046F5F728FA324B03F662
:100E5000241293F87E3C4FF4D67101FB03F3711C0E
:100E600003EB01131344013583ED020A20462021D0
:100E700072F0C6F80446C0B10378202B03D114F8F1
:100E8000013F202BFBD02046F5F708FA224B03F652
:100E9000241293F87E3C4FF4D67101FB03F303EB6D
:100EA00006131344013583ED070A2021204672F012
:100EB000A7F8C0B10378202B03D110F8013F202BF5
:100EC000FBD0154C94F87E7CF5F7E8F94FF4D67317
:100ED00007FB03F304F6241403EB06162644032D44
:100EE00086ED080A04D0BDE8F0410C48FDF7B6BD18
:100EF0001433E1180022BDE8F041012094E6BDE87A
:100F0000F041074907480B230022FDF7A7BD05461E
:100F10008CE700BF9411090898A4002070100908FC
:100F200040170908B01109082DE9F04F91B0DFF81A
:100F300034B1079282460C469046002509AF0BAEAD
:100F40003AE01A4643493046F4F786FD079B002BEA
:100F500049D098F800C02378634547D04FF0000986
:100F60003D4B059300230493B8F912300393B8F96D
:100F700010303A4A02930192CDF800C02B465A46EF
:100F800049465046FFF774FA0597237D0493B4F958
:100F900012300393B4F9102014F8203B0093CDE9EC
:100FA00001622B465A46494650460135FEF7C0FEBF
:100FB000082D08F120084AD004F1150904224946F9
:100FC000384672F0C9F90022A3688DF82820E2683B
:100FD000082B72F10001B4D321493046F4F73CFDEF
:100FE000079B002BB5D1DDF81C90CDE7D4E90202B8
:100FF000D8E902139A4208BF8842AFD1227D98F8FF
:1010000014309A42AAD199F8002098F815309A42E3
:10101000A4D199F8012098F816309A4209F10109F3
:101020009CD119F8012F98F817309A4296D199F867
:10103000012098F818309A4290D12269D8F81030DF
:10104000A2EB0309B9FA89F94FEA591988E711B0F7
:10105000BDE8F08FD81D09081C780908C0190908D7
:10106000081509081415090898B32DE9F04F0378FD
:1010700083B0804633B300F1004CA54D0CF1FF3C2A
:10108000014603E0984228D1614512D011F8013B96
:10109000A3F14102192A15F8012BA2F1410798BFCB
:1010A0002033192F02F12000ECD99A4215D1002BE0
:1010B000EAD198484FF48072002103B0BDE8F04FA8
:1010C00070F026B893490022012003B0BDE8F04F2C
:1010D0002AE790490022012026E74046F5F792F9D9
:1010E00083B2072B074600F2EE802021404671F0C4
:1010F00087FF8146002800F0F8800378202B03D179
:1011000019F8013F202BFBD04846F5F77BF9012564
:101110000FFA80F82021484671F072FF002800F095
:10112000E7800378202B03D110F8013F202BFBD060
:10113000002B00F0E7800026014600F1100C344639
:10114000A3F13002D2B2092AA3F1610E0CD9BEF18B
:10115000050FA3F15702A3F1410E04D9BEF1050F0B
:1011600011D8A3F13702D2B211F8013F240144EAA9
:10117000167442EA0616002B00F0B480202B00F013
:10118000B1806145DCD1002301930135EDB220210E
:1011900071F036FF8246002800F0B2800378202BE1
:1011A00003D11AF8013F202BFBD05046F5F72AF95E
:1011B00001350FFA80F9EDB25046202171F020FF81
:1011C0008346002800F09A800378202B03D11BF877
:1011D000013F202BFBD05846F5F714F901350FFAE3
:1011E00080FAEDB25846202171F00AFF83460028AC
:1011F00000F082800278202A03D11BF8012F202AD8
:10120000FBD05846F5F7FEF8013543B20093EDB236
:101210005846202171F0F4FE034600286AD0027877
:10122000202A03D113F8012F202AFBD00135EDB27B
:10123000032D51D91FFA88F2022A4DD809F226222D
:1012400092B2B2F5E16F47D80AF2262292B2B2F515
:10125000E16F41D89DF800B0BBF1060F3CD81846AD
:10126000009372F00DF8042836D8019B002B33D080
:10127000294A009B294D3FB202F54B6178010E507F
:1012800001EB47114C6002EB47110A4681F8A88C2C
:10129000A1F8B89CA1F8BAAC81F8BCBC02F6BC427B
:1012A000591E033311F8010F2C5C04F00304022CC7
:1012B00008BF203802F8010F087808B19942F1D12F
:1012C00003B0BDE8F08F164916480723002203B08B
:1012D000BDE8F04FFDF7C2BB134803B0BDE8F04FC7
:1012E000FDF7BCBB012301934FE70546804611E79C
:1012F00001904CE70D4B9BE7009089E7824671E730
:10130000814659E71E461C46012301933DE700BF75
:101310009411090840B1002098A400205107090841
:1013200038150908B0110908701009081C78090857
:101330002DE9F04FDFF8AC9087B0924680460C461E
:1013400015460026BAF1000F35D06B7A617AB5F9EF
:101350000AC0B5F90CE095F808B09942D5E900202B
:101360002BD00027CDE90020CDE9023CCDE904EBEC
:1013700033464A4639464046FFF77AF8237A0593C2
:10138000B4F90C300493B4F90A300393637A0293EE
:10139000626854F8103B3946CDE900324046334686
:1013A0004A460136FEF7C4FC112E05F11005C9D1DD
:1013B00007B0BDE8F08F5746E0E721689142D0D1F1
:1013C00061688142CDD1B4F90A106145C9D1B4F93F
:1013D0000C107145C5D1277AA7EB0B07B7FA87F731
:1013E0007F09BFE748150908A0B32DE9F04F03783E
:1013F00083B005463BB300F1004E804C0EF1FF3E3A
:10140000014603E0984229D1714513D011F8013B00
:10141000A3F14102192A14F8012BA2F1410C98BF43
:101420002033BCF1190F02F12000EBD99A4215D1FB
:10143000002BE9D172484FF48872002103B0BDE857
:10144000F04F6FF065BE6E490022012003B0BDE889
:10145000F04F6DE76A490022012069E72846F4F75A
:10146000D1FFC3B2102B064600F2AC8020212846E3
:1014700071F0C6FD0446002800F0B1800378202BEF
:1014800003D114F8013F202BFBD02046F4F7BAFF1C
:10149000012507462046202171F0B2FD04460028B0
:1014A00000F09B800378202B03D114F8013F202B00
:1014B000FBD02046F4F7A6FF01358046EDB220466A
:1014C000202171F09DFD0446002800F084800378FF
:1014D000202B03D114F8013F202BFBD02046F4F73A
:1014E00091FF0128814667D80135EDB220462021C1
:1014F00071F086FD0446002874D00378202B03D1B8
:1015000014F8013F202BFBD02046F4F77BFF00F5B9
:10151000B473B3F5347F82464ED80135EDB2204620
:10152000202171F06DFD834600285DD00378202BCB
:1015300003D11BF8013F202BFBD05846F4F762FF84
:1015400000F5B473B3F5347F044635D80135EDB2F8
:101550005846202171F054FD8346002846D0037878
:10156000202B03D11BF8013F202BFBD05846F4F76A
:1015700049FF031E18BF012301355846202101935E
:10158000EDB271F03DFD08B10135EDB2062D13D17C
:101590001C4B019A76B203EB0613C3F8A87DC3F87F
:1015A000AC8D83F8B19DA3F8B2ADA3F8B44D83F828
:1015B000B02D03B0BDE8F08F134803B0BDE8F04F85
:1015C000FDF74CBA114912481023002203B0BDE8C0
:1015D000F04FFDF743BA814688E780466FE705463E
:1015E000074657E782469AE70446B1E7202171F0A3
:1015F00007FD0028E0D0CDF804B0C5E79411090834
:1016000040B2002098A4002070100908681509084D
:10161000B01109082DE9F047DFF8B4A088B0904672
:1016200081460C4615460026B8F1000F34D098F8D4
:101630000D20637B9A4231D00027AB7B05936B7BF7
:1016400004932B7B0393AB6802936B6801936A78D6
:101650002B780092394652464846FEF709FFA37B95
:101660000693637B0593237B0493A36803936368CA
:101670000293627814F8103B3946CDE900324846AF
:10168000334652460136FEF753FB3F2E05F1100557
:10169000CAD108B0BDE8F0874746E0E72288B8F82D
:1016A00000309A42C8D1A268D8F808309A42C3D113
:1016B0006268D8F804309A42BED1E368D8F80C20AA
:1016C000534033F07F430CBF01270027B5E700BF2D
:1016D0007C1509082DE9F04F8FB00C460992079050
:1016E0001546002630E02868BDF828100C9080B21E
:1016F000AB88ADF834308142B5F9023095F801C0BD
:1017000095F804E02A7834D00021CDE9023ECDE9F5
:10171000002C07981E4ACDF8108033460891FEF73A
:10172000A7FE08991A4A0798CDF800903346CDE9EC
:1017300003B8CDE901A70136FEF7FAFA242E04F129
:10174000060405F106051FD0B4F90270A3882068CD
:1017500094F801A094F804B094F9058094F80090EE
:101760000A90ADF82C307FB1099B002BBBD10999B1
:10177000D8E79F42C8D1BDF82C10BDF83400091A33
:10178000B1FA81F14909C0E70FB0BDE8F08F00BFA1
:101790009C150908F0B589B0064671F071FD10F08E
:1017A000FF020DD1474991F87E3C4FF4D67000FB03
:1017B000031101F6F811012009B0BDE8F04089E7F6
:1017C000414C751D314603E09E452AD1A94213D0F4
:1017D00011F8013BA3F14102192A14F8012BA2F1DF
:1017E000410C98BF2033BCF1190F02F1200EEBD948
:1017F0009A4216D1002BE9D1324A344B92F87E1C22
:101800004FF4D67000FB01221868998802F6F8138D
:1018100002F52D621860998006339A42FAD109B018
:10182000F0BD2B4901AA30466DF0E2FF4FF0FF33C7
:10183000079380B1264E02AD0024F4F7E3FD034682
:1018400045F8043B002001AA314601346DF0D0FF79
:1018500030B1062CF1D11F48FDF700F909B0F0BDF9
:10186000042CF8DD029B232BF5D8039A112AF2D819
:10187000049C3C2CEFD8059F07F57A71B1F5FA6FFF
:10188000E9D8069EFF2EE6D8079D691C4029E2D8BC
:101890000C4991F87E0C4FF4D67E0EFB00F04FF011
:1018A000060E0EFB03030B440B4883F8F82983F85C
:1018B000F949A3F8FA7983F8FC6983F8FD59FFF731
:1018C00069FFACE798A40020941109088C6A080805
:1018D000C8700908701009081C7809082DE9F04F34
:1018E0009FB098460F908B4692464FF00009109299
:1018F0000AE0C8450BD009F10109B9F1400F0BF11D
:10190000140B0AF1140A7AD0B8F1FF3FF1D15D4609
:101910000FCD14AC0FC42B6823609BF813300B93CE
:101920009BF810300C939BF911300D939BF81230FB
:10193000DBF808200E93109B0A929BF80C209BF872
:10194000047008900992002B46D0DAF80030119309
:10195000DAF80830129356469AF8133013930FCEE4
:1019600019AD0FC5189C33689AF804C09AF80CE0BA
:101970002B605C4034F07F442CD167452ED00B9B0C
:1019800007930A9B0693099B0593089B1D4A0F9892
:10199000CDE903730E9B02930D9B01930C9B009367
:1019A00021464B46FEF764FD0B9B07930A9B06936B
:1019B000099B0593089B134A0F98CDE903730E9B6F
:1019C00002930D9B01930C9B009321464B46FEF71F
:1019D000AFF990E70024D2E7109CE5E7089B83422B
:1019E000CDD1099B7345CAD10A9B129A9342C6D1A5
:1019F0000B9B139A9C1AB4FA84F46409BFE71FB0D6
:101A0000BDE8F08FB41509082DE9F0418AB005460C
:101A10000C4671F035FC10F0FF0011D1524991F8DD
:101A2000562022B1631C3BD10AB0BDE8F0814FF0D3
:101A3000FF3301F6B86101200AB0BDE8F0414DE77F
:101A40004A4C681D294603E09E452CD1884213D09C
:101A500011F8013BA3F14102192A14F8012BA2F15C
:101A6000410C98BF2033BCF1190F02F1200EEBD9C5
:101A70009A4218D1002BE9D13D483E4A904203D307
:101A8000D2E714309042CFD20388C3F30B03B3F5EF
:101A90007E7FF6D138490AB0BDE8F041F5F76EB95E
:101AA00023460246C5E735496A4628466DF0A0FE42
:101AB00078B1324E6D460024F4F7A4FC6A4645F82E
:101AC000040F3146002001346DF092FE38B1092C2C
:101AD000F2D12B48FCF7C2FF0AB0BDE8F081092C17
:101AE000F7D101993F29F4D8029B012BF1D8039833
:101AF000421C402AEDD8049F382FEAD8DDF814E0C4
:101B0000BEF1070FE5D8DDF818C01E4C0CF57422A5
:101B100002F51072A242DCD8079E072ED9D8089D84
:101B200005F5742202F51072A242D2D8099CFF2C4E
:101B3000CFD80D4A4FF0140808FB012209B282F8F1
:101B4000C90E114882F8C83E82F8CA7E82F8BCEEFF
:101B5000C2F8B8CE82F8C46EC2F8C05E82F8CB4E2E
:101B6000FFF752FF60E700BF98A400209411090816
:101B7000EC8109085087090850B30020C870090893
:101B80007010090880841E001C7809084FF0FF318E
:101B90003AE700BF2DE9F04FA5B08B461190924671
:101BA0004FF000091292DBF808300C939BF80C30D0
:101BB0000B93BBF810300D93BBF812300E93BBF8AB
:101BC00014300F935D46BBF8163010930FCD16AC52
:101BD0000FC495E80700129BDBF800709BF80480A7
:101BE0009BF8186084E80700002B4DD0DAF800302D
:101BF0001393DAF80830159355469AF80C3014937D
:101C00000FCD1DAC0FC495E807009AF818E09AF8BC
:101C100004C0B64584E8070038D00024109B089320
:101C20000F9B07930E9B06930D9B05930C9B0493B0
:101C30000B9B214A1198CDE90273CDE900684B4610
